:100000000C9473240C94A2240C94A2240C94A22487
:100010000C94A2240C94A2240C94A2240C94A22448
:100020000C94A2240C94A2240C94A2240C94A22438
:100030000C94A2240C947B4A0C94A2240C94A22429
:100040000C94A2240C94A2240C94A2240C94A22418
:100050000C94A2240C94A2240C94A2240C94A22408
:100060000C94A2240C94FAD50C94A2240C9426D6B9
:100070000C94A2240C94569E0C94A2240C94A224BA
:100080000C94A2240C94A2240C94A2240C94A224D8
:100090000C94A2240C94A2240C94A2240C94A224C8
:1000A0000C94A2240C94A2240C94A2240C94A224B8
:1000B0000C94A2240C94A2240C94A2240C94DD474A
:1000C0000C94A2240C94A2240C94A2240C94A22498
:1000D0000C94A2240C94A2240C94A2240C94A22488
:1000E0000C94A2241D4045404A4027404F409C406C
:1000F0009C4027406D409C4072407A407F40844045
:1001000059405E406340274068409C402240544034
:1001100089408E4092409C409C4096405072657051
:100120006172696E6720666F7220736C6565703AE4
:1001300049276D20636F6D706C6574696E6720610F
:100140006E792020717565756564206D6F766573B5
:100150002E20202020202020004368616E67696ED9
:10016000672046696C616D656E743A202049276D81
:1001700020636F6D706C6574696E6720616E7920A5
:1001800020717565756564206D6F7665732E20200E
:10019000202020202000494E56414C494420544FF5
:1001A0004F4C3A2020202020202049207265636592
:1001B000697665642061204C656674202020546F48
:1001C0006F6C20636F6D6D616E642C20627574209E
:1001D00049206F6E6C792068617665206F6E6520AE
:1001E000546F6F6C2E2000494E56414C49442043B9
:1001F0004F4D4D414E443A202020204920726563E6
:100200006569766564206120636F6D6D616E6466FB
:100210006F7220612068656174656420706C617420
:10022000652C20627574204920646F6E27742068E5
:10023000617665206F6E65004920736177206120CB
:10024000676C6974636820696E206D79534420631C
:100250006172642E20496620746869732069732076
:10026000746865206669727374206572726F722C8F
:100270002074727974686973206D6F64656C206195
:100280006761696E2E20202000492074696D6564C5
:10029000206F7574207768696C6520202061747404
:1002A000656D7074696E6720746F20686561742075
:1002B000206D792065787472756465722E20202017
:1002C000202020202000492074696D6564206F750E
:1002D00074207768696C65202020617474656D7086
:1002E00074696E6720746F206865617420206D7971
:1002F00020706C6174666F726D2E2020202020208B
:10030000202000507265706172696E6720666F729E
:1003100020736C6565703A49276D20636F6F6C6957
:100320006E67206D7920202020202068656174652B
:10033000727320616E6420676F696E6720746F6DE1
:1003400079207761697420706F736974696F6E2E9C
:10035000202020004368616E67696E672046696CE3
:10036000616D656E743A202049276D20676F696E54
:100370006720746F206D792077616974706F73697D
:1003800074696F6E2E202020202020202020202025
:10039000004D7920686561746572732074696D65BC
:1003A00064206F75744920616D206E6F7720696ECF
:1003B00020536C65657020202028436F6C642050AA
:1003C00061757365292E20202020202020202020E8
:1003D000202020202020202020202020202020201D
:1003E000200052657374617274696E672074686569
:1003F000204275696C640054686973206973206ECB
:100400006F7420746865207833672076657273692D
:100410006F6E204920776F726B206265737420774E
:100420006974682E20466F722068656C7020736551
:10043000653A206D616B6572626F742E636F6D2F0C
:1004400068656C70202020005468697320627569AB
:100450006C6420697320666F72202020616E6F7457
:1004600068657220626F742E205365653A202020E3
:100470006D616B6572626F742E636F6D2F68656C52
:100480007020202000546865205265706C6963619B
:100490007430720049276D2043616E63656C6C692E
:1004A0006E672E2020202020506C656173652057D8
:1004B0006169742E20202020202020200020004868
:1004C0006561746572732073687574646F776E20EC
:1004D00020202064756520746F20696E61637469E3
:1004E000766974792020200048656174696E672000
:1004F0004661696C7572652023312120536F6674E3
:10050000776172652054656D70204C696D69742047
:10051000526561636865642120506C656173652074
:100520002020202053687574646F776E206F7220CE
:1005300052657374617274200048656174696E67F6
:10054000204661696C75726520233221204D792027
:1005500065787472756465727320617265206E6F60
:100560007468656174696E672070726F7065726C13
:10057000792E202020436865636B206D7920636F9E
:100580006E6E656374696F6E730048656174696E41
:1005900067204661696C75726520233321204D798F
:1005A00020657874727564657273206172652020AD
:1005B00020206C6F73696E672074656D7065726161
:1005C000747572652E20436865636B206D792063B6
:1005D0006F6E6E656374696F6E73004865617469F0
:1005E0006E67204661696C7572652023352120494C
:1005F000276D2072656164696E67206F7574206F66
:1006000066202072616E67652074656D7065726129
:1006100074757265732E20436865636B206D792055
:10062000636F6E6E656374696F6E730048656174A5
:10063000696E67204661696C7572652023342120DC
:100640004D792074656D7065726174757265207284
:1006500065616473617265206661696C696E6721AA
:1006600020506C6561736520436865636B206D790C
:1006700020636F6E6E656374696F6E7300930269B9
:100680000000006900EE016900000069002601B861
:10069000010000000020065500000055002D0855FF
:1006A00000000055004D0A550000005500400CABFD
:1006B000000000AB002D095500000055002D085525
:1006C00000000055004D0AAB00000055000000007E
:1006D00001C00D5500000055002D08560100000016
:1006E00000C00D20015311BC005B12B101000000DD
:1006F00000C00DC80000001400C00DC800000014A8
:1007000000910E9001000014005A10900100001496
:1007100000C00D200300000000C805C80000001440
:1007200000C805C80000001400C805C80000001477
:1007300000DD04B004000014007505C800000014BA
:10074000007505C800000014007505C800000014FD
:10075000009704B00400000000B8075500000055E1
:1007600000B909AB000000AB007D06550000005544
:1007700000C805550000005500B807AB000000ABED
:1007800000C805550000005500DD04550000005567
:1007900000C805550000005500B807550000005579
:1007A000007D065601000000003F03550000005583
:1007B00000FA0C5500000055003F0355000000559D
:1007C00000B9095500000055003F035500000055D1
:1007D000002D095500000055003F0355000000554D
:1007E00000EA0A5500000055003F0355000000557F
:1007F00000B909AB0000000000534420436172645B
:100800002052656D6F766564202020200024F4045A
:10081000D9201BC40C5C0E9804C4095F02650771E3
:1008200001F405F900FB04B30048048700C1036923
:10083000005803550003034500BE023A008402310C
:100840000053022A002902250004022000E4011CB2
:1008500000C8011900AF01170098011400840113AA
:1008600000710110006101100051010E0043010DE3
:100870000036010B002B010B0020010B00150109B4
:10088000000C01090003010800FB000800F3000848
:1008900000EB000700E4000600DE000600D80006BA
:1008A00000D2000600CC000500C7000500C200050C
:1008B00000BD000400B9000400B5000400B100044C
:1008C00000AD000400A9000400A5000300A200037D
:1008D000009F0004009B00030098000300950002A5
:1008E0000093000300900003008D0002008B0003C2
:1008F00000880002008600020084000300810002DC
:10090000007F0002007D0002007B000200790002EF
:1009100000770001007600020074000200720001FE
:1009200000710002006F0002006D0001006C000207
:10093000006A000100690002006700010066000112
:100940000065000100640002006200010061000116
:1009500000600001005F0002005D0001005C00011A
:10096000005B0001005A000100590001005800011D
:10097000005700010056000100550001005400011D
:10098000005300000053000100520001005100011B
:1009900000500001004F0001004E0000004E000119
:1009A000004D0001004C0001004B0000004B000115
:1009B000004A000100490001004800000048000111
:1009C000004700010046000000460001004500000D
:1009D0000045000100440001004300000043000105
:1009E00000420000004200010041000000410001FF
:1009F00000400001003F0000003F0001003E0000F9
:100A0000003E0001003D0000003D0001003C0000F0
:100A1000003C0000003C0001003B0000003B0001E6
:100A2000003A0000003A00010039000000390001DE
:100A300000380000003800000038000100370000D6
:100A400000370001003600000036000000360001CB
:100A500000350000003500000035000100340000C2
:100A600000340000003400010033000000330000B7
:100A700000330001003200000032000000320001AB
:100A800000310000003100000031000100300000A2
:100A90000030000000300001002F0000002F000097
:100AA000002F0000002F0001002E0000002E00008B
:100AB000002E0001002D0000002D0000002D000080
:100AC000002D0001002C0000002C0000002C000074
:100AD000002C0001002B0000002B0000002B000068
:100AE000002B0001002A0000002A0000002A00005C
:100AF000002A000100290000002900000029000050
:100B00000029000000290001002800000028000042
:100B10000028000000280000002800010027000035
:100B20000027000000270000002700000027000128
:100B3000002600000026000000260000002600001D
:100B4000002600010025000000250000002500000F
:100B50000025000000250000002500010024000001
:100B600000240000002400000024000000240001F4
:100B700000230000002300000023000000230000E9
:100B800000230000002300000023000100220000D9
:100B900000220000002200000022000000220000CD
:100BA00000220001002100000021000000210000BF
:100BB00000210000002100000021000000210001B0
:100BC00000200000002000000020000000200000A5
:100BD0000020000000200000002000000020000194
:100BE000001F0000001F0000001F0000001F000089
:100BF000001F0000001F0000001F0001001E000079
:100C0000001E0000001E0000001E00000024F4D49E
:100C10003050C38E20C2A24017828B7011127A917D
:100C20000D816CD90AA861E108C758660761514374
:100C3000061E4B5D05C145A7041A411104093D98E4
:100C400003713931034036DB0265339102D43054ED
:100C500002802E1D02632CEE01752AC501B028A06A
:100C600001102781018F2564012B244B01E02234E0
:100C700001AC211F018D200D01801FFC00841EEDA1
:100C800000971DDF00B81CD200E61BC600201BBC6D
:100C900000641AB200B219A8000A19A0006A1899D3
:100CA00000D117910040178B00B516840031167ED5
:100CB00000B31579003A157300C7146F0058146A11
:100CC00000EE1366008813630025135E00C7125BF5
:100CD000006C12570015125400C111510070114FD1
:100CE0000021114B00D61049008D104700461044DA
:100CF0000002104200C00F4000800F3E00420F3C37
:100D000000060F3B00CB0E3800930E37005C0E350B
:100D100000270E3400F30D3200C10D3100900D306C
:100D200000600D2E00320D2D00050D2C00D90C2B6E
:100D300000AE0C2900850C29005C0C2700350C271F
:100D4000000E0C2600E80B2400C40B2400A00B238B
:100D5000007D0B23005A0B2100390B2100180B20BA
:100D600000F80A1F00D90A1E00BB0A1E009D0A1DBA
:100D700000800A1D00630A1C00470A1B002C0A1B86
:100D800000110A1A00F7091A00DD091900C409192F
:100D900000AB091900920917007B091800630917B5
:100DA000004C09160036091600200916000A09151C
:100DB00000F5081500E0081400CC081400B8081469
:100DC00000A4081400900813007D0812006B08139B
:100DD00000580812004608120034081100230811B8
:100DE000001208110001081100F0071000E00710C0
:100DF00000D0071000C0071000B0070F00A10710B7
:100E00000091070E0083070F0074070F0065070E9F
:100E10000057070E0049070E003B070D002E070E76
:100E20000020070D0013070D0006070D00F9060C42
:100E300000ED060D00E0060C00D4060C00C8060C00
:100E400000BC060C00B0060C00A4060B0099060CB2
:100E5000008D060B0082060B0077060B006C060B5C
:100E60000061060A0057060B004C060A0042060AFB
:100E70000038060A002E060A0024060A001A060A8E
:100E8000001006090007060A00FD050900F405091F
:100E900000EB050900E2050900D9050900D00509A4
:100EA00000C7050900BE050900B5050800AD050825
:100EB00000A50509009C050800940508008C05089C
:100EC00000840508007C050800740508006C05070F
:100ED00000650508005D050700560508004E05077A
:100EE00000470507004005080038050700310507E1
:100EF000002A050700230507001C05060016050744
:100F0000000F0507000805060002050700FB0406A0
:100F100000F5040700EE040600E8040600E20407FA
:100F200000DB040600D5040600CF040600C9040651
:100F300000C3040600BD040600B7040600B10405A2
:100F400000AC040600A6040600A00405009B0406ED
:100F50000095040500900406008A04050085040538
:100F600000800406007A040500750405007004057D
:100F7000006B04050066040500610405005C0405BF
:100F80000057040500520405004D040500480405FF
:100F900000430405003E0404003A0405003504053E
:100FA00000300404002C0405002704040023040579
:100FB000001E0404001A04040016040500110404B1
:100FC000000D0404000904050004040400000404E6
:100FD00000FC030400F8030400F4030400F003041D
:100FE00000EC030400E8030400E4030400E003044D
:100FF00000DC030400D8030400D4030400D003047D
:1010000000CC030400C8030300C5030300950200DD
:101010000000506C6561736520776169742E2E2E17
:101020000084036901000014008304880000001498
:10103000008C000000000000000030F8FFFF0000FE
:101040000000000000008E00000000000000000012
:1010500000000000000000000000005729040018F4
:101060008304DC0500001400901F891F9502000016
:1010700000506C6561736520776169740084037D3D
:10108000010000140083048800000014008C00009C
:1010900000000000000030F8FFFF0000000000002A
:1010A00000008E00000000000000000000000000B2
:1010B0000000000000000057290400188304DC052C
:1010C000000014008C97340000F3190000000000A9
:1010D00000000000000000000095000000005469BE
:1010E000676874656E2065616368206F6620746848
:1010F00065200095010000007468726565206B6EC4
:101100006F627320756E6465722020200095010067
:101110000000746865206275696C6420706C61748D
:10112000666F726D202000950700000061626F7588
:101130007420666F7572207475726E732E00950040
:1011400000000049276D20676F696E6720746F206B
:101150006D6F7665206D79009501000000657874EB
:1011600072756465722061726F756E6420746F2091
:1011700020009501000000646966666572656E7402
:1011800020706F696E747320736F200095070000E4
:1011900000796F752063616E20636865636B2E2E26
:1011A0002E00950000000074686520686569676816
:1011B000742E204174206561636820009501000051
:1011C00000706F696E742C206C6F6F73656E207485
:1011D0006865202020009501000000737065636938
:1011E00066696564206B6E6F6220756E74696C0051
:1011F0009507000000746865206E6F7A7A6C652030
:10120000616C6D6F73742E2E2E00950000000074BB
:101210006F756368657320746865206275696C64B6
:10122000202020009501000000706C6174652E2064
:10123000546865206E6F7A7A6C6520697300950139
:10124000000000617420746865207269676874200A
:101250006865696768742000950700000077686515
:101260006E2061207468696E2070696563652E2E3A
:101270002E0095000000006F66207061706572207E
:1012800077696C6C20736C696465200095010000BF
:10129000006265747765656E20746865206E6F7A8C
:1012A0007A6C652020009501000000616E64206268
:1012B00075696C6420706C6174652077697468006E
:1012C000950700000020736F6D6520667269637476
:1012D000696F6E2E009502000000506C65617365A9
:1012E0002077616974008E97340000F3190000D0F4
:1012F00007000000000000000000009AE903001849
:101300008E0000000038180000D007000000000028
:1013100000000000006C692E00188E0000000038EC
:10132000180000000000000000000000000000E0C5
:1013300093040018950000000041646A75737420DE
:101340007468652072656172206B6E6F6200950132
:10135000000000756E74696C207061706572206A9F
:1013600075737420202020009501000000736C69C3
:10137000646573206265747765656E2074686520A6
:10138000200095070000006E6F7A7A6C6520616E10
:101390006420706C617465009502000000506C65FB
:1013A0006173652077616974008E00000000381851
:1013B0000000D00700000000000000000000E093E3
:1013C0000400188E9C100000C8E7FFFFD007000043
:1013D0000000000000000000802A2D00188E9B10E5
:1013E0000000C8E7FFFF0000000000000000000050
:1013F0000000E093040018950000000041646A7545
:1014000073742066726F6E7420726967687420202E
:101410000095010000006B6E6F6220756E74696C40
:10142000207061706572202020200095010000006E
:101430006A75737420736C69646573206265747770
:1014400065656E200095070000006E6F7A7A6C6506
:1014500020616E6420706C6174650095020000006C
:10146000506C656173652077616974008E9C100013
:1014700000C8E7FFFFD007000000000000000000E8
:1014800000E0930400188E64EFFFFFC8E7FFFFD071
:101490000700000000000000000000004C1D0018C4
:1014A0008E65EFFFFFC8E7FFFF00000000000000AF
:1014B0000000000000E093040018950000000041C7
:1014C000646A7573742066726F6E74206C656674DE
:1014D0002020200095010000006B6E6F6220756E69
:1014E00074696C2070617065722020202000950165
:1014F0000000006A75737420736C69646573206200
:1015000065747765656E200095070000006E6F7A40
:101510007A6C6520616E6420706C61746500950260
:10152000000000506C656173652077616974008EFE
:1015300064EFFFFFC8E7FFFFD007000000000000D6
:1015400000000000E09304001895000000004E6FBA
:10155000772049276D20676F696E6720746F2020A0
:10156000202000950100000073656E64206D7920D5
:10157000657874727564657220746F20009501003F
:101580000000616C6C20746872656520706F696E14
:1015900074732020202000950700000061676169B6
:1015A0006E20746F207265636865636B2E00950210
:1015B000000000506C656173652077616974008E6E
:1015C0000000000038180000D007000000000000F4
:1015D0000000000080191B00188E00000000381861
:1015E0000000000000000000000000000000E09388
:1015F000040018950000000041646A75737420743B
:10160000686520726561722020202020009501000D
:1016100000006B6E6F6220756E74696C2070617073
:101620006572202020200095010000006A75737407
:1016300020736C69646573206265747765656E20DC
:101640000095070000006E6F7A7A6C6520616E6409
:1016500020706C617465009502000000506C65613B
:1016600073652077616974008E00000000381800EF
:1016700000D00700000000000000000000E093041C
:1016800000188E402B0000C8E7FFFFD007000000C5
:1016900000000000000000A65D2200188E3F2B0015
:1016A00000C8E7FFFF00000000000000000000008D
:1016B00000E093040018950000000041646A75730F
:1016C000742066726F6E74207269676874202000DF
:1016D00095010000006B6E6F6220756E74696C205E
:1016E0007061706572202020200095010000006A62
:1016F00075737420736C69646573206265747765B3
:10170000656E200095070000006E6F7A7A6C652088
:10171000616E6420706C6174650095020000005079
:101720006C656173652077616974008E402B0000E1
:10173000C8E7FFFFD0070000000000000000000025
:10174000E0930400188EC0D4FFFFC7E7FFFFD00767
:1017500000000000000000000000C0C62D00188E30
:10176000C1D4FFFFC8E7FFFF000000000000000039
:1017700000000000E09304001895000000004164A0
:101780006A7573742066726F6E74206C656674205F
:1017900020200095010000006B6E6F6220756E7452
:1017A000696C207061706572202020200095010016
:1017B00000006A75737420736C69646573206265D8
:1017C000747765656E200095070000006E6F7A7A69
:1017D0006C6520616E6420706C6174650095020018
:1017E0000000506C656173652077616974008EC07C
:1017F000D4FFFFC8E7FFFFD0070000000000000093
:10180000000000E0930400188E00000000000000BB
:1018100000D00700000000000000000000913B1A0B
:1018200000188E0000000000000000000000000012
:1018300000000000000000E0930400189500000084
:10184000004E6F77206C6574277320747269706C1A
:101850006520202020009501000000636865636B0F
:101860002D2D2070617065722073686F756C640037
:1018700095010000006A75737420736C69646520BB
:101880006265747765656E20200095070000006E24
:101890006F7A7A6C6520616E6420706C617465008B
:1018A000891F9502000000506C65617365207761A7
:1018B00069740084037D0100001400830488000023
:1018C0000014008C000000000000000030F8FFFF52
:1018D00000000000000000008E000000000000007A
:1018E0000000000000000000000000000057290474
:1018F00000188304DC05000014008C97340000F30A
:101900001900000000000000000000000000009529
:10191000000000005469676874656E206561636843
:10192000206F6620746865200095010000007468CF
:10193000726565206B6E6F627320756E64657220D0
:101940002020009501000000746865206275696CB4
:101950006420706C6174666F726D202000950700C2
:10196000000061626F757420666F75722074757205
:101970006E732E00950000000049276D20676F6987
:101980006E6720746F206D6F7665206D790095010C
:1019900000000065787472756465722061726F75FD
:1019A0006E6420746F202000950100000064696659
:1019B000666572656E7420706F696E747320736FE4
:1019C00020009507000000796F752063616E206329
:1019D0006865636B2E2E2E0095000000007468650C
:1019E000206865696768742E2041742065616368AA
:1019F00020009501000000706F696E742C206C6FE0
:101A00006F73656E207468652020200095010000CA
:101A100000737065636966696564206B6E6F622030
:101A2000756E74696C009507000000746865206E1F
:101A30006F7A7A6C6520616C6D6F73742E2E2E0038
:101A40009500000000746F756368657320746865A5
:101A5000206275696C6420202000950100000070F0
:101A60006C6174652E20546865206E6F7A7A6C659F
:101A7000206973009501000000617420746865207E
:101A800072696768742068656967687420009507E3
:101A90000000007768656E2061207468696E2070B0
:101AA000696563652E2E2E0095000000006F66208C
:101AB00070617065722077696C6C20736C69646505
:101AC000200095010000006265747765656E2074E2
:101AD0006865206E6F7A7A6C6520200095010000A1
:101AE00000616E64206275696C6420706C6174655D
:101AF000207769746800950700000020736F6D659A
:101B0000206672696374696F6E2E00950200000092
:101B1000506C656173652077616974008E9734003D
:101B200000F2190000D007000000000000000000D3
:101B3000009AE90300188EB605000039180000D09D
:101B400007000000000000000000002461290018C8
:101B50008EB50500003818000000000000000000ED
:101B60000000000000E09304001895000000004110
:101B7000646A757374207468652072656172206B85
:101B80006E6F62009501000000756E74696C2070C4
:101B900061706572206A75737420202020009501A1
:101BA000000000736C696465732062657477656515
:101BB0006E2074686520200095070000006E6F7A23
:101BC0007A6C6520616E6420706C617465009502AA
:101BD000000000506C656173652077616974008E48
:101BE000B505000038180000D00700000000000014
:101BF00000000000E0930400188E51160000C8E7B2
:101C0000FFFFD00700000000000000000000802A55
:101C10002D00188E51160000C8E7FFFF00000000DD
:101C20000000000000000000E09304001895000090
:101C3000000041646A7573742066726F6E7420725E
:101C40006967687420200095010000006B6E6F6268
:101C500020756E74696C2070617065722020202080
:101C60000095010000006A75737420736C696465E7
:101C700073206265747765656E200095070000002B
:101C80006E6F7A7A6C6520616E6420706C61746529
:101C9000009502000000506C6561736520776169F2
:101CA00074008E51160000C7E7FFFFD00700000048
:101CB00000000000000000E0930400188E69F4FFAB
:101CC000FFC8E7FFFFD00700000000000000000091
:101CD000003FE81D00188E69F4FFFFC8E7FFFF0012
:101CE0000000000000000000000000E09304001865
:101CF000950000000041646A7573742066726F6E0F
:101D000074206C6566742020200095010000006B33
:101D10006E6F6220756E74696C20706170657220E0
:101D20002020200095010000006A75737420736CF8
:101D300069646573206265747765656E2000950738
:101D40000000006E6F7A7A6C6520616E6420706CA2
:101D5000617465009502000000506C656173652038
:101D600077616974008E69F4FFFFC8E7FFFFD00751
:101D700000000000000000000000E093040018953F
:101D8000000000004E6F772049276D20676F696E55
:101D90006720746F202020200095010000007365EB
:101DA0006E64206D79206578747275646572207434
:101DB0006F20009501000000616C6C2074687265F2
:101DC0006520706F696E74732020202000950700D5
:101DD0000000616761696E20746F207265636865D9
:101DE000636B2E009502000000506C6561736520E6
:101DF00077616974008EB505000038180000D007BF
:101E00000000000000000000000078381B00188E61
:101E1000B6050000381800000000000000000000B7
:101E200000000000E09304001895000000004164E9
:101E30006A75737420746865207265617220202051
:101E400020200095010000006B6E6F6220756E749B
:101E5000696C20706170657220202020009501005F
:101E600000006A75737420736C6964657320626521
:101E7000747765656E200095070000006E6F7A7AB2
:101E80006C6520616E6420706C6174650095020061
:101E90000000506C656173652077616974008EB5D0
:101EA00005000038180000D0070000000000000006
:101EB000000000E0930400188E2C290000C8E7FF02
:101EC000FFD007000000000000000000005AC51FFE
:101ED00000188E2D290000C8E7FFFF000000000059
:101EE00000000000000000E09304001895000000CE
:101EF0000041646A7573742066726F6E7420726933
:101F000067687420200095010000006B6E6F6220EE
:101F1000756E74696C2070617065722020202000DD
:101F200095010000006A75737420736C69646573B1
:101F3000206265747765656E200095070000006E6D
:101F40006F7A7A6C6520616E6420706C61746500D4
:101F50009502000000506C656173652077616974BB
:101F6000008E2C290000C8E7FFFFD007000000000A
:101F7000000000000000E0930400188E12E2FFFF52
:101F8000C8E7FFFFD00700000000000000000000CD
:101F9000D0A02500188E13E2FFFFC8E7FFFF000066
:101FA00000000000000000000000E093040018950D
:101FB0000000000041646A7573742066726F6E746D
:101FC000206C6566742020200095010000006B6E77
:101FD0006F6220756E74696C20706170657220206C
:101FE00020200095010000006A75737420736C69ED
:101FF000646573206265747765656E2000950700DF
:1020000000006E6F7A7A6C6520616E6420706C617E
:102010007465009502000000506C6561736520775F
:10202000616974008E12E2FFFFC8E7FFFFD007006E
:10203000000000000000000000E0930400188EB5CE
:1020400005000000000000D00700000000000000B4
:1020500000000095CD1600188EB6050000000000A7
:1020600000000000000000000000000000E09304F9
:10207000001895000000004E6F77206C6574277380
:1020800020747269706C652020202000950100008A
:1020900000636865636B2D2D20706170657220731D
:1020A000686F756C640095010000006A7573742098
:1020B000736C696465206265747765656E202000C5
:1020C00095070000006E6F7A7A6C6520616E64205F
:1020D000706C61746500891F99000000006E6F7A52
:1020E0007A6C6543616C6962726174696F6E0096A7
:1020F0000000860084035201000014008304A6003F
:10210000000014008C000000000000000030F8FF08
:10211000FF00000000000000008B00000000000035
:102120000000000000000000000000000000A60009
:1021300000008304DC0500001400901F8C9734001D
:1021400000F2190000000000000000000000000084
:10215000008B40D9FFFFBFE6FFFF60EA00000000F0
:1021600000000000000080000000910114910014A4
:1021700091041491031488001F026E008D00640006
:10218000580288000302E60088010302E600870087
:102190006400580287016400580291017F91007F1A
:1021A00091047F91037F8BC8E7FFFF09EBFFFF6876
:1021B0000100000000000000000000800000008B13
:1021C000C8E7FFFF09EBFFFF68010000E4FFFFFF26
:1021D000000000000C0300008BC8E7FFFF09EBFFC5
:1021E000FFF0000000D0FFFFFF000000003E0000F5
:1021F000008BC8E7FFFF09EBFFFFF0000000B3FF13
:10220000FFFF00000000850100008BF1D9FFFF09EE
:10221000EBFFFFF00000004FFEFFFF000000007F1B
:102220000300008BC8E7FFFF88EEFFFFF00000000F
:102230007FFEFFFF00000000D30000008BC8E7FF17
:10224000FF88EEFFFFF000000063FEFFFF000000CC
:1022500000850100008B67DDFFFF88EEFFFFF000C7
:102260000000FEFCFFFF00000000820300008BC89E
:10227000E7FFFF06F2FFFFF00000002EFDFFFF006A
:10228000000000D80000008BC8E7FFFF06F2FFFF48
:10229000F000000012FDFFFF0000000085010000BB
:1022A0008B67DDFFFF06F2FFFFF0000000ADFBFFD4
:1022B000FF00000000820300008BC8E7FFFF85F5E8
:1022C000FFFFF0000000DDFBFFFF00000000D80072
:1022D00000008BC8E7FFFF85F5FFFFF0000000C19D
:1022E000FBFFFF00000000850100008B67DDFFFFA2
:1022F00085F5FFFFF00000005CFAFFFF0000000022
:10230000820300008BC8E7FFFF03F9FFFFF0000026
:10231000008DFAFFFF00000000D80000008BC8E726
:10232000FFFF03F9FFFFF000000070FAFFFF00005D
:102330000000850100008B67DDFFFF03F9FFFFF060
:102340000000000BF9FFFF00000000820300008B7B
:10235000C8E7FFFF82FCFFFFF00000003CF9FFFF31
:1023600000000000D80000008BC8E7FFFF82FCFFE0
:10237000FFF00000001FF9FFFF00000000850100D2
:10238000008B67DDFFFF82FCFFFFF0000000BAF763
:10239000FFFF00000000820300008BC8E7FFFF0082
:1023A000000000F0000000EBF7FFFF00000000D885
:1023B0000000008BC8E7FFFF00000000F0000000F5
:1023C000CEF7FFFF00000000850100008B67DDFFF6
:1023D000FF00000000F000000069F6FFFF000000B1
:1023E00000820300008BC8E7FFFF7E030000F000BF
:1023F00000009AF6FFFF00000000D80000008BC824
:10240000E7FFFF7E030000F00000007DF6FFFF0005
:10241000000000850100008B67DDFFFF7E030000E8
:10242000F000000019F5FFFF00000000820300002B
:102430008BC8E7FFFFFD060000F000000049F5FF34
:10244000FF00000000D80000008BC8E7FFFFFD067A
:102450000000F00000002CF5FFFF000000008501E7
:1024600000008B67DDFFFFFD060000F0000000C8E4
:10247000F3FFFF00000000820300008BC8E7FFFFAE
:102480007B0A0000F0000000F8F3FFFF00000000EE
:10249000D80000008BC8E7FFFF7B0A0000F00000B7
:1024A00000DBF3FFFF00000000850100008B67DD0B
:1024B000FFFF7B0A0000F000000077F2FFFF000042
:1024C0000000820300008BC8E7FFFFFA0D0000F058
:1024D000000000A7F2FFFF00000000D80000008B02
:1024E000C8E7FFFFFA0D0000F00000008AF2FFFFCE
:1024F00000000000850100008B67DDFFFFFA0D0082
:1025000000F000000026F1FFFF0000000082030041
:10251000008BC8E7FFFF78110000F000000056F1C3
:10252000FFFF00000000D80000008BC8E7FFFF7825
:10253000110000F000000039F1FFFF0000000085ED
:102540000100008B67DDFFFF78110000F000000044
:10255000D5EFFFFF00000000820300008BC8E7FFFB
:10256000FFF7140000F000000005F0FFFF0000007E
:1025700000D80000008BC8E7FFFFF7140000F00050
:102580000000E8EFFFFF00000000850100008B67FE
:10259000DDFFFFF7140000F000000084EEFFFF00F5
:1025A000000000820300008B6AF5FFFF15F9FFFFB2
:1025B00068010000B4EEFFFF000000000E01000003
:1025C0008B6AF5FFFF15F9FFFFF000000084EEFFB6
:1025D000FF000000009C0000008B6AF5FFFF15F96A
:1025E000FFFFF000000067EEFFFF00000000850124
:1025F00000008B6AF5FFFFEB060000F0000000030F
:10260000EDFFFF000000007F0300008BE9F8FFFFF3
:1026100015F9FFFFF000000033EDFFFF00000000A0
:10262000D30000008BE9F8FFFF15F9FFFFF0000071
:102630000016EDFFFF00000000850100008BE9F8A7
:10264000FFFF75030000F0000000B2EBFFFF000089
:102650000000820300008B67FCFFFF15F9FFFFF00D
:10266000000000E2EBFFFF00000000D80000008B3C
:1026700067FCFFFF15F9FFFFF0000000C5EBFFFF4F
:1026800000000000850100008B67FCFFFF75030060
:1026900000F000000061EAFFFF000000008203007C
:1026A000008BE6FFFFFF15F9FFFFF000000091EA45
:1026B000FFFF00000000D80000008BE6FFFFFF15C1
:1026C000F9FFFFF000000074EAFFFF000000008542
:1026D0000100008BE6FFFFFF75030000F000000023
:1026E00010E9FFFF00000000820300008B6403007C
:1026F0000015F9FFFFF000000040E9FFFF000000B7
:1027000000D80000008B6403000015F9FFFFF00003
:10271000000023E9FFFF00000000850100008B643A
:1027200003000075030000F0000000BFE7FFFF009A
:10273000000000820300008BE206000015F9FFFF95
:10274000F0000000EFE7FFFF00000000D8000000ED
:102750008BE206000015F9FFFFF0000000D2E7FF52
:10276000FF00000000850100008BE20600007503F9
:102770000000F00000006EE6FFFF00000000820392
:1027800000008B610A000015F9FFFFF00000009EB9
:10279000E6FFFF00000000D80000008B610A000087
:1027A00015F9FFFFF000000081E6FFFF00000000C8
:1027B000850100008B610A000075030000F0000035
:1027C000001DE5FFFF00000000820300008BDF0D0D
:1027D000000015F9FFFFF00000004DE5FFFF0000CD
:1027E0000000D80000008BDF0D000015F9FFFFF09E
:1027F00000000030E5FFFF00000000850100008BB5
:10280000DF0D000075030000F0000000CCE3FFFFC7
:1028100000000000820300008B5E11000015F9FF2C
:10282000FFF0000000FCE3FFFF00000000D8000004
:10283000008B5E11000015F9FFFFF0000000DFE3E0
:10284000FFFF00000000850100008B5E1100007595
:10285000030000F00000007BE2FFFF0000000082A8
:102860000300008BDC14000015F9FFFFF0000000EE
:10287000ABE2FFFF00000000D80000008BDC14007A
:102880000015F9FFFFF00000008EE2FFFF000000DE
:1028900000850100008BDC14000075030000F000CF
:1028A00000002AE1FFFF00000000820300008B5BB4
:1028B00018000015F9FFFFF00000005AE1FFFF00CB
:1028C000000000D80000008B5B18000015F9FFFF26
:1028D000F00000003DE1FFFF000000008501000066
:1028E0008B5B18000075030000F0000000D9DFFFCB
:1028F000FF00000000820300008BDA1B000015F9C6
:10290000FFFFF000000009E0FFFF00000000D8001A
:1029100000008BDA1B000015F9FFFFF0000000EC4F
:10292000DFFFFF00000000850100008BDA1B0000C4
:1029300075030000F000000088DEFFFF00000000CB
:10294000820300008B581F000015F9FFFFF0000004
:1029500000B8DEFFFF00000000D80000008B581F09
:10296000000015F9FFFFF00000009BDEFFFF0000F4
:102970000000850100008B581F000075030000F067
:1029800000000037DDFFFF00000000820300008B25
:10299000581F000075030000F000000067DDFFFF16
:1029A000000000000C0300008C581F00007503009D
:1029B00000F0000000000000000000000086018917
:1029C000188BC8E7FFFF3EEBFFFF68010000000027
:1029D000000000000000DF0000008BC8E7FFFF3EA2
:1029E000EBFFFF6801000000000000E4FFFFFF0CA8
:1029F0000300008BC8E7FFFF3EEBFFFFF000000085
:102A000000000000D0FFFFFF3E0000008BC8E7FF82
:102A1000FF3EEBFFFFF000000000000000B3FFFFEF
:102A2000FF850100008B2AF2FFFF3EEBFFFFF00065
:102A30000000000000004FFEFFFF820300008BC873
:102A4000E7FFFFB4EEFFFFF0000000000000007F92
:102A5000FEFFFFD80000008BC8E7FFFFB4EEFFFFCA
:102A6000F00000000000000063FEFFFF8501000091
:102A70008B2AF2FFFFB4EEFFFFF000000000000021
:102A800000FEFCFFFF820300008BC8E7FFFF2AF275
:102A9000FFFFF0000000000000002EFDFFFFD80047
:102AA00000008BC8E7FFFF2AF2FFFFF000000000E4
:102AB00000000012FDFFFF850100008B2AF2FFFFDE
:102AC0002AF2FFFFF000000000000000ADFBFFFF56
:102AD000820300008BC8E7FFFF9FF5FFFFF00000B7
:102AE0000000000000DDFBFFFFD80000008BC8E7FE
:102AF000FFFF9FF5FFFFF000000000000000C1FB9A
:102B0000FFFF850100008B2AF2FFFF9FF5FFFFF01A
:102B1000000000000000005CFAFFFF820300008B51
:102B2000C8E7FFFF15F9FFFFF000000000000000FC
:102B30008DFAFFFFD80000008BC8E7FFFF15F9FFF3
:102B4000FFF00000000000000070FAFFFF850100A8
:102B5000008B2AF2FFFF15F9FFFFF00000000000D4
:102B600000000BF9FFFF820300008BC8E7FFFF8B1B
:102B7000FCFFFFF0000000000000003CF9FFFFD860
:102B80000000008BC8E7FFFF8BFCFFFFF000000098
:102B9000000000001FF9FFFF850100008B2AF2FFF3
:102BA000FF8BFCFFFFF000000000000000BAF7FF01
:102BB000FF820300008BC8E7FFFF00000000F00069
:102BC000000000000000EBF7FFFFD80000008BC8FA
:102BD000E7FFFF00000000F000000000000000CE52
:102BE000F7FFFF850100008B2AF2FFFF00000000C5
:102BF000F00000000000000069F6FFFF8203000003
:102C00008BC8E7FFFF75030000F000000000000024
:102C1000009AF6FFFFD80000008BC8E7FFFF75039E
:102C20000000F0000000000000007DF6FFFF8501BD
:102C300000008B2AF2FFFF75030000F00000000087
:102C400000000019F5FFFF820300008BC8E7FFFFBB
:102C5000EB060000F00000000000000049F5FFFF57
:102C6000D80000008BC8E7FFFFEB060000F0000073
:102C700000000000002CF5FFFF850100008B2AF208
:102C8000FFFFEB060000F000000000000000C8F3AA
:102C9000FFFF820300008BC8E7FFFF610A0000F01E
:102CA00000000000000000F8F3FFFFD80000008BD8
:102CB000C8E7FFFF610A0000F0000000000000000C
:102CC000DBF3FFFF850100008B2AF2FFFF610A00A2
:102CD00000F00000000000000077F2FFFF82030018
:102CE000008BC8E7FFFFD60D0000F00000000000D9
:102CF0000000A7F2FFFFD80000008BC8E7FFFFD657
:102D00000D0000F0000000000000008AF2FFFF85C7
:102D10000100008B2AF2FFFFD60D0000F00000003A
:102D20000000000026F1FFFF820300008BC8E7FFD0
:102D3000FF4C110000F00000000000000056F1FF01
:102D4000FFD80000008BC8E7FFFF4C110000F00027
:102D500000000000000039F1FFFF850100008B2A10
:102D6000F2FFFF4C110000F000000000000000D551
:102D7000EFFFFF820300008BC8E7FFFFC2140000D3
:102D8000F00000000000000005F0FFFFD800000088
:102D90008BC8E7FFFFC2140000F000000000000035
:102DA00000E8EFFFFF850100008B2AF2FFFFC2144D
:102DB0000000F00000000000000084EEFFFF82032E
:102DC00000008B9FF5FFFFB4EEFFFF6801000000DD
:102DD000000000B4EEFFFFCE0000008B9FF5FFFF68
:102DE000B4EEFFFFF00000000000000084EEFFFFE3
:102DF0009C0000008B9FF5FFFFB4EEFFFFF000008A
:102E0000000000000067EEFFFF850100008B9FF5CA
:102E1000FFFF15F9FFFFF00000000000000003EDC8
:102E2000FFFF820300008B15F9FFFFB4EEFFFFF0F8
:102E30000000000000000033EDFFFFD80000008B11
:102E400015F9FFFFB4EEFFFFF000000000000000E6
:102E500016EDFFFF850100008B15F9FFFF15F9FF47
:102E6000FFF000000000000000B2EBFFFF82030053
:102E7000008B8BFCFFFFB4EEFFFFF00000000000B2
:102E80000000E2EBFFFFD80000008B8BFCFFFFB4DB
:102E9000EEFFFFF000000000000000C5EBFFFF8523
:102EA0000100008B8BFCFFFF15F9FFFFF000000015
:102EB0000000000061EAFFFF820300008B000000B9
:102EC00000B4EEFFFFF00000000000000091EAFFF8
:102ED000FFD80000008B00000000B4EEFFFFF00000
:102EE00000000000000074EAFFFF850100008B0075
:102EF00000000015F9FFFFF00000000000000010C6
:102F0000E9FFFF820300008B75030000B4EEFFFFB2
:102F1000F00000000000000040E9FFFFD8000000C2
:102F20008B75030000B4EEFFFFF00000000000000E
:102F30000023E9FFFF850100008B7503000015F9F0
:102F4000FFFFF000000000000000BFE7FFFF82036A
:102F500000008BEB060000B4EEFFFFF00000000065
:102F6000000000EFE7FFFFD80000008BEB06000039
:102F7000B4EEFFFFF000000000000000D2E7FFFF0A
:102F8000850100008BEB06000015F9FFFFF0000043
:102F900000000000006EE6FFFF820300008B610A64
:102FA0000000B4EEFFFFF0000000000000009EE60D
:102FB000FFFFD80000008B610A0000B4EEFFFFF0B5
:102FC0000000000000000081E6FFFF850100008B8B
:102FD000610A000015F9FFFFF0000000000000008A
:102FE0001DE5FFFF820300008BD60D0000B4EEFF4D
:102FF000FFF0000000000000004DE5FFFFD80000DA
:10300000008BD60D0000B4EEFFFFF00000000000C2
:10301000000030E5FFFF850100008BD60D00001594
:10302000F9FFFFF000000000000000CCE3FFFF828A
:103030000300008B4C110000B4EEFFFFF000000015
:1030400000000000FCE3FFFFD80000008B4C1100E3
:1030500000B4EEFFFFF000000000000000DFE3FF1F
:10306000FF850100008B4C11000015F9FFFFF000F7
:103070000000000000007BE2FFFF820300008BC223
:10308000140000B4EEFFFFF000000000000000ABF1
:10309000E2FFFFD80000008BC2140000B4EEFFFF77
:1030A000F0000000000000008EE2FFFF850100003C
:1030B0008BC214000015F9FFFFF0000000000000B3
:1030C000002AE1FFFF820300008B38180000B4EEF5
:1030D000FFFFF0000000000000005AE1FFFFD800F1
:1030E00000008B38180000B4EEFFFFF00000000075
:1030F0000000003DE1FFFF850100008B3818000053
:1031000015F9FFFFF000000000000000D9DFFFFF0D
:10311000820300008BAD1B0000B4EEFFFFF0000047
:10312000000000000009E0FFFFD80000008BAD1B8D
:103130000000B4EEFFFFF000000000000000ECDF34
:10314000FFFF850100008BAD1B000015F9FFFFF0AC
:103150000000000000000088DEFFFF820300008BFB
:10316000231F0000B4EEFFFFF0000000000000008D
:10317000B8DEFFFFD80000008B231F0000B4EEFF75
:10318000FFF0000000000000009BDEFFFF85010053
:10319000008B231F000015F9FFFFF0000000000066
:1031A000000037DDFFFF820300008B231F000015A6
:1031B000F9FFFF30F200000000000037DDFFFFC51F
:1031C000000000890088000302000088010302005B
:1031D0000088001F0200005F0036083608FF10203C
:1031E000546865205265706C696361746F72203237
:1031F0002020200020202D2D2D2D2D2D2D2D2D2D6D
:103200002D2D2D2D2020202000496E7465726E61B9
:103210006C2052656C656173652020202000466932
:10322000726D776172652056657273696F6E2037B3
:103230002E2000436F6F6C21005374617274205014
:103240007265686561742100526967687420546F03
:103250006F6C004E4120004F4E20004F4646004507
:1032600078747275646572004C65667420546F6F73
:103270006C00506C6174666F726D0057656C636FA3
:103280006D65212049276D202020202020202054FA
:103290006865205265706C696361746F7220322EAC
:1032A00020202050726573732074686520726564F5
:1032B000204D20746F2020676574207374617274D0
:1032C0006564212020202020202020004120626CE5
:1032D000696E6B696E6720274D27206D65616E737F
:1032E00049276D2077616974696E6720616E64207B
:1032F00077696C6C636F6E74696E7565207768654D
:103300006E20796F75202020707265737320746849
:103310006520627574746F6E2E2E2E20004120730E
:103320006F6C696420274D27206D65616E732020C6
:103330002049276D20776F726B696E6720616E641C
:103340002077696C6C757064617465206D79207389
:103350007461747573202020207768656E2049277A
:103360006D2066696E69736865642E2E2E004F7538
:1033700072206E6578742073746570732077696C41
:103380006C20676574206D652073657420757021ED
:1033900020202020202046697273742C2077652716
:1033A0006C6C20726573746F72656D7920627569DB
:1033B0006C6420706C6174666F726D2E2E2E0073BB
:1033C0006F2069742773206E69636520616E6420C5
:1033D0002020206C6576656C2E2049742773207040
:1033E000726F6261626C796120626974206F6666D7
:1033F0002066726F6D202020202020736869707015
:10340000696E672E2E2E20202020202020202000D4
:10341000416161682C2074686174206665656C7315
:10342000202020206D756368206265747465722E9B
:1034300020202020202020204C6574277320676FD7
:10344000206F6E20616E64206C6F6164736F6D65B8
:103450002066696C616D656E74212020202020201B
:10346000005765276C6C2074727920616761696E02
:10347000212020202020202020202020202020204B
:10348000202020202020202020202020202020203C
:10349000202020202020202020202020202020202C
:1034A000202020202020202020202020202020201C
:1034B00020005765276C6C206B65657020676F690D
:1034C0006E6720202020616E64206C6F6164207321
:1034D0006F6D652020202020202066696C616D655D
:1034E0006E742C466F722068656C7020676F746F05
:1034F000206D616B6572626F742E636F6D2F6865EE
:103500006C70005765276C6C20676F20746F207497
:103510006865206D61696E6D656E752E2049662047
:10352000796F75206E65656420202068656C702059
:10353000676F20746F3A2020202020202020206DEB
:10354000616B6572626F742E636F6D2F68656C704E
:1035500020202000417765736F6D65212020202099
:1035600020202020202020205765276C6C20676FAA
:1035700020746F2074686520534420206361726456
:10358000206D656E7520616E6420796F7520202036
:1035900063616E2073656C6563742061206D6F6478
:1035A000656C21200049276D20676F696E67207464
:1035B0006F206D616B6520202061207365726965E5
:1035C00073206F66206C696E657320736F7765205A
:1035D00063616E2066696E64206D79202020202052
:1035E000206E6F7A7A6C6520616C69676E6D656EAE
:1035F000742E202020004C6F6F6B20666F72207439
:10360000686520626573742020206D61746368654D
:1036100064206C696E6520696E20656163686178FD
:103620006973207365742E204C696E657320617216
:1036300065206E756D626572656420312D313320B1
:10364000616E642E2E2E006C696E65206F6E652093
:1036500069732065787472612020206C6F6E672E0C
:1036600020546865205920617869732073657469F6
:1036700073206C656674206F6E2074686520706CB2
:10368000617465616E642058206178697320697384
:103690002072696768742E0047726561742120206A
:1036A00049277665207361766564202074686573A8
:1036B000652073657474696E677320616E64202081
:1036C00049276C6C20757365207468656D20746F74
:1036D000202020206D616B65206E696365206D6F11
:1036E00064656C73212020200053656C6563742031
:1036F00062657374206C696E65732E005820417882
:103700006973204C696E65002D2D3E00202020003D
:10371000592041786973204C696E6500446F6E656D
:1037200021004D792074656D7065726174757265E4
:103730002077617320206368616E67656420657817
:103740007465726E616C6C792E20526573656C6560
:1037500063742066696C616D656E742020206D65F0
:103760006E7520746F2074727920616761696E2EA6
:103770002020004D7920657874727564657273201D
:10378000617265202020206E6F7420686561746905
:103790006E672075702E2020202020436865636BA3
:1037A000206D792020202020202020202020206330
:1037B0006F6E6E656374696F6E7321202020202008
:1037C0002020200049276D2068656174696E67209C
:1037D0007570206D79202020726967687420657883
:1037E00074727564657220736F20776563616E20F3
:1037F0006C6F61642066696C616D656E742E20204B
:103800004265206361726566756C2C207468652E54
:103810002E2E20200049276D2068656174696E672F
:10382000207570206D79202020657874727564652C
:103830007220736F2077652063616E20206C6F614A
:1038400064207468652066696C616D656E742E20F5
:10385000204265206361726566756C2C2074686512
:103860002E2E2E202000506C6561736520776169D3
:1038700074207768696C6520492068656174206DE3
:10388000792065787472756465722120202020206B
:103890002020202020202020202020202020202028
:1038A0002020202020202020202020202020202018
:1038B000202020202020006E6F7A7A6C65207769A6
:1038C0006C6C2067657420686F74215768696C653B
:1038D0002049276D2068656174696E672C2020720D
:1038E000656D6F7665207468652066696C616D65CD
:1038F0006E7420747562652066726F6D20746865E1
:103900002E2E2E20202020006E6F7A7A6C65207774
:10391000696C6C2067657420686F74215768696CE6
:10392000652049276D2068656174696E672C2020C9
:1039300072656D6F7665207468652066696C616D6F
:10394000656E7420747562652066726F6D20746890
:10395000652E2E2E202020200065787472756465F7
:103960007220626C6F636B2E204665656466696CBD
:10397000616D656E742066726F6D207468652020BD
:103980002073706F6F6C207468726F756768207435
:1039900068652020207475626520756E74696C20DE
:1039A00069742E2E2E2020202000706F7073206FDF
:1039B000757420696E2066726F6E742E20205768B1
:1039C000656E207468652066696C616D656E742033
:1039D000697372656164792C207072657373202736
:1039E0004D2720746F20636F6E74696E75652E208D
:1039F000202020202020202020200048656174699C
:103A00006E672050726F67726573733A20202020B2
:103A100020202020202020202020202020202020A6
:103A20002020202020202020202020202020202096
:103A30002020202020202020202020202020202086
:103A40002020202020202020202020004F4B204913
:103A5000276D20726561647921202020202020209C
:103A60004E6F77207765276C6C206C6F61642074D3
:103A7000686520207269676874206578747275645F
:103A800065722E2020202020507573682066696C96
:103A9000616D656E7420696E2E2E2E20004F4B20B6
:103AA00049276D2072656164792120202020202023
:103AB0002050757368207468652066696C616D6557
:103AC0006E742020207468726F7567682E2E2E2009
:103AD00020202020202020202020202020202020E6
:103AE00020202020202020202020202020004927C6
:103AF0006D207265616479212050756C6C2074684A
:103B0000652067756964652074756265206F6666F7
:103B100020616E642020707573682074686520666B
:103B2000696C616D656E742020207468726F7567B2
:103B3000682E2E2E2020202020202020202000490A
:103B4000276D207265616479212050756C6C20743A
:103B500068652067756964652074756265206F66A5
:103B60006620616E64202070756C6C20746865201E
:103B700066696C616D656E7420202067656E746C7B
:103B8000792E2E2E202020202020202020202000D2
:103B900049276D20726561647921204465746163F1
:103BA00068202020746865206775696465207475D5
:103BB000626520616E6420206D6F76652074686593
:103BC000206C6576657220746F20202074686520F3
:103BD00072696768742E202050756C6C2E2E2E2012
:103BE0000049276D20726561647921204465746104
:103BF0006368202020746865206775696465207497
:103C000075626520616E6420206D6F766520746832
:103C100065206C6576657220746F2020207468655D
:103C2000206C6566742E202050756C6C2E2E2E2014
:103C30002000756E74696C20796F75206665656CFF
:103C40002074686520206D6F746F72207475672012
:103C5000697420696E2E20202020507573682066BC
:103C60006F72206120666577206D6F7265207365C5
:103C7000636F6E64732C207468656E20776169745D
:103C80002E20005768656E2066696C616D656E74E4
:103C9000206973202020206265696E672065787432
:103CA00072756465642066726F6D20746865206E3D
:103CB0006F7A7A6C652C205072657373204D207476
:103CC0006F2073746F7020657874727564696E67A5
:103CD0002E2020005768656E2066696C616D656EE8
:103CE00074206973202020206265696E67206578E2
:103CF0007472756465642066726F6D2074686520E7
:103D00006E6F7A7A6C652C202020202020202020C5
:103D1000507265737320274D2720746F2065786972
:103D2000742E2020005768656E206D792066696CBE
:103D3000616D656E742069732072656C6561736571
:103D4000642C20202020202020202020205072655C
:103D5000737320274D2720746F20657869742E2097
:103D60002020202020202020202020202020202053
:103D700020202020200066696C616D656E742066CD
:103D800072656520616E64202020636C6F7365200E
:103D9000746865206C657665722E20202020507234
:103DA00065737320274D2720746F20657869742E02
:103DB0002020202020202020202020202020202003
:103DC0002020202020200047726561742120204996
:103DD000276C6C2073746F7020202072756E6E6972
:103DE0006E67206D792065787472756465722E50E7
:103DF00072657373204D20746F20636F6E74696EEB
:103E000075652E202020202020202020202020200A
:103E100020202020202020004F4B212049276C6C9F
:103E2000206B656570206D79202020206D6F746F88
:103E3000722072756E6E696E672E20596F75202024
:103E40006D6179206E65656420746F20707573688C
:103E5000202020206861726465722E2E2E20202082
:103E60002020202020202020005765276C6C206B0C
:103E700065657020676F696E672E20202049662077
:103E8000796F7527726520686176696E67202020DA
:103E90002074726F75626C652C20636865636B209B
:103EA0006F757420206D616B6572626F742E636F25
:103EB0006D2F68656C70202020004D79206D6F7427
:103EC0006F722074696D6564206F7574202061665F
:103ED0007465722035206D696E757465732E2020AF
:103EE00020205072657373204D20746F20657869AF
:103EF000742E202020202020202020202020202060
:103F00002020202020202020202000486F772764B8
:103F100020697420676F3F2052656164792020001A
:103F2000746F206D616B6520736F6D657468696E69
:103F3000673F202000596573202020004E6F20200D
:103F4000202000446F6573206D79206E6F7A7A6C43
:103F500065200068656967687420636865636B2025
:103F60006F75743F20004D7920686569676874201B
:103F7000697320676F6F64212020004C657427737C
:103F80002074727920616761696E2E004469642033
:103F9000706C6173746963206578747275646520F0
:103FA0000066726F6D20746865206E6F7A7A6C653A
:103FB0003F20202020004C6F616420726967687484
:103FC000004C6F616400556E6C6F616420726967AC
:103FD000687400556E6C6F6164004C6F6164206C96
:103FE00065667400556E6C6F6164206C6566740064
:103FF00020202020204A6F67206D6F6465202020DC
:1040000020202020002020202020202020582B208D
:1040100020202020202020202000202020202020C0
:10402000284261636B29202020592D3E202000204A
:1040300020202020202020582D202020202020203B
:10404000202020002020202020202020592B20204C
:1040500020202020202020200020203C2D58202817
:104060004261636B2920205A2D3E20202000202011
:10407000202020202020592D2020202020202020FA
:1040800020200020202020202020205A2D20202009
:10409000202020202020200020203C2D59202842B4
:1040A00061636B2920202020202020200020202058
:1040B00020202020205A2B202020202020202020BB
:1040C000200047414D45204F56455221004865612B
:1040D00074696E673A202020202020202020202094
:1040E000200048656174696E673A00202020202016
:1040F0002000202D2D25006572726F722100202076
:1041000020202020202020202020202020202020AF
:1041100020200045787472756465723A2020202D45
:104120002D2D2F2D2D2D430052204578747275644E
:1041300065723A202D2D2D2F2D2D2D43004C20451D
:10414000787472756465723A202D2D2D2F2D2D2DCA
:104150004300506C6174666F726D3A2020202D2DE3
:104160002D2F2D2D2D430020204E412020202000DA
:1041700077616974696E6720002F20202043004317
:1041800020202020006820206D0020507265686586
:1041900061742053657474696E6773202020005227
:1041A0006967687420546F6F6C20202020202020C5
:1041B000202020004C65667420546F6F6C202020F6
:1041C000202020202020202000506C6174666F7217
:1041D0006D2020202020202020002052657365744F
:1041E0002053657474696E677320746F20200020FB
:1041F00044656661756C742076616C7565733F000B
:10420000556E5061757365202020202020202020CD
:104210002020200050617573652020202020202060
:10422000202020202020200043616E63656C204206
:1042300075696C642020202020202000576169745B
:10424000696E6720666F7220486F6D696E67200027
:104250004368616E67652046696C616D656E7420A8
:1042600020202000536C6565702028436F6C64200B
:104270005061757365292000526573756D65204224
:1042800075696C6420202020202020005A20506175
:1042900075736520486569676874202020202000B8
:1042A0004C454420436F6C6F72202020202020203A
:1042B00020202000524544202020004F52414E47EC
:1042C000450050494E4B202000475245454E2000A6
:1042D000424C5545202000505552504C45005748FF
:1042E0004954452000435553544F4D004F464620F6
:1042F00020200046696C616D656E742046616E20F9
:10430000202020202020004275696C6420537461B5
:1043100074697374696373202020004261636B20A9
:10432000746F204D6F6E69746F72202020200042E0
:1043300075696C642046696E697368656421202024
:10434000202020202020202020202020202020206D
:10435000202020202020204275696C642054696D43
:10436000652020202020206820206D004275696C87
:10437000642054696D653A20202020206820206D3B
:10438000004C696E653A202020202020202020202B
:10439000202020202000457374696D6174656420BD
:1043A0004275696C642054696D654C696665746911
:1043B0006D6520546F74616C3A2020202068004C99
:1043C000617374204275696C643A20202020206853
:1043D00020206D0043616E63656C207468697320F2
:1043E0006275696C643F0051756974207468697303
:1043F0002070726F636573733F004275696C64204F
:1044000066726F6D205344202020202020005072BF
:104410006568656174202020202020202020202035
:1044200020005574696C6974696573202020202010
:10443000202020202000496E666F20616E6420538A
:10444000657474696E67732020004D6F6E69746FB8
:1044500072204D6F646520202020202020004368BA
:10446000616E67652046696C616D656E7420202001
:1044700020004C6576656C204275696C6420506C38
:104480006174652020004A6F67204D6F64652020AD
:1044900020202020202020202000486F6D65204112
:1044A00078657320202020202020202020005275B5
:1044B0006E205374617274757020536372697074E6
:1044C0002000456E61626C65205374657070657282
:1044D00073202020200044697361626C652053744E
:1044E0006570706572732020200053746F702042D5
:1044F0006C696E6B696E6721202020202000426C61
:10450000696E6B204C454473202020202020202001
:10451000200043616C696272617465204E6F7A7A23
:104520006C657320200065786974206D656E752058
:1045300020202020202020202000426F742053744F
:1045400061746973746963732020202020004765BB
:104550006E6572616C2053657474696E6773202098
:104560002000507265686561742053657474696ECB
:1045700067732020200056657273696F6E204E7538
:104580006D626572202020202000526573746F7266
:10459000652044656661756C7473202020002020BE
:1045A000205A2050617573652048656967687420DA
:1045B0002020005A20506F736974696F6E2020208C
:1045C0002020206D6D20005061757365204163745B
:1045D0006976652020202020202000536F756E64AE
:1045E00020202020202020202020202020200048C3
:1045F000656174656420506C61746500546F6F6C04
:1046000020436F756E742020202020202020200061
:1046100053494E474C45004455414C2020004865C5
:104620006174204C4544732020202020202020202D
:1046300020004865617420486F6C64202020202091
:10464000206D2020200048656C702054657874200F
:1046500020202020202020202000416363656C65FD
:1046600072617465202020202020202020004E6FC1
:10467000205344206361726420666F756E6400533A
:104680004420636172642072656164206572726F98
:104690007200492063616E27742072656164207422
:1046A0006869732020205344206361726420666F20
:1046B000726D61742120202020205472792072654F
:1046C000666F726D617474696E6720202020746853
:1046D00065206361726420746F2046415431362E28
:1046E000202000492063616E277420726561642078
:1046F0005344202020202063617264732077697402
:10470000682073746F7261676520206C61726765E1
:1047100072207468616E203247422E2020202020B3
:104720002020202020202020202020202020202089
:104730002020200020534420636172642072656150
:1047400064206572726F720049276D20616C72651A
:10475000616479206275696C64696E670057617283
:104760006E696E673A4275696C6420737065656442
:1047700073666173746572207468616E2035306D84
:104780006D2F7320207265717569726520783367AB
:1047900020666F726D61742020666F72206265738F
:1047A0007420726573756C74732E20202000D0FE07
:1047B000C0FF18FFD0FF63FFE0FFB1FFF0FF000074
:1047C000000051001000A4002000F800300040015B
:1047D0004000A2015000F70160004B0270009F02F0
:1047E0008000F20290004503A0009703B000E803A8
:1047F000C0003A04D0008C04E000DF04F000320571
:10480000000186051001DB0520012F063001DA06C4
:1048100050013007600186077001DC0780016808DD
:10482000900120F9C9FFE0FCE7FFF8FF000000005D
:104830000000080000002003190040063200600953
:104840004B00000A5000800C640000108000010042
:104850009403360009016B00D800A000BD00D5000C
:10486000AB000A019D003F01840074017C00A90196
:104870007400DE016D0013026600480260007D02D4
:104880005900B2025200E7024B001C0344005103DE
:104890003A0086033000BB032200F0030200F2332B
:1048A00019340C38DE416142FF4CA74E22527F532F
:1048B0000E67A478B37BBF86F1871489158AC58BF0
:1048C000F48BB38D6B991A9AF19D839E6C9F29A0EE
:1048D00053A17BA6C7A6C8AA9BAE3AD0F8D17FD376
:1048E000C9D482D55ED611241FBECFEFD1E2DEBF80
:1048F000CDBF15E0A0E0B2E0E0E6FAEB01E00BBFCF
:1049000002C007900D92A03BB107D9F72DE1A0EBB3
:10491000B5E001C01D92A336B207E1F718E4C6EE78
:10492000D8E400E006C022970109FE010BBF0E94F7
:104930001DDCCE39D10780E00807A9F70E942E427E
:104940000C942EDD0C940000FA01DC0102C00590ED
:104950000D9221503040D8F70895F8948091F405D5
:104960009091F5052091F2053091F305281B390B44
:104970007894C90108958093EB05089581E08093B0
:10498000E90508958091EB0508958091EA05089561
:104990002091F4053091F50581E0232B09F080E0AA
:1049A00008951092F5051092F4051092F7051092F3
:1049B000F6051092FA051092FB051092ED05109283
:1049C000EE051092EF051092F0051092EC05109292
:1049D000EB051092EA051092E4051092E50510929D
:1049E000E6051092E7051092CF051092E3051092AC
:1049F000E2051092E105089581E02091E1053091F2
:104A0000E2052630310509F080E008956091ED055A
:104A10007091EE058091EF059091F0050895109248
:104A2000ED051092EE051092EF051092F005089535
:104A30004F925F926F927F928F929F92AF92BF92AE
:104A4000CF92DF92EF92FF920F931F93CF93DF935A
:104A5000CDB7DEB7C256D1090FB6F894DEBF0FBE90
:104A6000CDBFCE018D5B9F4F0E94F37D84E1FE019F
:104A7000ED5BFF4FA3EBB5E001900D928A95E1F756
:104A800045E06FE87AE1CE01CD960E941DD3CE01BC
:104A9000CD960E945FD38093B20564E070E083EB13
:104AA00095E00E94074FDC016D917D918D919C9165
:104AB0000E94E2D82B013C0184E00E942F7B9B01E5
:104AC000AC0163E070E083EB95E0A0962FAFA09778
:104AD000A1963FAFA197A2964FAFA297A3965FAFC3
:104AE000A3970E94074FFC0180809180A280B38031
:104AF00083E00E942F7B6B966CAF7DAF8EAF9FAF34
:104B00006B9762E070E083EB95E00E94074FDC0159
:104B1000CD90DD90ED90FC9061E070E083EB95E04E
:104B20000E94074FDC018D919D910D90BC91A02DAD
:104B30006F968CAF9DAFAEAFBFAF6F9760E070E088
:104B400083EB95E00E94074F8C016B966CAD7DADB9
:104B50008EAD9FAD6B970E94B4D8860E971EA81E8F
:104B6000B91ED8018D919D910D90BC91A02D6B9691
:104B70008CAF9DAFAEAFBFAF6B97A0962FADA09798
:104B8000A1963FADA197A2964FADA297A3965FAD18
:104B9000A397C301B2010E9492D70E94AFD89F93FE
:104BA0008F937F936F936F960CAD1DAD2EAD3FAD80
:104BB0006F976B964CAD5DAD6EAD7FAD6B97CE01D3
:104BC00089960E94CB4E48E052E060E070E0CE0152
:104BD00089960E94897E8FE399E00E9463A4909356
:104BE000CA058093C9058EED99E00E9463A4909355
:104BF000CC058093CB058EE19CE00E9463A490934A
:104C0000C8058093C7050F900F900F900F9080916B
:104C1000E805882391F060E070E08FE399E00E945E
:104C20008DA360E070E08EED99E00E948DA360E0BE
:104C300070E08EE19CE00E948DA384E1FE01B996B4
:104C4000DE01559601900D928A95E1F762E070E0E1
:104C5000CE0145960E94074F8C0182E00E942F7B77
:104C60000E94AFD89B01AC01A6E9B0E00E94E4DA53
:104C7000F801608371838283938384E1FE017596DA
:104C8000DE01119601900D928A95E1F760E070E0E7
:104C9000CE0101960E94074F8C0180E00E942F7B7D
:104CA00020E030E04DED52EC0E94E6D90E94AFD8F2
:104CB000D8016D937D938D939C93139761E070E081
:104CC000CE0101960E94074F8C0181E00E942F7B4C
:104CD00020E030E044E952EC0E94E6D90E94AFD8CF
:104CE000F80160837183828393834CE850E060E035
:104CF00070E0CE0145960E94897E42E850E060E077
:104D000070E0CE0101960E94897E60E089EC98E017
:104D10000E94974BCE59DF4F0FB6F894DEBF0FBEFF
:104D2000CDBFDF91CF911F910F91FF90EF90DF905A
:104D3000CF90BF90AF909F908F907F906F905F903B
:104D40004F9008950F931F93CF93DF93CDB7DEB7A6
:104D500064970FB6F894DEBF0FBECDBFCE010196AB
:104D60000E94F37D63E070E0CE0101960E94074F40
:104D70008C0163E070E083EB95E00E94074FFC013B
:104D80004081518162817381F80140835183628344
:104D9000738364E070E0CE0101960E94074F8C019E
:104DA00064E070E083EB95E00E94074FFC014081D6
:104DB000518162817381F8014083518362837383DF
:104DC000CE0101960E94767C62E070E0CE010196F1
:104DD0000E94074F8C0162E070E083EB95E00E9437
:104DE000074FFC014081518162817381F80140834A
:104DF0005183628373834CE850E060E070E0CE0141
:104E000001960E94897E42E850E060E070E083EB0A
:104E100095E00E94897E6091B20589EC98E00E943D
:104E2000974B64960FB6F894DEBF0FBECDBFDF91EF
:104E3000CF911F910F9108956091C9057091CA0596
:104E40008FE399E00E948DA36091CB057091CC0512
:104E50008EED99E00E948DA36091C7057091C80501
:104E60008EE19CE00E948DA38EE19CE00E9477A4DD
:104E7000882329F18EE19CE00E9491A481111FC03A
:104E800017C061E08FE399E00E94C3A481E08093A2
:104E9000EC058EED99E00E9491A4811110C061E0B3
:104EA0008EED99E00E94C3A481E08093EC05089503
:104EB0008FE399E00E9491A48111EBCFE2CF089596
:104EC000CF93DF93EB0170930502609304029091FE
:104ED000EA05981709F44BC0882329F1209781F43B
:104EE00081E08093E8056CE171E083ED9AE00E9437
:104EF000F7A781E090E09093CE058093CD050FC099
:104F00006130710561F41092E80569E571E083EDA7
:104F10009AE00E94F7A7D093CE05C093CD0581E01B
:104F20008093EA0524C08091CD059091CE05813013
:104F3000910529F41092CE051092CD0516C082304D
:104F4000910529F40E941C2784E090E006C0039795
:104F500049F40E941C2785E090E09093CE05809351
:104F6000CD0505C06230710511F41092EA05DF919C
:104F7000CF910895CF93FC01C62F828193816081E8
:104F800071818617970798F44281538184819581B6
:104F9000840F951F0E9465DAA681B781A80FB91FFB
:104FA000CC938281938101969383828302C081E0B6
:104FB0008087CF910895682F82EF95E00C94BA27EF
:104FC000CF93DF93FC0182819381892B21F481E0CF
:104FD000818780E019C08481958120813181B90168
:104FE0000E9465DAC681D781C80FD91F8481958157
:104FF0000196B9010E9465DA958384838281938149
:105000000197938382838881DF91CF9108951F93C5
:10501000CF93DF9300D0CDB7DEB782EF95E00E944B
:10502000E027682F82EF95E06A830E94E027782FBF
:1050300082EF95E079830E94E027182F82EF95E0B8
:105040000E94E027982F6A817981812F0F900F901D
:10505000DF91CF911F910895CF9382EF95E00E9449
:10506000E027C82F82EF95E00E94E027982F8C2F31
:10507000CF91089582EF95E00C94E027CF93DF93D2
:105080000E943A28D82F0E943A28C82F0E943A2816
:10509000CA3009F4E9C098F4C63009F4E2C048F413
:1050A000C43009F4E1C008F0DFC0C33009F0DFC04C
:1050B0001AC0C83009F4D8C008F0D6C0D2C0CE306B
:1050C00009F4D2C030F4CC3009F46CC008F078C0D8
:1050D000CBC0C73109F45FC0CF3109F47AC0CF30FB
:1050E00009F0C5C0C1C08091B1058823A1F08FE34C
:1050F00099E00E9493A28EED99E00E9493A2809184
:10510000B005811104C08EE19CE00E9493A2109230
:10511000B0051092B1050E942C28BC01D13019F4C1
:1051200086ED99E002C087E399E008960E948DA37E
:105130008EE19CE00E9477A4882309F4A3C08EE14D
:105140009CE00E9491A481119DC0D13019F486ED9C
:1051500099E002C087E399E008960E9491A481112A
:1051600091C087C086ED99E061E003C086ED99E0CB
:1051700060E008960E94C3A440E061E070E089EC22
:1051800098E00E945F45D13009F090C00E94C3357D
:1051900081117EC08BC09091EB0581E089270E9430
:1051A0001C3C84C00E943A28682F6170D13019F4E9
:1051B00086ED99E002C087E399E00E94A58976C058
:1051C0000E943A28682F617089EC98E00E94974B02
:1051D0006DC061E089EC98E00E94924B8091B1052E
:1051E000882319F081E08093B0050E942C28BC012F
:1051F0008EE19CE00E948DA38EE19CE00E9491A430
:10520000C1E0C827C093EC056C2F8FE399E00E94A2
:10521000C3A46C2F8EED99E00E94C3A440E061E02E
:1052200070E089EC98E00E945F450E94B0368111E1
:105230003DC00E94A63B059741F021E040E067EEAB
:1052400071E089EC98E00E943D4560E070E08EE1FD
:105250009CE00E948DA360E089EC98E00E94924B54
:1052600025C00E94072822C00E943A281FC080E063
:105270001EC081E08093EC05D13009F473CF87E341
:1052800099E072CFD13009F471CF87E399E070CF04
:1052900021E040E066E971E089EC98E00E943D453C
:1052A00060E070E08EED99E00E948DA381E0DF91D7
:1052B000CF9108952F923F924F925F926F927F927B
:1052C0008F929F92AF92BF92CF92DF92EF92FF9216
:1052D0000F931F93CF93DF93CDB7DEB7E7970FB64A
:1052E000F894DEBF0FBECDBF0E948850882309F41A
:1052F00093C08091F4059091F5052091F2053091CD
:10530000F3052817390711F40C94D0320E94F65097
:1053100081110C94D6320C94D032C090E405D09018
:10532000E505E090E605F090E7050E943750C616C7
:10533000D706E806F90610F00C94FD328091CF05EF
:1053400081110C94FD320C94F23283ED9AE00E94AC
:105350001DA721E040E068E372E089EC98E00E943C
:105360003D4581E08093CF050E94C1831092F505F1
:105370001092F4051092F7051092F6051092FA05B6
:105380001092FB0560E070E08FE399E00E948DA32E
:1053900060E070E08EED99E00E948DA360E070E027
:1053A0008EE19CE00E948DA3CE0101960E945F7D5C
:1053B00062E070E0CE0101960E94074F8C0182E00E
:1053C0000E942F7B20E030E046E153E40E94E6D9C2
:1053D0000E94AFD8F8016083718382839383109217
:1053E000EB0546E950E060E070E0CE0101960E94D6
:1053F000897E0E9408511092E3050EC08091F40549
:105400009091F505892B41F48091E1059091E20599
:10541000892B11F40C9404330E947287882311F1B4
:105420008091F4059091F5052091F2053091F305F6
:105430002817390711F40C9408330E947B878111D7
:105440000C940F330C9408338091F4059091F5057A
:10545000892B41F48091E1059091E205892B11F4AB
:105460000C9418338091EC05882391F08EE19CE038
:105470000E943FA4882361F060E08FE399E00E94DE
:10548000C3A460E08EED99E00E94C3A41092EC05E5
:105490008091EB0581110C94D9338091E90581113C
:1054A0000C94D9338091E1059091E205039789F43A
:1054B0000E94D27B811101C008C082ED95E00E945C
:1054C000F8D4882331F00E94C1831092E205109233
:1054D000E1058091E1059091E205019741F40E9478
:1054E000D27B811104C01092E2051092E1058091F7
:1054F000E1059091E205029751F482ED95E00E945A
:10550000F8D4882321F01092E2051092E1058091F1
:10551000E1059091E205049709F04AC082ED95E01B
:105520000E94F8D4882351F021E040E069E872E05D
:1055300089EC98E00E943D450C9429338091F10557
:10554000813019F486ED99E002C087E399E008966E
:105550000E943FA4882311F40C941C338091F10520
:10556000813019F486ED99E002C087E399E0FC01EF
:10557000E258FF4F808181110C941C330C94263328
:1055800087E399E008960E9477A4811111C0809169
:10559000F105813019F486ED99E002C087E399E0C6
:1055A000FC01E258FF4F8081882311F40C942933C9
:1055B0008091E1059091E205059701F582ED95E076
:1055C0000E94F8D4882349F021E040E066EC72E0C4
:1055D00089EC98E00E943D450DC08EE19CE00E9460
:1055E00077A4811101C006C08EE19CE00E943FA417
:1055F000882321F01092E2051092E1058091E105E7
:105600009091E205069709F03FC082ED95E00E9477
:10561000F8D48823B1F08091D00581FF06C060E006
:1056200089EC98E00E94204C2FC01092E205109265
:10563000E10540E060E170E089EC98E00E945F45A0
:1056400023C083ED9AE00E94C0AA8823E9F08091EC
:10565000D00582FF04C083ED9AE00E948CA840E050
:1056600050E060E070E089EC98E00E943E4840E045
:1056700060E170E089EC98E00E945F450E946D8ACD
:105680001092E2051092E1058091E1059091E2050A
:10569000892B09F06AC78091EA05882309F4E2C0E2
:1056A0008091CD059091CE05019709F0D8C70E9451
:1056B000DC658111DBC7D3C763E073E004C00197E9
:1056C00031F464E573E083ED9AE00E94F7A70E944D
:1056D000182582E090E096C00E94DC658111D7C752
:1056E000CDC740E059EE64EA75E382ED95E00E9493
:1056F000D4D486E00E946A4E809104029091050203
:10570000892B11F00C94D93364E180E00E94D88297
:1057100064E181E00E94D88264E183E00E94D88243
:1057200064E184E00E94D8820C94D9338091040211
:1057300090910502019711F00C94D93382ED95E018
:105740000E94F8D48111B3C70C94D933049749F05F
:105750008091CD059091CE058530910509F0E5C782
:10576000E9C70E94DC658111E5C7F2CF6FE780E0F1
:105770000E94D8826FE781E00E94D8828091040263
:1057800090910502892B41F46FE783E00E94D88253
:105790006FE784E00E94D88262EE73E083ED9AE0C6
:1057A0000E94F7A71092F10585E090E09093E20542
:1057B0008093E10540E052ED69E47BE682ED95E0FF
:1057C0000E94D4D486E090E09093CE058093CD05DE
:1057D00024E140E063E089EC98E00E948845E9C755
:1057E0001092F10584E090E09093E2058093E1054A
:1057F00040E052ED69E47BE682ED95E00E94D4D46E
:1058000087E090E09093CE058093CD05D2C7873096
:105810009105A1F481E08093F10584E090E09093FC
:10582000E2058093E10540E052ED69E47BE682ED1C
:1058300095E00E94D4D488E090E0E4CF88309105D0
:1058400049F489EC98E00E949E450E94A22689E0D6
:1058500090E0D8CF099709F0ACC70E94DC658111B0
:1058600071C7A7C78091F4059091F505892B09F4BC
:105870007CC689EC98E00E94C0478091F605909123
:10588000F7056091F2057091F3050E9465DAE091E9
:10589000F805F091F905E80FF91F10811B3809F49C
:1058A00064C71E3809F469C71B3909F456C719388B
:1058B00009F46BC7163909F434C3163809F471C7F3
:1058C0001C3841F48091F4059091F505459708F452
:1058D0004CC6D0C11C3909F424C3103909F421C3C2
:1058E000133809F41EC3143809F41BC3183809F41B
:1058F00018C30E94DC65811150C75BC789EC98E032
:105900000E94C0470E943A2881E090E09093E2050F
:105910008093E1050E94072868A779A78AA79BA71B
:105920000E9407286CA77DA78EA79FA70E94072823
:105930006B017C010E9407284B015C010E94072833
:10594000162F072F382E292E0E9407282B013C01E5
:105950008091ED059091EE05A091EF05B091F005D5
:105960000196A11DB11D8093ED059093EE05A093C6
:10597000EF05B093F0052F923F920F931F930CA564
:105980001DA52EA53FA548A559A56AA57BA5CE01B5
:1059900001960E94CB4EB301A201CE0101960E9456
:1059A000897E58C089EC98E00E94C0470E943A283E
:1059B00081E090E09093E2058093E1050E94072842
:1059C00068A779A78AA79BA70E9407286CA77DA72D
:1059D0008EA79FA70E9407286B017C010E940728C1
:1059E0004B015C010E940728162F072F282E9EAB23
:1059F0000E9407282B013C010E943A28382E8091F2
:105A0000ED059091EE05A091EF05B091F00501969E
:105A1000A11DB11D8093ED059093EE05A093EF05B8
:105A2000B093F0052EA92F932F920F931F930CA5DF
:105A30001DA52EA53FA548A559A56AA57BA5CE0104
:105A400001960E94CB4E232DB301A201CE010196F7
:105A50000E94787F0F900F900F900F9086C589EC71
:105A600098E00E94C0470E943A2881E090E090931D
:105A7000E2058093E1050E94072868A779A78AA715
:105A80009BA70E9407286CA77DA78EA79FA70E94AF
:105A900007286B017C010E9407284B015C010E94D2
:105AA0000728162F072F282E9EAB0E9407282B01B0
:105AB0003C010E943A28382E0E94072868AB79AB37
:105AC0008AAB9BAB0E942C289DAB8CAB8091ED05E3
:105AD0009091EE05A091EF05B091F0050196A11D02
:105AE000B11D8093ED059093EE05A093EF05B09363
:105AF000F0052EA92F932F920F931F930CA51DA590
:105B00002EA53FA548A559A56AA57BA5CE0101965E
:105B10000E94CB4ECCA8DDA8E8A8F9A80AA91BA929
:105B2000232DB301A201CE0101960E94888092CF5D
:105B30000E943A280E943A288093F1054091ED0591
:105B40005091EE056091EF057091F0054F5F5F4F4A
:105B50006F4F7F4F4093ED055093EE056093EF0537
:105B60007093F0050E94E68200C50E943A280E94C8
:105B70003A28E82E4091ED055091EE056091EF0531
:105B80007091F0054F5F5F4F6F4F7F4F4093ED0572
:105B90005093EE056093EF057093F0050E94DC656D
:105BA000882309F4E2C4DE2CDD1CDD24DD1C00E0CA
:105BB00010E0F12CC701002E02C0959587950A943C
:105BC000E2F780FF04C06D2D802F0E94BF820F5F1F
:105BD0001F4F0530110571F7C8C48091F4059091ED
:105BE000F5050B9708F4C1C40E943A280E943A2890
:105BF000182F0E943A28282F30E0F4E61F9F200D2E
:105C0000311D11242436310541F021E040E067EFD9
:105C100073E089EC98E00E943D450E943A280E947A
:105C200007280E942C288531904B41F020E040E06D
:105C300068E474E089EC98E00E943D450E942C28BD
:105C40000E9407280E9407280E943A288091ED05AB
:105C50009091EE05A091EF05B091F0050196A11D80
:105C6000B11D8093ED059093EE05A093EF05B093E1
:105C7000F0057BC40E943A280E9407282B013C01B2
:105C80000E94072868A779A78AA79BA70E940728D0
:105C90006B017C010E9407284B015C010E940728D0
:105CA0009B014091ED055091EE056091EF057091DB
:105CB000F0054F5F5F4F6F4F7F4F4093ED0550935F
:105CC000EE056093EF057093F0059F938F933F93DC
:105CD0002F9308A519A52AA53BA5B301A201CE01C2
:105CE00001960E94CB4ECE0101960E94767CB2CEE8
:105CF000153849F58091F4059091F505059708F45C
:105D000034C482E090E09093E2058093E1050E9424
:105D10003A280E9407289B01AC018091ED059091E3
:105D2000EE05A091EF05B091F0050196A11DB11D02
:105D30008093ED059093EE05A093EF05B093F005E9
:105D4000A8EEB3E074C1143909F047C08091F4059E
:105D50009091F505059708F408C40E943A280E941E
:105D60003A288093D1050E942C288C010E943A2861
:105D70008093D0054091ED055091EE056091EF05BF
:105D80007091F0054F5F5F4F6F4F7F4F4093ED0570
:105D90005093EE056093EF057093F0050115110522
:105DA00071F0D80120E432E44FE050E00E94E4DAE0
:105DB000AB01BC0182ED95E00E94D4D496C0CE0127
:105DC00045960E94D0D48FE0FE017596A2EDB5E015
:105DD00001900D928A95E1F788C0153909F0A1C0AC
:105DE00083ED9AE00E943EA78C018091F40590918A
:105DF000F505069708F4B9C30E943A280E943A288C
:105E0000E82E0E943A28C82E0E943A28D82E0E94D6
:105E10003A28F82E4091ED055091EE056091EF057E
:105E20007091F0054F5F5F4F6F4F7F4F4093ED05CF
:105E30005093EE056093EF057093F005E0FC03C00E
:105E4000C8010E9467CCF801C282D38262EF75E07C
:105E5000C8010E94CBCBE1FE88C3E091020CEE0F9B
:105E6000FF0BEC50F44F208131812017310731F0C6
:105E7000B80183ED9AE00E945AA703C0C8010E94AE
:105E8000B0CC8E2D8470FF2039F0811105C06F2DAC
:105E9000C8010E94A0CC69C3882309F466C3FF200F
:105EA00079F0AF2DB0E020E432E44FE050E00E9402
:105EB000E4DAAB01BC0182ED95E00E94D4D40DC0C0
:105EC000CE0145960E94D0D48FE0FE017596A2EDDA
:105ED000B5E001900D928A95E1F784E08093D105B9
:105EE0008091D00584708093D0054FE050E069E147
:105EF00070E089EC98E00E943E486091D10583ED06
:105F00009AE00E94BBAA41E060E170E089EC98E071
:105F10000E945F4586E090E09093E2058093E10562
:105F200024C3812F8358823008F043C08091F40548
:105F30009091F505089708F418C30E943A280E942A
:105F40003A28082F0E9407286B017C010E942C2808
:105F5000DC014091ED055091EE056091EF057091E7
:105F6000F0054F5F5F4F6F4F7F4F4093ED055093AC
:105F7000EE056093EF057093F00583E090E0909359
:105F8000E2058093E10520E432E44FE050E00E9416
:105F9000E4DAAB01BC0182ED95E00E94D4D481E04B
:105FA000143809F080E0A7019601602F0E94258235
:105FB000DCC2173851F48091F4059091F5050697ED
:105FC00008F4D3C284E090E00BC01D38C9F580917D
:105FD000F4059091F505069708F4C7C285E090E0B6
:105FE0009093E2058093E1050E943A280E943A28A6
:105FF0008093F1050E942C280E942C284091ED05E9
:106000005091EE056091EF057091F0054F5F5F4F85
:106010006F4F7F4F4093ED055093EE056093EF0572
:106020007093F005DC0120E432E44FE050E00E9480
:10603000E4DAAB01BC0182ED95E00E94D4D495C2B4
:106040001F3809F06EC08091F4059091F505029714
:1060500008F48BC20E943A280E943A284091ED052C
:106060005091EE056091EF057091F0054F5F5F4F25
:106070006F4F7F4F4093ED055093EE056093EF0512
:106080007093F00524E2E22E22E0F22E00E010E010
:10609000C82ED12C38EE832E33E0932EA12CB12CB8
:1060A000C601002E02C0959587950A94E2F780FFFD
:1060B0002EC0CE0101960E94F37DB801CE0101965B
:1060C0000E94FF4EFC0160817181828193816CA3EB
:1060D0007DA38EA39FA3402F0E94457B20E030E04C
:1060E0004AE754E40E94E6D90E94AFD8A501940182
:1060F0000E94AFDA2CA33DA34EA35FA3F89444E023
:1061000050E0B701CE0184960E9401DD78940F5FC4
:106110001F4FF4E0EF0EF11C0530110509F0C0CF60
:1061200024C2103909F06DC08091F4059091F505F5
:10613000029708F41AC20E943A280E943A28C82EF0
:106140004091ED055091EE056091EF057091F005DD
:106150004F5F5F4F6F4F7F4F4093ED055093EE05BC
:106160006093EF057093F005AA24A394B12CAC0EB4
:10617000BD1EC5010E94F37D94E2E92E92E0F92E46
:1061800000E010E0D12C9A2C8B2CC601002E02C00E
:10619000959587950A94E2F780FF26C0F894B80198
:1061A000892D982D0E94074F44E050E0B7010E94CE
:1061B000EBDC7894B801892D982D0E94074F5C0183
:1061C000B801892D982D0E94074FFC0160817181D3
:1061D000828193810E94E2D8402F0E945E7BF5016C
:1061E00060837183828393830F5F1F4FF4E0EF0E10
:1061F000F11C0530110549F6CE0101960E94027D81
:10620000B4C1113939F58091F4059091F5050397E2
:1062100008F4ABC10E943A280E943A28182F0E9425
:106220003A284091ED055091EE056091EF0570918F
:10623000F0054F5F5F4F6F4F7F4F4093ED055093D9
:10624000EE056093EF057093F005682F812F0E9493
:10625000D8828BC11239A9F58091F4059091F5058A
:10626000069708F482C10E943A280E943A28182F03
:106270000E943A288FAB0E943A288EAB0E943A289F
:10628000082F0E943A28C090ED05D090EE05E090CE
:10629000EF05F090F0052FEFC21AD20AE20AF20AD7
:1062A000C092ED05D092EE05E092EF05F092F00578
:1062B000802F0E94DB8A4EA96FA9812F0E945C8AE1
:1062C00054C1133951F58091F4059091F505069765
:1062D00008F44BC10E943A280E942C288C010E948D
:1062E0002C287C010E943A284091ED055091EE0542
:1062F0006091EF057091F0054F5F5F4F6F4F7F4FDB
:106300004093ED055093EE056093EF057093F00513
:10631000B701C8010E94034E28C11838D9F58091F1
:10632000F4059091F505049708F41FC18091F605D6
:106330009091F7052091F4053091F5050396609151
:10634000F2057091F3050E9465DAE091F805F0918D
:10635000F905E80FF91F808190E0049628173907A6
:1063600008F403C10E943A288091ED059091EE0552
:10637000A091EF05B091F0050196A11DB11D80938C
:10638000ED059093EE05A093EF05B093F0050E9404
:106390003E28EBC0163931F58091F4059091F50552
:1063A000039708F4E2C00E943A280E943A28182F66
:1063B0000E943A284091ED055091EE056091EF055D
:1063C0007091F0054F5F5F4F6F4F7F4F4093ED052A
:1063D0005093EE056093EF057093F005812F0E94B6
:1063E000A7A6C3C0173911F58091F4059091F50562
:1063F000029708F4BAC00E943A280E943A284091B5
:10640000ED055091EE056091EF057091F0054F5F3D
:106410005F4F6F4F7F4F4093ED055093EE056093B4
:10642000EF057093F0050E946A4E9FC0183931F550
:106430008091F4059091F505029708F496C00E94AA
:106440003A280E943A288091ED059091EE05A0919E
:10645000EF05B091F0050196A11DB11D8093ED05EA
:106460009093EE05A093EF05B093F0050E941836C7
:1064700060E089EC98E00E94204C77C0193951F512
:106480008091F4059091F505059708F46EC00E947F
:106490003A280E9407288091ED059091EE05A09181
:1064A000EF05B091F0050196A11DB11D8093ED059A
:1064B0009093EE05A093EF05B093F00582EF95E081
:1064C0000E94803C81E08093B10589EC98E00E94B5
:1064D000D1474BC01A3911F58091F4059091F5051B
:1064E000029708F442C00E943A280E943A2840913C
:1064F000ED055091EE056091EF057091F0054F5F4D
:106500005F4F6F4F7F4F4093ED055093EE056093C3
:10651000EF057093F0050E94993D27C01C3929F5BD
:106520008091F4059091F5050297F8F00E943A28C1
:106530000E943A284091ED055091EE056091EF05DB
:106540007091F0054F5F5F4F6F4F7F4F4093ED05A8
:106550005093EE056093EF057093F00591E0813064
:1065600009F090E0892F0E94E3828091ED059091DF
:10657000EE05A091EF05B091F00581309A4CAA4943
:10658000BB4308F416C181E09AECAAE9BBE380930F
:10659000ED059093EE05A093EF05B093F00509C1CA
:1065A0000E94F650811129C00C948D298091E40538
:1065B0009091E505A091E605B091E7050196A11D32
:1065C000B11D8093E4059093E505A093E605B09393
:1065D000E7050E94F950682F82EF95E00E94BA27E4
:1065E0000C9479298091E3058F5F8093E3058630D1
:1065F00010F40C940C2A0C94A5290E94F6508111D9
:106600000C940C2A0C94FE290E9408510C940C2A1C
:106610000E947B8781110C94322A0C94242A0E94B8
:106620008987682F82EF95E00E94BA270C94102A80
:106630000E94EB870C94322A8091F105813011F091
:106640000C94C02A86ED99E00C94C22A87E00E943F
:106650006A4E1092E2051092E1050C94D82A8091BE
:10666000CD059091CE05029749F436C88091040279
:1066700090910502009709F022C81EC88091CD05AF
:106680009091CE058330910509F060C84FC80E94F3
:10669000BAA683E090E09093CE058093CD058091DB
:1066A000040290910502019709F026C81AC8CE018C
:1066B00045960E94D0D48FE0FE017596A2EDB5E01C
:1066C00001900D928A95E1F7109205021092040252
:1066D0000E94BAA621E040E061E973E089EC98E00D
:1066E0000E943D4564E180E00E94D88264E181E03F
:1066F0000E94D88264E183E00E94D88264E184E051
:106700000E94D88260E070E08FE399E00E948DA340
:1067100060E070E08EED99E00E948DA360E070E093
:106720008EE19CE00E948DA344C08630910509F063
:106730006EC856C88091040290910502019709F035
:1067400015C81CC883ED9AE00E9484AA1092CE0559
:106750001092CD051092EA052CC08091F40590911D
:10676000F505809708F401CF7AC98091F4059091DE
:10677000F505499708F4F9CEC1C88091F4059091C8
:10678000F5054A9708F4F1CE0DC98091F405909172
:10679000F505029708F0E9C9E8CE1D3909F0A8CA45
:1067A0001CCA8091F4059091F505029708F0C0C9C4
:1067B000DCCEE7960FB6F894DEBF0FBECDBFDF91FB
:1067C000CF911F910F91FF90EF90DF90CF90BF90EE
:1067D000AF909F908F907F906F905F904F903F9081
:1067E0002F90089540E065E87AE18CEF97E00E94F1
:1067F0001DD380E092E09093F3058093F205109210
:10680000F5051092F4051092F7051092F6058CEF3D
:1068100095E09093F9058093F8051092FA0510928F
:10682000FB0582ED95E00E94D0D483EB95E00C94BB
:10683000CA4E40E065E87AE188E298E00E941DD304
:1068400082E098E00C9497D2CF93DF9300D0CDB73D
:10685000DEB721E0298322E32A8342E050E0BC0135
:10686000CE0101960E9401DD0F900F90DF91CF9134
:106870000895CF93DF93EC0140E050E060EE70E4C8
:106880000E9417A146E656E666EA7EE3CE0102962E
:106890000E9417A140E050E060E172E4CE0104964E
:1068A000DF91CF910C9417A10F931F93CF93DF9398
:1068B000EB018B01085E1F4F892B31F467E0CE019D
:1068C0000E940BDD6CE005C068E3CE010E940BDD89
:1068D00060E2C8010E940BDDCE010A960E943934A5
:1068E000CE0140960E943934CE014A960E9424344B
:1068F00064EF71E0CE0106960E9421DD65E070E054
:10690000CE0102960E9421DD64EF71E0CE01049673
:106910000E9421DD6CE271E0CE010896DF91CF91FB
:106920001F910F910C9421DD0F931F93CF93DF9351
:1069300000D01F92CDB7DEB78C0160E00E940BDD66
:1069400061E0C80102960E940BDD8FEF89831B82F4
:106950001A82B8016C5F7F4F43E050E0CE01019690
:106960000E9401DD0F900F900F90DF91CF911F914A
:106970000F910895FF920F931F93CF93DF9300D051
:1069800000D0CDB7DEB7F82E062F1FB7F89468E019
:1069900080E491E04C830E940BDDF9820A834C81F4
:1069A0004B8343E050E064E471E0CE0101960E9425
:1069B00001DD1FBF0F900F900F900F90DF91CF91CF
:1069C0001F910F91FF90089561E00C940BDDCF9320
:1069D000DF93EC0166EE70E00E9421DD66EE70E070
:1069E000CE0102960E9421DD6EE670E0CE01049693
:1069F0000E9421DD65E0CE010696DF91CF910C94D7
:106A00000BDD61E08EE691E00E940BDD68EE73E045
:106A100082E791E00E9421DD68EE73E084E791E077
:106A20000E9421DD66E970E086E791E00E9421DDA9
:106A300060EA7FE088E791E00E9421DD60EA7FE084
:106A40008AE791E00E9421DD60ED77E080E791E048
:106A50000E9421DD60EA7FE086E891E00E9421DD6E
:106A60006AE070E08CE791E00E9421DD6AE070E06E
:106A70008EE791E00E9421DD6AE070E080E891E01D
:106A80000E9421DD6EE170E082E891E00E9421DD4C
:106A90006EE170E084E891E00E9421DD42E553E080
:106AA00060E070E088ED91E00E9419DD44E853E079
:106AB00060E070E08CED91E00E9419DD60E070E034
:106AC00080EE91E00E9421DD60E070E082EE91E0D6
:106AD0000E9421DD61E084EE91E00E940BDD60E820
:106AE00088E891E00C940BDDCF93CFB7F89440E1A8
:106AF00050E062E270E089EF92E00E9401DDCFBFDA
:106B0000CF910895EF92FF920F931F93CF93DF934E
:106B1000CDB7DEB72D970FB6F894DEBF0FBECDBF51
:106B20008DE0E9EFF2E0DE01119601900D928A9579
:106B3000E1F7EE24E394F12CEC0EFD1E02E210E0EE
:106B400060E0C8010E9466A0F70121917F0190E0FA
:106B5000332727FD30958217930739F40F5F1F4FB6
:106B60000E32110569F781E001C080E02D960FB665
:106B7000F894DEBF0FBECDBFDF91CF911F910F9173
:106B8000FF90EF90089561E082E490E00E9466A09B
:106B900091E0813009F090E0892F08951F93CF9301
:106BA000DF93CDB7DEB764970FB6F894DEBF0FBEA4
:106BB000CDBF84E1EBEBF2E0DE01119601900D9286
:106BC0008A95E1F70E94C335882381F088E990E037
:106BD000A0E0B0E089839A83AB83BC8388E490E033
:106BE000A0E0B0E08D839E83AF83B8871FB7F89491
:106BF00044E150E064E272E0CE0101960E9401DDC2
:106C00001FBF64960FB6F894DEBF0FBECDBFDF91F5
:106C1000CF911F910895CF93CFB7F894682F82E456
:106C200090E00E940BDD0E94CE35CFBFCF9108953A
:106C30001F93CF93DF93CDB7DEB729970FB6F894A4
:106C4000DEBF0FBECDBF85E0EFECF2E0DE011196B6
:106C500001900D928A95E1F70E9474351FB7F89460
:106C600081EC93E29F838E8384E094EB99878887FD
:106C700045E050E066E070E0CE0101960E9401DD43
:106C80006FE984E090E00E940BDD6BE18CE090E026
:106C90000E940BDD60E084E492E00E940BDD0E9424
:106CA000CE3560E080E592E00E940BDD44E150E0EB
:106CB00060E172E086E093E00E9401DD44E150E093
:106CC00064EA71E08AE193E00E9401DD4AE050E06D
:106CD00066E472E08EE293E00E9401DD0E940135DD
:106CE00060E070E080EA91E00E9421DD60E082EAED
:106CF00091E00E940BDD61E080E691E00E940BDDF7
:106D000088E591E00E94E73444E050E064E470E0FC
:106D1000CE0106960E9401DD60E071E080E090E027
:106D20000E9454346CE171E081E090E00E945434A0
:106D300080E491E00E9494348AE491E00E94E4347B
:106D400060E086E591E00E940BDD1FBF29960FB63B
:106D5000F894DEBF0FBECDBFDF91CF911F91089594
:106D600061E08CE490E00E9466A091E0813009F03F
:106D700090E0892F0895CF93CFB7F89480E491E005
:106D80000E9494348AE491E00E94E43488E591E022
:106D90000E94E73461E080E691E00E940BDD61E053
:106DA0008EE691E00E940BDD81E00E940B3660E0F0
:106DB00084E492E00E940BDD60E080E592E00E94B6
:106DC0000BDD60E08CE490E00E940BDDCFBFCF9143
:106DD00008951F93CF93DF93CDB7DEB72C970FB6EF
:106DE000F894DEBF0FBECDBF1FB7F89488EB98E8CC
:106DF000A0E0B0E089839A83AB83BC831D821E82AE
:106E00001F82188619861A861B861C864CE050E065
:106E100068E372E0CE0101960E9401DD1FBF2C964F
:106E20000FB6F894DEBF0FBECDBFDF91CF911F919B
:106E30000895FF920F931F93CF93DF93F82E162F91
:106E400060E070E080EA91E00E9483A0EC0160E0E5
:106E500082EA91E00E9466A0282F210F822F6CE326
:106E60000E9459DA092F2D3308F021961FB7F894A4
:106E7000BE016F0D711D80EA91E00E9421DD602F3F
:106E800082EA91E00E940BDD1FBFDF91CF911F913D
:106E90000F91FF9008951F93CF93DF9300D01F921F
:106EA000CDB7DEB70E94183619821A821B821FB72F
:106EB000F89467E182E090E00E940BDD61E082E4FB
:106EC00090E00E940BDD0E94E93660E08CE490E0E7
:106ED0000E940BDD61E088E092E00E940BDD43E060
:106EE00050E06AE072E0CE0101960E9401DD61E7A8
:106EF0008EE092E00E940BDD1FBF0F900F900F906D
:106F0000DF91CF911F9108951F93CF93DF93CDB75A
:106F1000DEB727970FB6F894DEBF0FBECDBF1D8238
:106F20001E821F821FB7F89444E150E060E172E0D6
:106F300086E093E00E9401DD44E150E064EA71E004
:106F40008AE193E00E9401DD4AE050E066E472E0ED
:106F50008EE293E00E9401DD0E9401350E94CE3551
:106F600061E088E092E00E940BDD43E050E06AE0DF
:106F700072E0CE0105960E9401DD61E78EE092E0AD
:106F80000E940BDD1FBF40E050E0BA0182E691E0B5
:106F90000E94A6A06C3326E9720721E682072EE93B
:106FA0009207A8F4A4E6B0E09B01AC010E94E4DAE9
:106FB00022E035E847E455E00E948DDA28513F474A
:106FC0004F4F5F4F29833A834B835C830EC022E08F
:106FD00035E847E455E00E948DDAA4E6B0E00E946F
:106FE000E4DA69837A838B839C830E94E9361FB736
:106FF000F89444E050E068E372E0CE0101960E940C
:1070000001DD1FBF27960FB6F894DEBF0FBECDBFC0
:10701000DF91CF911F91089540E065E87AE18EE21B
:1070200098E00C941DD3CF92DF92EF92FF920F93D2
:107030001F93CF93DF93EC018B018881811102C0F4
:1070400080E048C0DC2ECD2E60E0CE010E9478D2D8
:1070500087FFF6CF0E948B50882329F0CE010E9433
:107060008E5061E828C00E948850811123C00E9480
:10707000728781111FC020914F0830915008243031
:107080003105F1F417C06C2F8D2D9C2D0E9478D204
:107090000E94DB27219603C0C0E0D0E07901CE1525
:1070A000DF058CF361E801C062E8C8010E94CED21E
:1070B000789404C06AE8C8010E94CED281E00AC078
:1070C000F894C8810E94AD242C2F30E082179307DA
:1070D00018F7EACFDF91CF911F910F91FF90EF90BA
:1070E000DF90CF90089586E090E0909350088093D1
:1070F0004F0881E0809334080895CF93DF93EB012C
:1071000061E00E947DD261E84A9730F4CE010E948E
:10711000CED260E070E005C0CE010E94CED261EC1C
:1071200072E0CE01DF91CF910C94D0D2CF93DF9358
:10713000EB0161E00E947DD261E8CE010E94CED2D7
:1071400061EC72E0CE010E94D0D265E070E0CE0129
:107150000E94D0D261E0CE010E94CED260E0CE018A
:107160000E94CED260E070E0CE01DF91CF910C940E
:10717000D0D2EF92FF920F931F93CF93DF938B01A7
:1071800061E8C8010E94CED2C1E5D8E07E016991D4
:10719000C8010E94CED2F7018081882321F0F8E057
:1071A000C037DF0799F7DF91CF911F910F91FF90C3
:1071B000EF900895CF93DF93EB0161E8CE010E9439
:1071C000CED20E94AD24AC0160E070E0CE01DF9130
:1071D000CF910C94E5D20F931F93CF93DF93CDB74C
:1071E000DEB764970FB6F894DEBF0FBECDBF8B013C
:1071F000F894CE0101960E94F37D61E8C8010E94D7
:10720000CED260E070E0CE0101960E94FF4EFC01FC
:107210004081518162817381C8010E94E5D261E0A1
:1072200070E0CE0101960E94FF4EFC014081518129
:1072300062817381C8010E94E5D262E070E0CE01F4
:1072400001960E94FF4EFC01408151816281738151
:10725000C8010E94E5D20E94F582682FC8010E94F1
:10726000CED2789464960FB6F894DEBF0FBECDBF31
:10727000DF91CF911F910F9108950F931F93CF939B
:10728000DF93CDB7DEB764970FB6F894DEBF0FBEBD
:10729000CDBF8B01F894CE0101960E94F37D61E889
:1072A000C8010E94CED260E070E0CE0101960E943B
:1072B000FF4EFC014081518162817381C8010E94AF
:1072C000E5D261E070E0CE0101960E94FF4EFC0124
:1072D0004081518162817381C8010E94E5D262E0E0
:1072E00070E0CE0101960E94FF4EFC014081518169
:1072F00062817381C8010E94E5D263E070E0CE0133
:1073000001960E94FF4EFC01408151816281738190
:10731000C8010E94E5D264E070E0CE0101960E94AF
:10732000FF4EFC014081518162817381C8010E943E
:10733000E5D20E94F582682F70E0C8010E94D0D289
:10734000789464960FB6F894DEBF0FBECDBFDF9180
:10735000CF911F910F9108950F931F93CF93DF93B8
:107360008C01EB0161E8CE010E94CED2C8010396E8
:107370000E94CF51682FCE01DF91CF911F910F91C5
:107380000C94CED2CF93DF93EB0161E8CE010E9443
:10739000CED20E94B650AB01BC01CE010E94E5D214
:1073A000DF91CF910C9419518F929F92AF92BF921F
:1073B000CF92DF92EF92FF920F931F93CF93DF93C1
:1073C000CDB7DEB77C018B01CDB6DEB69EB6BDB6BD
:1073D000AEB661E8C8010E94CED261E0C7010E944A
:1073E00078D2882379F00E940E52009759F0682FC6
:1073F000C8010E94CED260E0C8010E94CED23C2DCE
:10740000292D2FC08DB79EB74F970FB6F8949EBF0A
:107410000FBE8DBFEDB6FEB6EFEFEE1AFE0A40E0EE
:1074200050E06FE1C7010E948C4FF70120812223B9
:1074300021F0009711F42E3291F3682FC8010E94B9
:10744000CED2912CE92DF0E08FE1981629F0EE0DC7
:10745000FF1D608161110DC060E0C8010E94CED2A5
:107460009501832F922F0FB6F8949EBF0FBE8DBF4C
:1074700005C0C8010E94CED29394E4CF0FB6F89411
:10748000DEBE0FBECDBEDF91CF911F910F91FF9059
:10749000EF90DF90CF90BF90AF909F908F90089526
:1074A000CF93DF93EB0161E8CE010E94CED2F89436
:1074B0000E94DC65882351F00E94C824882331F0A3
:1074C00061E0CE010E94CED2789402C060E0F9CF94
:1074D000DF91CF9108957F928F929F92AF92BF924A
:1074E000CF92DF92EF92FF920F931F93CF93DF9390
:1074F000CDB7DEB78C015B018DB69EB661E00E9410
:107500007DD27C0163E0C8010E9478D2C82ED12CC4
:107510002DB73EB72C193D090FB6F8943EBF0FBEEC
:107520002DBF0DB71EB70F5F1F4F7FB6F894482FC2
:1075300050E0B701C8010E94EBDC7FBE61E8C501E5
:107540000E94CED2780106C0F80161918F01C50179
:107550000E94CED2C8018E199F098C159D05A4F3F7
:107560000FB6F8949EBE0FBE8DBEDF91CF911F91D6
:107570000F91FF90EF90DF90CF90BF90AF909F90D2
:107580008F907F9008952F923F924F925F926F92CB
:107590007F928F929F92AF92BF92CF92DF92EF92A3
:1075A000FF920F931F93CF93DF931F92CDB7DEB758
:1075B000882E792E6B012DB63EB661E00E947DD2F9
:1075C000582E692E63E0882D972D0E9478D2982E30
:1075D000A82EB12C8DB79EB78A199B090FB6F894C7
:1075E0009EBF0FBE8DBF0DB71EB70F5F1F4FFFB6FB
:1075F000F894402E1983492D50E0652D762DC80151
:107600000E94EBDCFFBE780100E010E00BC0602FB1
:107610006C5F882D972D0E9478D2F70181937F01AE
:107620000F5F1F4F0A151B0594F31FB7F894492DE0
:1076300050E0652D762D842D99810E9401DD1FBFBC
:1076400061E8C6010E94CED2692DC6010E94CED249
:107650000FB6F8943EBE0FBE2DBE0F90DF91CF91B6
:107660001F910F91FF90EF90DF90CF90BF90AF9060
:107670009F908F907F906F905F904F903F902F9052
:1076800008950F931F93CF93DF931F92CDB7DEB76B
:107690008B0161E00E9478D280FF04C089830E9440
:1076A000C183898181FD0E94D12461E8C8010E94C3
:1076B000CED260E0C8010F90DF91CF911F910F9162
:1076C0000C94CED2CF93DF93EC0161E80E94CED22E
:1076D00060919F0CCE01DF91CF910C94CED210928D
:1076E000700808950F931F93CF93DF9380917008D4
:1076F000882329F080917008882389F01DC000E755
:1077000018E0C2E2D0E060E0CE010E9466A0F8017D
:1077100081938F012196C233D105A9F7EBCFE5E81C
:10772000F4E0A0E7B8E084918D93319684E0E339EA
:10773000F807C9F710927E0880E798E0DF91CF91B3
:107740001F910F91089581E598E0089580914F0869
:10775000909150080895CF93DF9383ED9AE00E94B3
:107760004CA781E598E00E949151EC01009789F4C3
:107770000E94D1240E94C1830E94D18360E089ECE1
:1077800098E00E94C74B82E090E09093500880936D
:107790004F08CE01DF91CF910895CF92DF92EF9203
:1077A000FF920F931F93CF93DF938C017B0161E8CE
:1077B000C7010E94CED281E5C82E88E0D82EC1E054
:1077C000D0E008C06C2FC8010E9478D2F6018193E6
:1077D0006F012196F801808190E0C817D90794F3D2
:1077E00010926F080E94AB3B682FC701DF91CF91C9
:1077F0001F910F91FF90EF90DF90CF900C94CED21D
:107800000E94A6878823B9F085E090E09093500805
:1078100080934F0883ED9AE00E9443A741E064E023
:1078200070E089EC98E00E945F450E94D1240E949C
:10783000C1830C94D1830895CF93C82F0E94C22492
:10784000C817C9F08C2F0E94BB24CC2341F083E0E1
:1078500090E090934E0880934D0861E007C081E06E
:1078600090E090934E0880934D0860E087E398E0A5
:10787000CF910C942AD5CF910895CF93DF93EB014C
:107880000E94C22491E089270E941C3C61E8CE013D
:10789000DF91CF910C94CED21F93CF93DF93182F0B
:1078A000EB010E94C5241817E1F0112341F025E0F7
:1078B00030E030934E0820934D0861E007C021E08E
:1078C00030E030934E0820934D0860E087E398E065
:1078D0000E942AD5BE01812FDF91CF911F910C9478
:1078E0006027DF91CF911F91089540E054EA63E94A
:1078F00076ED87E398E00E94D4D41092460808956C
:10790000CF92DF92EF92FF920F931F93CF93DF936B
:10791000CDB7DEB76F970FB6F894DEBF0FBECDBF01
:10792000FC0180914F08909150088130910509F435
:107930004DC024F4892B09F443C075C082309105F1
:1079400021F0059709F06FC041C09E012F5F3F4FA6
:107950006E0180E2C80ED11C41E082819381892BA7
:1079600019F4418780E01AC084819581E080F1801C
:10797000B7010E9465DA06811781080F191F8481FB
:1079800095810196B7010E9465DA9583848382818F
:107990009381019793838283D8018C91D9018D9330
:1079A0009D01882309F44AC0AC15BD05B1F646C057
:1079B000BE016F5F7F4F81E598E00E94BCDC33C061
:1079C00081E090E09093500880934F0821E538E0E3
:1079D00041E082819381892B19F4418780E01AC0AC
:1079E00084819581E080F180B7010E9465DA06818B
:1079F0001781080F191F848195810196B7010E9494
:107A000065DA95838483828193810197938382834E
:107A1000D8018C91D9018D939D01882321F0B8E084
:107A200020373B07B1F60E94753C0E940F2581E08C
:107A300090E090934E0880934D0809C068E373E08E
:107A4000CE0101960E94B3DC009769F3B1CF6F9627
:107A50000FB6F894DEBF0FBECDBFDF91CF911F915F
:107A60000F91FF90EF90DF90CF90089587E398E01B
:107A70000E94F8D4882369F040E054EA63E976ED87
:107A800087E398E00E94D4D4809146088F5F80936A
:107A900046080895CF93DF93EB0120913708211119
:107AA00008C020914C08FC01208380914B088883FA
:107AB0000FC020914608FC01208387E398E00E94D4
:107AC00059D520E037E843E953E00E948DDA288356
:107AD000DF91CF910895CF93DF93CDB7DEB72F9786
:107AE0000FB6F894DEBF0FBECDBF6BE478E08CE438
:107AF00098E00E944A3D60914B0880914C080E949A
:107B00001937CE0101960E94D0D48FE0FE01319644
:107B1000A7E3B8E001900D928A95E1F7109246082C
:107B20002F960FB6F894DEBF0FBECDBFDF91CF9179
:107B30000895CF93DF9300D000D000D0CDB7DEB74B
:107B400061E070E083ED9AE00E94B3A70E946B3D74
:107B50000E9406256093470870934808809349085F
:107B600090934A0882E090E090934E0880934D08ED
:107B70001092500810924F0860E083E00E94BF828C
:107B800060E084E00E94BF8245E06FE87AE1CE01C8
:107B900001960E941DD360E0CE0101960E946CD335
:107BA00026960FB6F894DEBF0FBECDBFDF91CF9102
:107BB00008950F931F93CF93DF93CDB7DEB76697EA
:107BC0000FB6F894DEBF0FBECDBF80914F089091E5
:107BD00050080197029708F077C00E94C18360E0C7
:107BE00083E00E94BF8260E084E00E94BF8241E0A7
:107BF00060E270E089EC98E00E945F450E940625F3
:107C000060934708709348088093490890934A0806
:107C10000E946B3D62E070E081E00E946027BE013F
:107C20006B5E7F4FCE0146960E944A3D0E94BC8605
:107C3000182F882309F444C0CE0101960E945F7D6D
:107C400062E070E0CE010196113059F40E94074FB6
:107C50008C0182E00E942F7B20E030E041E153E480
:107C60000AC00E94074F8C0182E00E942F7B20E017
:107C700030E046E153E40E94E6D90E94AFD8F80113
:107C8000608371838283938380E00E94BB2446E9F2
:107C900050E060E070E0CE0101960E94897E64E9C8
:107CA00074E083ED9AE00E94F7A781E08093070CCF
:107CB00040E856E968E970E080E898E00E94D4D492
:107CC00089EC98E00E94C74780914F089091500836
:107CD0000197B9F480914D0890914E08049789F06E
:107CE00084E090E09093500880934F0881E0809367
:107CF000340840E452E46FE070E08FE898E00E94BE
:107D0000D4D48091B509811118C08091540A811191
:107D100014C080E00E94437840E064E070E089ECA9
:107D200098E00E945F4581E08093360884E090E00F
:107D300090934E0880934D080BC060E08FE399E06C
:107D40000E94C3A460E08EED99E00E94C3A4E1CF3D
:107D500066960FB6F894DEBF0FBECDBFDF91CF9110
:107D60001F910F9108950F931F93CF93DF9300D02E
:107D7000CDB7DEB78C0161E80E94CED2BE016F5F45
:107D80007F4FCE0102960E944A3D60914D08C80186
:107D90000E94CED26A81C8010E94CED26981C801F8
:107DA0000E94CED280914D0890914E08813091056D
:107DB00029F08330910511F0059729F40E940625DA
:107DC000AB01BC0108C04091470850914808609140
:107DD000490870914A08C8010E94E5D240E050E08D
:107DE000BA01C8010E94E5D20F900F90DF91CF91A8
:107DF0001F910F910895EF92FF920F931F93CF93CE
:107E0000DF937C01EB01FC018081882309F4F2C03F
:107E100061E0C7010E9478D2082F62E0C7010E948A
:107E200078D2803209F446C060F4823001F118F44F
:107E30008823B1F0DFC0863139F18E3109F0DAC024
:107E400030C0833209F44CC020F4813209F0D2C032
:107E50003EC0843209F44EC0853209F0CBC082C0E6
:107E600061E8CE010E94CED261EC72E0BEC061E852
:107E7000CE010E94CED2013019F486ED99E002C005
:107E800087E399E0089613C061E8CE010E94CED244
:107E9000013019F486ED99E002C087E399E0089675
:107EA00025C061E8CE010E94CED28EE19CE00E9406
:107EB00069A49AC061E8CE010E94CED2013019F4C3
:107EC00086ED99E002C087E399E0089606C061E874
:107ED000CE010E94CED28EE19CE00E9463A484C0B9
:107EE00061E8CE010E94CED28EE19CE00E943FA4C8
:107EF000682F34C061E8CE010E94CED2013019F45F
:107F000086ED99E002C087E399E008960E9471A689
:107F1000882311F010E801C010E08EE19CE00E947F
:107F200071A6882311F080E401C080E0182B013095
:107F300019F486ED99E002C087E399E008960E9463
:107F400076A6182B013019F486ED99E002C087E37C
:107F500099E008960E943FA4612F682BCE010E94F1
:107F6000CED246C061E8CE010E94CED2013019F4D3
:107F700086ED99E002C087E399E008960E946EA41E
:107F8000BC01CE010E94D0D2013019F486ED99E0F7
:107F900002C087E399E008960E9471A4BC01CE015B
:107FA0000E94D0D2013019F486ED99E002C087E337
:107FB00099E008960E9474A4BC01CE010E94D0D220
:107FC0008EE19CE00E946EA4BC01CE010E94D0D242
:107FD0008EE19CE00E9471A4BC01CE010E94D0D22F
:107FE0008EE19CE00E9474A4BC01CE010E94D0D21C
:107FF00081E001C080E0DF91CF911F910F91FF9050
:10800000EF9008950F931F93CF93DF938C01EB01B3
:10801000FC018081811101C08FC060E0C8010E9415
:1080200078D287FD89C0E82FF0E0EC31F10508F047
:1080300083C0EE58FF4F0C94CBDABE01C8010E94FA
:108040007D3878C0BE01C8010E94B93873C08091E4
:108050004F08909150089C01215031092230310580
:1080600010F0059779F484E090E090934E088093A7
:108070004D080E94D93D64E070E089EC98E00E94D0
:10808000074803C081E08093360861E8CE010E9472
:10809000CED250C0BE01C8010E94DA384BC0BE012A
:1080A000C8010E94EB3846C0BE01C8010E943D399C
:1080B00041C0BE01C8010E94AC393CC0BE01C8012C
:1080C0000E94C23937C0BE01C8010E94CD3B32C0F8
:1080D000BE01C8010E94D4392DC0BE01C8010E9452
:1080E0003D3C28C0BE01C801DF91CF911F910F9187
:1080F0000C94FB3EBE01C8010E94503A1BC0BE0159
:10810000C8010E946B3A16C0BE01C8010E94C33A62
:1081100011C0BE01C8010E94413B0CC0CE010E94AB
:10812000623B08C0CE010E94B33E04C0BE01C8013C
:108130000E94963881E001C080E0DF91CF911F91CD
:108140000F910895CF93DF93CDB7DEB72F970FB67A
:10815000F894DEBF0FBECDBF80914D1D90914E1D96
:10816000892B09F407C180914D1D90914E1D0497F4
:1081700009F01BC1FFC080913408811106C08091B5
:108180008008882309F4FBC007C08FE898E00E94AC
:10819000F8D48111F4CFFCC080E898E00E94F8D4B4
:1081A0008111EDC00E94DC658111E9C0F1C083300E
:1081B000910511F0059741F484E090E090934E080A
:1081C00080934D080E94D93D1092360810923408D1
:1081D000CE0101960E94D0D48FE0FE013196AFE827
:1081E000B8E001900D928A95E1F7CE0101960E94C8
:1081F000D0D48FE0FE013196A0E8B8E001900D9256
:108200008A95E1F7809135080E94F5411092350872
:10821000CE0101960E94D0D48FE0FE013196AEE9E6
:10822000B8E001900D928A95E1F7109270081092D3
:1082300051081092500810924F08B7C08091271D26
:108240009091281D049709F0ABC016C040E45DE092
:1082500063E070E08EE998E00E94D4D40DC08EE90E
:1082600098E00E94F8D4882339F084E09DE10E94D0
:1082700017D284E08093261D8091261D882321F04B
:1082800084E09DE10E9425D28091271D9091281DB8
:10829000049709F049C08EE998E00E9424D58AE24B
:1082A0009DE10E948FD280914F08909150082091BB
:1082B0003408069761F4222341F069E88AE29DE1DF
:1082C0000E94CED21092340827C06BE821C022232E
:1082D00071F069E88AE29DE10E94CED210923408E2
:1082E00066E070E089EC98E00E94074815C06AE2F9
:1082F0007DE184E09DE10E94133881110DC06AE2A6
:108300007DE184E09DE10E940240811105C065E8A5
:108310008AE29DE10E94CED284E09DE10E9425D2B6
:1083200080E09DE10E94AFD580914F089091500868
:10833000029741F40E948850811104C010925008A5
:1083400010924F0880914F0890915008059779F44A
:108350000E947287811104C01092500810924F0839
:1083600040E064E070E089EC98E00E945F450E9484
:10837000363D1BC0809136088111FDCE09C0809129
:108380004D0890914E088130910509F010CF14CF1F
:108390008091271D9091281D892B09F04FCF6CCF1C
:1083A00080919E0881115BCF51CF2F960FB6F89424
:1083B000DEBF0FBECDBFDF91CF91089540E065E8ED
:1083C0007AE18DEA98E00E941DD38EE998E00E9440
:1083D000D0D48FE898E00E94D0D480E898E00E9442
:1083E000D0D487E398E00C94D0D4CF93DF931F923E
:1083F000CDB7DEB7F89494B78823A1F098E10FB613
:10840000F89490936000109260000FBE14BE99E241
:1084100028E130E00FB6F894A895209360000FBED5
:108420009093600089830E9419510E940A4D0E9416
:1084300075870E94D1240E9430A00E945E7C0E9419
:10844000C1830E94D1838981682F89EC98E00E94C2
:10845000204C78940F90DF91CF910895CF93DF93C4
:1084600000D000D000D0CDB7DEB747E06BE97AE1AD
:10847000CE0101960E941DD361E0CE0101960E94BB
:108480004CD347E06BE97AE1CE0101960E941DD3FF
:1084900060E0CE0101960E946CD389EC98E00E94C6
:1084A000FC4381E00E94F54178940E94A2400E9422
:1084B0005A2989EC98E00E947E480E945A4EA8955D
:1084C000F4CF40E065E87AE183EB98E00C941DD3AB
:1084D0000F931F93CF93DF9300D000D000D0CDB780
:1084E000DEB7062F1FB7F89445E06DE87AE1CE01BC
:1084F00001960E941DD361E0011101C060E0CE0130
:1085000001960E946CD31FBF26960FB6F894DEBF6B
:108510000FBECDBFDF91CF911F910F910895CF93E3
:10852000DF9300D000D000D0CDB7DEB71092C108E5
:108530001092C00842E067E97AE1CE0101960E94FC
:108540001DD360E0CE0101960E946CD342E067E942
:108550007AE1CE0101960E941DD360E0CE01019622
:108560000E946CD326960FB6F894DEBF0FBECDBF27
:10857000DF91CF9108956F927F928F929F92AF92E9
:10858000CF92EF92FF920F931F93CF93DF93CDB7CC
:10859000DEB768970FB6F894DEBF0FBECDBF4C01B3
:1085A00004960E94D0D4C40143960E94D0D4C40142
:1085B00082960E94D0D4C401C1960E94D0D446E0D5
:1085C00063E97AE1CE0101960E941DD347E063E999
:1085D0007AE1CE0107960E941DD342E063E97AE179
:1085E000CE010D960E941DD342E06DE87AE1CE01E6
:1085F00043960E941DD38E010F5F1F4F9E01295F7E
:108600003F4FAE01435F5F4FBE016D5E7F4FC401C0
:10861000805C9F4F0E94FB8B44E06DE87AE1C801CB
:108620000E941DD345E063E97AE1CE0107960E94DE
:108630001DD3E12CFF24F39400E09E012F5F3F4FF8
:10864000AE01495F5F4F60E0C40182599F4F0E94B5
:108650001B8944E063E97AE1CE0101960E941DD3B3
:1086600043E063E97AE1CE0107960E941DD39CE1C5
:10867000E92EFF24F39401E09E012F5F3F4FAE01EE
:10868000495F5F4F61E0C401835F9E4F0E941B8979
:10869000C40184559E4F0E94D0D4C40185549E4F7E
:1086A0000E94D0D4840106531E4FC80102960E9436
:1086B000D0D4C80141960E94D0D441E067E97AE164
:1086C000CE0101960E941DD340E067E97AE1CE0118
:1086D00007960E941DD343E067E97AE1CE010D962B
:1086E0000E941DD3340182E1681A8EEF780A9E0140
:1086F0002F5F3F4FAE01495F5F4FBE01635F7F4F0A
:10870000C3010E94FDAAA301B801C401865F9D4F69
:108710000E94CFA63401EFEB6E1AECEF7E0A40E028
:1087200063E0C3010E94B7D4A4014D5A5C4F89E4B1
:1087300093E0FA019183808322E0A22EC12C30E1E4
:10874000E32EFF24F39400E211EA27E030E0B301C6
:10875000C4018B5A9C4F0E944EA261E08CE490E0D1
:108760000E9466A0F401E153FC4F91E0811101C029
:1087700090E0908368960FB6F894DEBF0FBECDBF31
:10878000DF91CF911F910F91FF90EF90CF90AF901D
:108790009F908F907F906F9008950E944F4D109200
:1087A00020018AE0809321011092220180E090E272
:1087B000909329018093280182E080937300809335
:1087C000B00094E09093B10099E19093B3001092BF
:1087D000B4008093700081E0809390008BE08093E0
:1087E0009100109299001092980010929D001092A2
:1087F0009C001092710008950F931F93CF93DF9305
:1088000000D000D000D0CDB7DEB78C0183E49DE06E
:108810000E94AD520E9482A6F801E359FF4F808367
:10882000F8011082118212821382C8010E94CD4386
:1088300047E069E97AE1CE0101960E941DD361E02B
:10884000CE0101960E944CD344E06FE87AE1CE015C
:1088500001960E941DD361E0CE0101960E944CD387
:1088600043E06FE87AE1CE0101960E941DD361E0FA
:10887000CE0101960E944CD347E06DE87AE1CE012B
:1088800001960E941DD361E0CE0101960E944CD357
:1088900040E061E97AE1CE0101960E941DD361E0DA
:1088A000CE0101960E944CD341E061E97AE1CE010C
:1088B00001960E941DD361E0CE0101960E944CD327
:1088C00042E061E97AE1CE0101960E941DD361E0A8
:1088D000CE0101960E944CD3C801805C9F4F0E943C
:1088E0007E8C40E950ED63E070E0C801C1960E94C3
:1088F000D4D4C80182599F4F0E947889C801835FF0
:108900009E4F0E94788945E06DE87AE1CE0101969C
:108910000E941DD361E0CE0101960E944CD3C80194
:108920008F5B9C4F0E94B1D4C8018B5A9C4F0E9410
:108930005AA140E251EA67E070E0C80185549E4FB9
:108940000E94D4D426960FB6F894DEBF0FBECDBFDA
:10895000DF91CF911F910F9108950F931F934FB700
:10896000F894FC0100811181228133814FBFB8014D
:10897000C9011F910F9108950E94C22481112DC039
:10898000809170008D7F80937000809173008D7F47
:108990008093730078940E948486F894809170008C
:1089A0008260809370008091730082608093730076
:1089B0002091240130912501809128019091290175
:1089C0002817390750F081E090E0909329018093B7
:1089D000280110922501109224010895CF93DF936E
:1089E000EC01FC01EC52FC4F718360836230710535
:1089F000E1F48B5A9C4F0E9471A681111BC00E940A
:108A0000C3358823B9F0CE018A589F4F0E9471A6C2
:108A10008823A1F0CE018B5E9E4F0E9471A681112A
:108A200009C00CC081E08093C808C053DC4F81E0CE
:108A3000888304C08091C8088823A1F3DF91CF9177
:108A40000895CF93DF93EC0189E18093C5088FE00F
:108A50008093C40881E090E09093C1088093C0089F
:108A60006FEFCE01865F9D4F0E94BBAACF52DC4FB5
:108A700081E08883DF91CF9108950F931F93CF9367
:108A8000DF931F92CDB7DEB78C01FC01EE52FC4F95
:108A90002083865F9D4F49830E94F7A7C8010E94EB
:108AA000214580E00E946A4EF801ED52FC4F498159
:108AB00040830F90DF91CF911F910F910895FC019A
:108AC000EA52FC4F442321F08081862B8083089555
:108AD00060958081682360830895CF93DF93EC01D4
:108AE0008A589F4F0E9477A481110EC0CE018B5EE1
:108AF0009E4F0E9477A4811107C0CE018B5A9C4FD4
:108B0000DF91CF910C9477A481E0DF91CF9108950C
:108B1000FC01E152FC4F31E03083FC01E052FC4F9C
:108B20006083FC01EF51FC4F4083FC01EE51FC4F90
:108B30002083FC01ED51FC4F10820895EF92FF92CB
:108B40000F931F93CF93DF93EC01FC01E152FC4F95
:108B500010828C0102511E4FFC01E052FC4F7C013F
:108B60008FE1E81A8CEFF80A4081F7016081C801B3
:108B70000E9485ADF701F080CE51DC4F06C063E462
:108B800073E0C8010E9480ACF3948881F816B8F3B2
:108B9000DF91CF911F910F91FF90EF9008959F92D9
:108BA000AF92BF92CF92DF92EF92FF920F931F93FB
:108BB000CF93DF93EC01D62E142FC22E241708F486
:108BC00078C030E0241B3109802F90E02817390746
:108BD0000CF46FC0FE01E452FC4F608171811616E7
:108BE0001706F4F4FE01E652FC4FCE0188529C4F6A
:108BF0000190F081E02DDC018D919C91E81BF90B37
:108C0000F7FF03C0F195E195F109E29FC001E39FF1
:108C1000900DF29F900D11240E9479DA962E01C0DA
:108C2000912C9016A8F47E01B2E1EB1ABEEFFB0A7C
:108C30004D2D612FC7010E9485AD012F06C063E451
:108C400073E0C7010E9480AC0F5F0C11F8CF00E009
:108C50007E0182E1E81A8EEFF80A602F610F4D2D38
:108C6000C7010E9485ADC12CD12C10E0A92CB12CDC
:108C700007C06FEFC7010E94C8ADAFEFCA1ADA0A8A
:108C80009601200F311F2A153B059CF3C252DC4F81
:108C9000888191E089278883882331F06DEB74E027
:108CA000C7010E9497AC06C06FEFC7010E94C8AD14
:108CB00001C0912C892DDF91CF911F910F91FF90D1
:108CC000EF90DF90CF90BF90AF909F900895BF92AC
:108CD000CF92DF92EF92FF920F931F93CF93DF9388
:108CE000EC018C0106521C4FF80111821082FC012C
:108CF000E452FC4F118210827C01F8E2EF1AFCEF83
:108D0000FF0AF701118210820E946D45882309F441
:108D1000C3C06E01FBEACF1AFCEFDF0AC6010E9456
:108D200077A48823D9F0C6010E94ADA4880F991FAB
:108D3000F70120813181280F391F31832083C6013B
:108D40000E9463A4880F991FF80120813181280FA8
:108D5000391F3183208306EE10E01AC0FE01E45172
:108D6000FF4F8081882331F060E0CE018A589F4F09
:108D70000E94C3A4FE01E557FE4F8081882331F095
:108D800060E0CE018B5E9E4F0E94C3A400E010E025
:108D90007E01F6E7EF0EF11CC7010E9477A488233D
:108DA00039F0FE01E451FF4F8081882309F4A1C00E
:108DB0007E018BEEE81A8EEFF80AC7010E9477A4B5
:108DC000882339F0FE01E557FE4F8081882309F49E
:108DD000ABC0FE01E652FC4F80819181FE01E8525A
:108DE000FC4F20813181FE01E452FC4F8217930732
:108DF0002CF4081B190B1183008302C0918380831C
:108E000080819181892B09F452C061E082E491E074
:108E10000E9466A0882309F44AC067E080E491E0DC
:108E20000E9466A0873009F09AC041C081E080832B
:108E3000FE01E852FC4FA081B181FE01E452FC4FDB
:108E4000C080D180EE24D7FCE094FE2CFE01E652D7
:108E5000FC4F008111810A1B1B0B17FF03C01195EA
:108E6000019511092FEF30E00E94DDDAA70196018C
:108E70000E94AFDAB22E2FEF30E0D8010E94DDDA87
:108E8000A70196010E94AFDAE22F20E04B2D60E0AF
:108E90008E2F0E941C8A0BC08E0109521C4FF801B4
:108EA0008081882321F00E946D8AF8011082FE01E2
:108EB000E152FC4F8081882309F458C07E01FDE116
:108EC000EF1AFCEFFF0ACE018E519C4FDE01AF512D
:108ED000BC4FBE0160527C4FF7010081FC01208134
:108EE0004C91FB016081CE010E94CF45F701808348
:108EF0003DC0C7010E94ADA4FE01E852FC4F208195
:108F00003181280F391F31832083C7010E9463A458
:108F1000FE01E652FC4F20813181280F391F318339
:108F200020830A511F4F44CFC7010E94ADA4FE0108
:108F3000E852FC4F20813181280F391F3183208373
:108F4000C7010E9463A4FE01E652FC4F20813181DB
:108F5000280F391F3183208302591F4F3ACFFE015A
:108F6000E952FC4F8081811163CF60CFDF91CF91B7
:108F70001F910F91FF90EF90DF90CF90BF900895D9
:108F800040E052ED69E47BE643960C94D4D4FC01B6
:108F9000EC51FC4F408151816281738182960C9427
:108FA000D4D4CF93DF93EC01A296CE010E9427D5B3
:108FB000CE01DF91CF910C9424D51F920F920FB662
:108FC0000F9211240BB60F922F933F934F935F9301
:108FD0006F937F938F939F93AF93BF93EF93FF9381
:108FE00089EC98E00E94BC44FF91EF91BF91AF9152
:108FF0009F918F917F916F915F914F913F912F91B1
:109000000F900BBE0F900FBE0F901F9018950F93EF
:109010001F93CF93DF9300D000D000D0CDB7DEB741
:109020008B016115710589F41092C3081092C20872
:1090300047E069E97AE1CE0101960E941DD360E024
:10904000CE0101960E946CD30CC08091C60890E0BE
:109050008617970731F082E090E09093C3088093E1
:10906000C2080093C60826960FB6F894DEBF0FBE5E
:10907000CDBFDF91CF911F910F910895CF93DF93D3
:1090800000D000D000D0CDB7DEB741155105E9F4CE
:109090001092C1081092C00842E067E97AE1CE015F
:1090A00001960E941DD361E0CE0101960E946CD30F
:1090B00042E067E97AE1CE0101960E941DD361E0AA
:1090C000CE0101960E946CD310C06115710519F490
:1090D0000E948F420AC06093C5084093C40881E093
:1090E00090E09093C1088093C00826960FB6F8943C
:1090F000DEBF0FBECDBFDF91CF910895DF92EF921B
:10910000FF920F931F93CF93DF93EC01FC01E35980
:10911000FF4F8081811102C0D12C1CC08E01065FDF
:109120001D4FC8010E9425A77E0124E0E20EF11C1C
:10913000C7010E94F8D4882379F3C8010E9412A9BC
:10914000C8010E942AA7AB01BC01C7010E94D4D468
:10915000DD24D394FE01E153FC4F8081882341F04C
:109160008E0105541E4FC8010E94F8D4811157C1C9
:109170007E018FE2E81A8CEFF80AF70180818823DC
:1091800049F18E01065F1D4FC8010E94C0AA8823C5
:1091900009F140E050E060E070E0CE010E943E48FE
:1091A0000E946D8AF70110827E01FEE2EF1AFCEF49
:1091B000FF0AF7016081C8010E94D3A881E0F7018E
:1091C0008083FE01ED52FC4F808181110E94D93DC8
:1091D0001092C7088E010E5D1F4FC8010E94F8D47F
:1091E000882321F080919F0C83FD26C1C8010E9435
:1091F000F8D4882339F0FE01E053FC4F80818111BF
:109200005BC007C0CE0143960E94F8D48111F3CF12
:1092100053C00E94A63B029709F44EC00E94A63B91
:10922000019709F00DC148C0CE018B5E9E4F0E9490
:1092300063A41816190674F4FE01EC51FC4F8081EA
:109240009181A281B38180349244AF40B10509F08D
:109250000AC109C0CE018B5A9C4F0E9463A4181604
:10926000190654F30AC0CE0143960E9459D56115E0
:10927000724D89449B4608F0F6C060E070E0C7017B
:109280000E948DA360E070E0CE018B5E9E4F0E9435
:109290008DA360E070E0CE018B5A9C4F0E948DA39D
:1092A000CE0143960E9427D5C8010E94F8D4882396
:1092B00019F0CE010E94D147FE01E053FC4F80819E
:1092C000882309F474C08091C708811170C00E947E
:1092D000574E81116CC0D8C068EE74E002C069E3DB
:1092E00075E0CE01865F9D4F0E94F7A738C06AE8FF
:1092F00075E0F7CF6BED75E0F4CF21E040E06CE274
:1093000076E0CE010E943D458E010A581F4FC801EC
:109310000E9471A6882329F060E070E0C8010E94D5
:109320008DA38E010B5E1E4FC8010E9471A688237B
:1093300029F060E070E0C8010E948DA38E010B5AF5
:109340001C4FC8010E9471A6882329F060E070E0DC
:10935000C8010E948DA3C053DC4F1882C4C060E0D6
:1093600070E0CE018A589F4F0E948DA360E070E0AC
:10937000CE018B5E9E4F0E948DA360E070E0CE0117
:109380008B5A9C4F0E948DA380E00E946A4E0E94DF
:10939000BC8B0E9473380E94BE240E94C18310E0DF
:1093A00060E0812F0E94BF821F5F1530C9F78E01D8
:1093B0000F5C1F4FC8010E94F8D4882309F493C0A2
:1093C000D11091C089C040E950ED63E070E0C80160
:1093D0000E94D4D4FE01E759FF4F8081882321F0F9
:1093E000813009F080C00FC0CE0182599F4F0E948A
:1093F0009889CE01DF91CF911F910F91FF90EF904F
:10940000DF900C946746CE01835F9E4FDF91CF9132
:109410001F910F91FF90EF90DF900C949889CE01EF
:109420008B5A9C4F0E944CA540E251EA67E070E0E5
:10943000C8010E94D4D49CCECE010E94D147D6CE82
:10944000FE01EA52FC4F80818E7F806480837E0122
:1094500086E7E80EF11CC7010E9463A418161906DE
:109460000CF4EACEE1CE6FEB74E0CE01865F9D4F47
:109470000E94F7A7CE010E94214521E04FEF60E056
:1094800080E00E941C8AF9CE81E08093C7088AE0C0
:109490008093C5088093C40881E090E09093C10850
:1094A0008093C008FE01EC52FC4F8081918188308E
:1094B000910509F414CF44F48230910509F41DCFCD
:1094C000049709F04CCF08CF8031910509F40FCFF4
:1094D000809709F044CF0ECFCE01805C9F4F0E9451
:1094E000CA8C811170CFDF91CF911F910F91FF90A6
:1094F000EF90DF9008951F920F920FB60F921124F4
:109500000BB60F922F933F934F935F936F937F937D
:109510008F939F93AF93BF93EF93FF93CF93DF937B
:10952000CDB7DEB72697DEBFCDBF8091C908909139
:10953000CA08A091CB08B091CC088C599F4FAF4F6F
:10954000BF4F8093C9089093CA08A093CB08B093EB
:10955000CC080E94BA868091B908982F9F5F90939B
:10956000B908853A08F4C3C01092B9088091BE08C2
:109570009091BF081816190614F401973AC080910B
:10958000C2089091C30881309105F1F48091BC0824
:109590009091BD0801969093BD088093BC0882E02D
:1095A00090E09093C3088093C20882E190E090938A
:1095B000BF088093BE0847E069E97AE1CE010196D1
:1095C0000E941DD360E034C082309105B9F48091CF
:1095D000C60890E02091BC083091BD0828173907D3
:1095E0009CF083E090E09093C3088093C20880E5EC
:1095F00090E09093BF088093BE081EC00397E1F4EB
:109600001092BD081092BC0881E090E09093C308CE
:109610008093C20882E190E09093BF088093BE08D7
:1096200047E069E97AE1CE0101960E941DD361E02D
:10963000CE0101960E946CD38091BA089091BB082C
:109640001816190634F401979093BB088093BA0852
:109650004EC08091C0089091C1088130910509F5F4
:1096600082E090E09093C1088093C0088091C50883
:109670008093BA081092BB0842E067E97AE1CE0114
:1096800001960E941DD361E0CE0101960E946CD329
:1096900042E067E97AE1CE0101960E941DD361E0C4
:1096A00022C0029721F581E090E09093C108809359
:1096B000C0088091C4088093BA081092BB0842E0A9
:1096C00067E97AE1CE0101960E941DD360E0CE01E8
:1096D00001960E946CD342E067E97AE1CE010196DF
:1096E0000E941DD360E0CE0101960E946CD32696A5
:1096F0000FB6F894DEBF0FBECDBFDF91CF91FF91C3
:10970000EF91BF91AF919F918F917F916F915F91F9
:109710004F913F912F910F900BBE0F900FBE0F9066
:109720001F90189581539C4FFC01608308950F93FF
:109730001F93CF93DF9300D000D000D0CDB7DEB71A
:10974000062F1FB7F89445E06FE87AE1CE01019645
:109750000E941DD361E0CE0101960E944CD345E0EA
:109760006FE87AE1CE0101960E941DD3602FCE01F1
:1097700001960E946CD31FBF26960FB6F894DEBFE9
:109780000FBECDBFDF91CF911F910F9108950F9321
:109790001F93CF93DF93EC01062FFC01EA52FC4F9D
:1097A00011E0108360E00E94974B0E94C335682F40
:1097B000CE018B5E9E4F0E9481A30E94B036682F1F
:1097C0006127CE018B5A9C4F0E9481A3CE010E943B
:1097D000C047011103C0CE010E94C7470E946D8A95
:1097E000FE01EF52FC4F1082FE01EE52FC4F81E071
:1097F0008083FE01E852FC4F11821082FE01E65286
:10980000FC4F11821082FE01E452FC4F1182108243
:10981000FE01E952FC4F1082FE01E152FC4F108222
:10982000FE01E052FC4F1082FE01EF51FC4F10820E
:10983000CE51DC4F1882DF91CF911F910F91089587
:10984000DF92EF92FF920F931F93CF93DF9300D09D
:1098500000D000D0CDB7DEB78C01D62E60E070E02E
:109860000E94074860E082E090E00E9466A0809538
:10987000881F8827881F0E94867E61E080E09DE126
:109880000E94D1D584E09DE10E9425D2F80110828A
:1098900011821282138260E084E492E00E9466A04A
:1098A000F801EC51FC4FA82FB0E020E037E843E985
:1098B00053E00E94E4DA605C7D4B804F9F4F6083F1
:1098C000718382839383F801E359FF4F808188235A
:1098D00009F45EC07801F6EFEF1AFDEFFF0AC70149
:1098E0000E9447A842E067E97AE1CE0101960E9412
:1098F0001DD361E0CE0101960E944CD342E067E99E
:109900007AE1CE0101960E941DD361E0CE0101965D
:109910000E944CD342E067E97AE1CE0101960E94B1
:109920001DD361E0CE0101960E946CD342E067E94D
:109930007AE1CE0101960E941DD361E0CE0101962D
:109940000E946CD360E086E591E00E9466A08111E0
:1099500003C065E070E002C064E070E0C7010E94EF
:10996000B3A7DD2049F02FEF8BE792E9215080402B
:109970009040E1F700C00000C7010E94AEA6C701F9
:109980000E942AA7AB01BC01C80104960E94D4D44E
:1099900040E050E060E070E0C8010E943E48DD20F9
:1099A00071F00E94758B83E00E946A4EF801E053CB
:1099B000FC4F1082F801EC52FC4F118210826D2D89
:1099C000C8010E94C74BF801E359FF4F80818823EB
:1099D00041F060E086E591E00E9466A081110E945E
:1099E000BAA626960FB6F894DEBF0FBECDBFDF91A4
:1099F000CF911F910F91FF90EF90DF90089540E07D
:109A000065E87AE181EB9CE00E941DD389EC98E047
:109A10000C94BB42CF93DF9300D000D000D0CDB7E1
:109A2000DEB761E08AE491E00E9466A091E08111D6
:109A300001C090E09093110D1092BA0C1092B90CE5
:109A40001092BC0C1092BB0C1092BF0C1092C00C68
:109A500082E19DE00E9427D51092210D43E06DE840
:109A60007AE1CE0101960E941DD361E0CE010196FC
:109A70000E944CD343E06DE87AE1CE0101960E944A
:109A80001DD360E0CE0101960E946CD326960FB6DE
:109A9000F894DEBF0FBECDBFDF91CF910895109235
:109AA000A0001092A1001092A9001092A80010929C
:109AB000AB001092AA001092A5001092A400109280
:109AC00072000895CF92DF92EF92FF92CF93809130
:109AD000B90C9091BA0C892B39F482E19DE00E9477
:109AE00027D51092210D4BC021E02093210D8091AC
:109AF000B90C9091BA0C892B31F42093C00CC12C75
:109B0000D12C76012EC08091BB0C9091BC0C209181
:109B1000B70C3091B80CB9010E9465DA880F991F13
:109B2000880F991FE091BD0CF091BE0CE80FF91F52
:109B30008091BB0C9091BC0C0196B9010E9465DA32
:109B40009093BC0C8093BB0C8091B90C9091BA0C93
:109B500001979093BA0C8093B90CC080D180E280B9
:109B6000F3809701A8EEB3E00E94D1DAAB01BC010B
:109B700082E19DE00E94D4D4C114D10439F4CF9184
:109B8000FF90EF90DF90CF900C944F4DA60160E0D6
:109B900070E0443F81E058076105710518F0C2E0AC
:109BA00083E002C0C3E086E09A01AB01220F331FBD
:109BB000441F551F04C0220F331F441F551F8A9591
:109BC000D2F760E074E284EF90E00E948DDA2150D9
:109BD000310980E48093A000C860C093A100309355
:109BE000A9002093A8001092AB001092AA00109236
:109BF000A5001092A40010927200CF91FF90EF90F8
:109C0000DF90CF9008950F931F93CF93DF938C0134
:109C1000D62FC72F8091110D882309F443C060917E
:109C2000B70C7091B80C4091B90C5091BA0C6417F4
:109C3000750771F14091B90C5091BA0C461757074E
:109C400020F54091B90C5091BA0C8091BB0C9091C9
:109C5000BC0C840F951F0E9465DA880F991F880F2E
:109C6000991FE091BD0CF091BE0CE80FF91F008325
:109C70001183D283C3838091B90C9091BA0C019661
:109C80009093BA0C8093B90C03C081E08093BF0C11
:109C90008091210D811106C0DF91CF911F910F910D
:109CA0000C94624DDF91CF911F910F910895809197
:109CB000210D08958091110D882359F08091210D77
:109CC000882339F082E19DE00E94F8D481110C9440
:109CD000624D0895FF920F931F93CF93DF938830C7
:109CE00028F5E82FF0E0EE0FFF1FE55BFC4F008149
:109CF000118101151105D1F0F12C24E0F29EC00173
:109D00001124F801E80FF91F25913491FC013296D6
:109D1000E00FF11FC591D491209721F0BE01C90138
:109D20000E94034EF394CD2B41F70BC064EF71E01A
:109D30008BE790E0DF91CF911F910F91FF900C94F2
:109D4000034EDF91CF911F910F91FF90089540E056
:109D500065E87AE182E29DE00E941DD384E190E013
:109D60009093B80C8093B70C1092BA0C1092B90C67
:109D70001092BC0C1092BB0C81EC9CE09093BE0C3A
:109D80008093BD0C1092BF0C1092C00C82E19DE03C
:109D90000C94D0D408958F929F92AF92BF92CF929D
:109DA000DF92EF92FF920F931F93CF93DF93CDB784
:109DB000DEB7FC0140835183628373830483158380
:109DC00026833783C086D186E286F386848695868D
:109DD000A686B7864F85588969897A89408B518BC9
:109DE000628B738BDF91CF911F910F91FF90EF905A
:109DF000DF90CF90BF90AF909F908F900895660FA7
:109E0000771F660F771F680F791FCB010895660FC4
:109E1000771F660F771F680F791FCB0108950F9387
:109E200000E02DE93DE944ED5CE966EC7BE981E287
:109E30009BE90E94729990933C0D80933B0D892B76
:109E400079F40FEF2DE93DE944ED5CE966EC7BE93F
:109E500081E29BE90E94729990933C0D80933B0DA7
:109E600081E020913B0D30913C0D232B09F480E0E3
:109E70000F91089580913B0D90913C0D0E94ED92C1
:109E800090933A0D8093390D21E0892B09F420E05D
:109E9000822F0895CF93DF93CDB7DEB7AB970FB680
:109EA000F894DEBF0FBECDBFAE014F5F5F4F6BE5D5
:109EB00073E08091390D90913A0D0E94ED97BE01AB
:109EC0006F5F7F4F8091390D90913A0D0E94E69619
:109ED0009093380D8093370D21E0892B09F420E011
:109EE000822FAB960FB6F894DEBF0FBECDBFDF91C9
:109EF000CF9108958091390D90913A0D0E944B9920
:109F00006095709580959095662797FD6395772766
:109F100088279927862F0895BF92CF92DF92EF92DC
:109F2000FF920F931F93CF93DF93CDB7DEB7AB971D
:109F30000FB6F894DEBF0FBECDBF8C016A0135E0CD
:109F4000B32EE62EF12C81E0E81AF108BE016F5F16
:109F50007F4F8091370D9091380D0E942D97F80119
:109F60008823E1F0DE01119620E030E02E153F0558
:109F700044F0F801E20FF31F10822115310559F06A
:109F800004C08D9181110CC0F4CFC114D10461F0D3
:109F9000F601208309C0BA94C9F606C0108204C035
:109FA00081932F5F3F4FE2CF80E090E0AB960FB6FA
:109FB000F894DEBF0FBECDBFDF91CF911F910F91FF
:109FC000FF90EF90DF90CF90BF9008950F931F9375
:109FD000CF93DF938C01EB010EC0B801CE010E943C
:109FE000B3DC009741F48091370D9091380D0E94B9
:109FF000209781E009C0BE018091370D9091380D06
:10A000000E942D978111E9CFDF91CF911F910F9180
:10A0100008950F931F93CF93DF93CDB7DEB7AB9720
:10A020000FB6F894DEBF0FBECDBF8B01BE016F5FD0
:10A030007F4F0E94E64F882371F0BE016F5F7F4F14
:10A040008091390D90913A0D0E946894F8019183A6
:10A05000808381E001C080E0AB960FB6F894DEBF4C
:10A060000FBECDBFDF91CF911F910F9108956091E9
:10A07000310D7091320D8091330D9091340D089512
:10A08000CF93DF93CDB7DEB7AB970FB6F894DEBFB3
:10A090000FBECDBFBE016F5F7F4F0E94E64F88238A
:10A0A00059F0BE016F5F7F4F8091390D90913A0D4D
:10A0B0000E94CF9881E001C080E0AB960FB6F89483
:10A0C000DEBF0FBECDBFDF91CF910895CF93DF9359
:10A0D000CDB7DEB7AB970FB6F894DEBF0FBECDBFDE
:10A0E000AE014F5F5F4FBC018091370D9091380DED
:10A0F0000E94799891E0811101C090E0892FAB9680
:10A100000FB6F894DEBF0FBECDBFDF91CF9108959B
:10A1100080912F0D08958091300D0895CF93DF9396
:10A12000EC018091350D9091360D0097E1F048815A
:10A13000BE016E5F7F4F50E00E94B79528818091ED
:10A140002B0D90912C0DA0912D0DB0912E0D820F05
:10A15000911DA11DB11D80932B0D90932C0DA093EB
:10A160002D0DB0932E0DDF91CF9108958091300D7C
:10A17000882381F08091350D9091360D009721F064
:10A180000E949C940E94B99A1092360D1092350D3F
:10A190001092300D60912B0D70912C0D80912D0D32
:10A1A00090912E0D08950E94819A882391F041E0AC
:10A1B00050E06AE27DE08091350D9091360D0E946D
:10A1C000B09421E0181619060CF020E02093290D18
:10A1D000089521E041E069EF77E089EC98E00E9482
:10A1E0003D451092290D1092280D08958091290D5A
:10A1F0000895CF93DF931F92CDB7DEB780912A0DDC
:10A2000089830E94D35089810F90DF91CF91089567
:10A2100010922F0D8091350D9091360D009721F001
:10A220000E949C940E94B99A1092360D1092350D9E
:10A23000089580912F0D81110E9408518091300D59
:10A2400081110E94B6508091370D9091380D009782
:10A2500031F00E941A971092380D1092370D8091AC
:10A26000390D90913A0D009731F00E94629410924E
:10A270003A0D1092390D80913B0D90913C0D009755
:10A2800031F00E94129A10923C0D10923B0D1092E8
:10A29000310D1092320D1092330D1092340D08953D
:10A2A0000E94269C81110EC00E94819A811105C0D6
:10A2B0000E94195121E030E032C00E94195122E081
:10A2C00030E02DC00E940F4F811105C00E9419512E
:10A2D00023E030E024C00E943A4F811105C00E9463
:10A2E000195124E030E01BC00E944A4F811105C083
:10A2F0000E94195125E030E012C00E947A4F81116E
:10A3000005C00E9419512AE030E009C00E949E9ABF
:10A31000882319F026E030E002C020E030E0C901D7
:10A320000895CF93DF93EC010E9419510E94505180
:10A330009C01009719F08630910569F510922B0D5C
:10A3400010922C0D10922D0D10922E0D1092360D94
:10A350001092350D65E37DE0CE010E9409508823FF
:10A3600031F08091350D9091360D009719F427E06A
:10A3700030E011C00E9445996093310D7093320D09
:10A380008093330D9093340D81E080932F0D0E94C4
:10A39000D35020E030E0C901DF91CF9108950F93B1
:10A3A0001F93CF93DF938C010E9419510E9450514B
:10A3B000EC01009769F510922B0D10922C0D109264
:10A3C0002D0D10922E0D1092360D1092350DC801E4
:10A3D0000E944050C8010E946650882389F065E3BE
:10A3E0007DE0C8010E940950882369F08091350DF5
:10A3F0009091360D892B51F081E08093300D08C08B
:10A40000C7E0D0E005C0C3E0D0E002C0C8E0D0E0C3
:10A41000CE01DF91CF911F910F9108950E941951A4
:10A420000E9450519C01009719F08630910541F42B
:10A430008091370D9091380D0E94209720E030E0F8
:10A44000C901089540E065E87AE18DE39DE00C9450
:10A450001DD3CF92DF92EF92FF920F931F93CF9372
:10A46000DF9300D000D000D0CDB7DEB78C017C01E7
:10A470006C018EE1C80ED11CC7010E940FD3E6E02B
:10A48000EE0EF11CEC14FD04B9F746E06BE97AE13D
:10A49000C8014E960E941DD385E0F80184A345E0D3
:10A4A00065E97AE1CE0101960E941DD386E0FE01A6
:10A4B0003196D80101900D928A95E1F746E067E860
:10A4C0007AE1CE0101960E941DD386E0FE0131960D
:10A4D000D801169601900D928A95E1F743E067E85E
:10A4E0007AE1CE0101960E941DD386E0FE013196ED
:10A4F000D8011C9601900D928A95E1F744E06BE932
:10A500007AE1CE0101960E941DD386E0FE013196CC
:10A51000D801529601900D928A95E1F747E06BE8D9
:10A520007AE1CE0101960E941DD386E0FE013196AC
:10A53000D801589601900D928A95E1F726960FB6AC
:10A54000F894DEBF0FBECDBFDF91CF911F910F9169
:10A55000FF90EF90DF90CF900895EF92FF920F93CE
:10A560001F93CF93DF93EC01F12C86E0E82E0EC011
:10A570008E01EF9C000D111D112461E0C8010E94A5
:10A580004CD361E0C8010E946CD3F3948CA1F816FF
:10A5900078F36E9661E0CE010E944CD361E0CE016B
:10A5A000DF91CF911F910F91FF90EF900C946CD39E
:10A5B0000F931F93CF93DF93EC0185E18A95F1F719
:10A5C000000061E0CE014E960E946CD385E18A9531
:10A5D000F1F7000010E006E009C061E0CE01019F44
:10A5E000800D911D11240E946CD31F5F8CA1181740
:10A5F000A0F385E18A95F1F70000DF91CF911F91DB
:10A600000F910895CF92DF92EF92FF920F931F93D5
:10A61000CF93DF93C62EEA0128E0E22EF12C30E83A
:10A62000D32E8C01025E1F4F9D2D9C2161E009F409
:10A6300060E0CE010E946CD361E0C8010E946CD33F
:10A6400085E18A95F1F7000060E0C8010E946CD3B3
:10A65000D69481E0E81AF10839F761E0CE010E9452
:10A660006CD360E0CE010E944CD361E0C8010E942F
:10A670006CD3CE010E945FD3F82E60E0C8010E9427
:10A680006CD361E0CE010E944CD381E08F25DF9135
:10A69000CF911F910F91FF90EF90DF90CF90089591
:10A6A000DF92EF92FF920F931F93CF93DF93EC0112
:10A6B000E62E8A01F12C46E0D42E09C060E0CE01DE
:10A6C000DF9C800D911D11240E946CD3F3948CA10A
:10A6D000F816A0F385E18A95F1F7000060E0CE015D
:10A6E0004E960E946CD3A8016E2DCE01DF91CF91C2
:10A6F0001F910F91FF90EF90DF900C94025340E078
:10A7000065E87AE188E69DE00E941DD383E49DE040
:10A710000C9429524F925F926F927F928F929F92E8
:10A72000AF92BF92CF92DF92EF92FF920F931F935F
:10A73000CF93DF938091800D9091810D892B09F04B
:10A7400021C49091AA0D8091A90D981771F0C09124
:10A75000A90D17E7C19FE0011124C555D24FFE0195
:10A76000EC58FF4F81E0808302C0C0E0D0E0D0937E
:10A77000810DC093800D209709F4B4C3888D998D05
:10A78000AA8DBB8D80930E1690930F16A093101672
:10A79000B09311168C8D9D8DAE8DBF8D809312164A
:10A7A00090931316A0931416B093151688A199A12F
:10A7B000AAA1BBA18093161690931716A093181602
:10A7C000B09319168CA19DA1AEA1BFA180931A16BA
:10A7D00090931B16A0931C16B0931D1688A599A5DF
:10A7E000AAA5BBA580931E1690931F16A0932016B2
:10A7F000B09321168AAD8093820D8091830D8111D3
:10A8000011C01092860D1092870D1092880D109233
:10A81000890DFE01E25AFF4F208131813F3408F05B
:10A8200046C051C0BE01E4E8FDE04CE75DE020E039
:10A8300030E0DB011C96CD90DD90ED90FC901F97F1
:10A84000CD28CE28CF2839F18081882321F1D90164
:10A85000A658B24F8C91D901AA0FBB1F15E0E12E6B
:10A8600016E1F12EEA0EFB1ED701882341F08D91EF
:10A870009C91DA010D911C91801B910B07C08D9169
:10A880009C91DA010D911C91800F911FD7011196B7
:10A890009C938E9310822F5F3F4F6C5F7F4F31965A
:10A8A0004E5F5F4F2230310509F4ABCFC2CF3D3947
:10A8B00030F403E0369527950A95E1F702C028E8C1
:10A8C00033E188E014C0383230F03695279536955C
:10A8D000279584E00CC0343120F03695279582E02E
:10A8E00006C02032310510F420E230E081E0809390
:10A8F0008A0D205231092115B8E03B07D8F0E32F2B
:10A90000FF27EE0FFF1FEE0FFF1FE35FF74F85914D
:10A910009591A591B491AC01BD01AA27279FC001D3
:10A92000269F810D9A1F06948A1F9A1F1124481B87
:10A93000590B1BC0F901F695E795EC7FE35FF34FE8
:10A940004591559165917491DB01277033272A9FBA
:10A95000B0012B9F700D3A9F700D1124E3E07695A6
:10A960006795EA95E1F7461B570B50938C0D409382
:10A970008B0D80918A0D80938D0DFE01EE58FF4F57
:10A980008081882309F474C0CA59DF4F8881998176
:10A9900090938F0D80938E0D9F3460F09D3930F42D
:10A9A00043E0969587954A95E1F702C088E893E1E0
:10A9B00028E014C0983230F0969587959695879543
:10A9C00024E00CC0943120F09695879522E006C0D3
:10A9D0008032910510F480E290E021E020938A0D0E
:10A9E0009C01205231092115C8E03C07D8F0E32F23
:10A9F000FF27EE0FFF1FEE0FFF1FE35FF74F85915D
:10AA00009591A591B491AC01BD01AA27279FC001E2
:10AA1000269F810D9A1F06948A1F9A1F1124481B96
:10AA2000590B1BC0F901F695E795EC7FE35FF34FF7
:10AA30004591559165917491DB01277033272A9FC9
:10AA4000B0012B9F700D3A9F700D112403E0769595
:10AA500067950A95E1F7461B570BCA01A0E0B0E0E5
:10AA60008093900D9093910DA093920DB093930DC0
:10AA70005093290140932801E091800DF091810DC0
:10AA800020AD2093940DEA58FF4F30818091051638
:10AA900090910616892B09F03360809107169091EA
:10AAA0000816892B09F034608091031638131CC0F6
:10AAB000E091800DF091810D40815181628173811F
:10AAC000F48805891689D789DF01AB58BF4F3C91BF
:10AAD00081E0411551056105710509F480E080931D
:10AAE0003E16811144C087C0A5E1B2E0E9E1F2E081
:10AAF00080E090E041E050E0BA01082E01C0660F0E
:10AB00000A94EAF7D62FC0910316C327C62341F152
:10AB1000D32370910316DD2391F0762B70930316E7
:10AB2000CD91DC9111971881BA01008002C0660FA7
:10AB3000771F0A94E2F760956123688311C06095DE
:10AB4000672360930316CD91DC9111971881BA01A8
:10AB5000008002C0660F771F0A94E2F7162B188355
:10AB600001969396B3968530910531F6A1CFC22F09
:10AB7000C1708F2D902FA12FBD2F6C017D01F594F9
:10AB8000E794D794C794F094E094D094C094C11CF7
:10AB9000D11CE11CF11CC0923F16D0924016E092ED
:10ABA0004116F0924216D1E03111D0E0D093361622
:10ABB0008093371690933816A0933916B0933A16AF
:10ABC00040934716509348166093491670934A165F
:10ABD000CC2311F08FEF01C081E080933C1681E01F
:10ABE0008C2780933D1610924316109244161092B3
:10ABF0004516109246164481558166817781F48806
:10AC000005891689D78981E04115510561057105CE
:10AC100009F480E080936716882309F446C021FB7D
:10AC2000CC27C0F98F2D902FA12FBD2F6C017D0156
:10AC3000F594E794D794C794F094E094D094C0949A
:10AC4000C11CD11CE11CF11CC0926816D09269167F
:10AC5000E0926A16F0926B16D1E0313009F0D0E044
:10AC6000D0935F168093601690936116A09362163E
:10AC7000B0936316409370165093711660937216DA
:10AC800070937316CC2311F08FEF01C081E0809395
:10AC9000651681E08C278093661610926C161092D0
:10ACA0006D1610926E1610926F1640855185628552
:10ACB0007385F48805891689D78981E04115510586
:10ACC0006105710509F480E080939016882309F4EA
:10ACD00046C022FBCC27C0F98F2D902FA12FBD2F6E
:10ACE0006C017D01F594E794D794C794F094E094B7
:10ACF000D094C094C11CD11CE11CF11CC0929116CF
:10AD0000D0929216E0929316F0929416D1E03230DF
:10AD100009F0D0E0D09388168093891690938A1614
:10AD2000A0938B16B0938C164093991650939A1655
:10AD300060939B1670939C16CC2311F08FEF01C08B
:10AD400081E080938E1681E08C2780938F1610927D
:10AD50009516109296161092971610929816448592
:10AD6000558566857785F48805891689D78981E0B8
:10AD7000411551056105710509F480E08093B9160C
:10AD8000882309F446C023FBCC27C0F98F2D902FD0
:10AD9000A12FBD2F6C017D01F594E794D794C79442
:10ADA000F094E094D094C094C11CD11CE11CF11C1F
:10ADB000C092BA16D092BB16E092BC16F092BD16A5
:10ADC000D1E0333009F0D0E0D093B1168093B216C1
:10ADD0009093B316A093B416B093B5164093C216D1
:10ADE0005093C3166093C4167093C516CC2311F00C
:10ADF0008FEF01C081E08093B71681E08C278093AC
:10AE0000B8161092BE161092BF161092C01610926D
:10AE1000C11640895189628973891489D589C68987
:10AE20003789EB58FF4FF08181E0411551056105ED
:10AE3000710509F480E08093E216882309F445C087
:10AE400024FBEE27E0F9812F9D2FAC2FB32F8C012F
:10AE50009D01359527951795079530952095109567
:10AE600001951F4F2F4F3F4F0093E3161093E416A9
:10AE70002093E5163093E61621E0F43009F020E047
:10AE80002093DA168093DB169093DC16A093DD16E0
:10AE9000B093DE164093EB165093EC166093ED16CC
:10AEA0007093EE16EE2311F08FEF01C081E08093D6
:10AEB000E01681E08E278093E1161092E71610923B
:10AEC000E8161092E9161092EA161092960D10925A
:10AED000950D10926E0D10926F0D1092700D1092D4
:10AEE000710D50C080ED97E0909329018093280167
:10AEF0008091051690910616892B09F043C0809128
:10AF0000071690910816892B11F40C9470633AC0BF
:10AF1000A901082E01C0440F0A94EAF7C42F6091DA
:10AF200003166727642341F1C72350910316CC23EE
:10AF300091F0542B50930316CD91DC9111976881B9
:10AF4000A901008002C0440F551F0A94E2F7409502
:10AF50004623488311C04095452340930316CD9165
:10AF6000DC9111976881A901008002C0440F551F30
:10AF70000A94E2F7642B688301969396B396853022
:10AF8000910531F68091830D811108C08091800D6B
:10AF90009091810D892B09F04BC047C04091800DE5
:10AFA0005091810DE4E8FDE0ACE7BDE080E090E089
:10AFB000FF24F394BA016A587F4F4115510569F097
:10AFC000EB01288130E0EC0123960C2E02C0359570
:10AFD00027950A94E2F720FD20C0208121111DC091
:10AFE000EC01C658D24F2881EC01CC0FDD1FCB5F9E
:10AFF000D94E222341F0288139810D911C9111975E
:10B00000200F311F07C0288139810D911C911197A4
:10B01000201B310B39832883F082019631961296DA
:10B020008230910509F4B2CFC8CF80E00C94E96377
:10B03000E0918A0D4091950D5091960DC090970D1D
:10B04000D090980DE090990DF0909A0DF094E094C6
:10B05000D094C094C11CD11CE11CF11CCD2CDE2C61
:10B06000EF2CFF24E7FCFA9470E021E030E061E08F
:10B070005EC5C091800DD091810DDE01AE58BF4FED
:10B080008C91811105C080913E16811177C05EC1FF
:10B0900041155105E9F042305105A1F58EAD9FAD46
:10B0A000919581959109AA2797FDA095BA2F809037
:10B0B000BA169090BB16A090BC16B090BD16880D25
:10B0C000991DAA1DBB1D8C0D9D1DAE1DBF1D12C05F
:10B0D0008CAC9DACAA2497FCA094BA2C8091BA1693
:10B0E0009091BB16A091BC16B091BD16880D991D0C
:10B0F000AA1DBB1D8093BA169093BB16A093BC16D5
:10B10000B093BD164115510599F48CAC9DACAA24A1
:10B1100097FCA094BA2C8091E3169091E416A0912C
:10B12000E516B091E616880D991DAA1DBB1D1DC020
:10B130004230510509F0A7CF8EAD9FAD9195819515
:10B140009109AA2797FDA095BA2F8090E3169090B9
:10B15000E416A090E516B090E616880D991DAA1D7C
:10B16000BB1D8C0D9D1DAE1DBF1D8093E3169093DE
:10B17000E416A093E516B093E61685CF80904716A7
:10B1800090904816A0904916B0904A1680913F16AC
:10B1900090914016A0914116B0914216880D991DCC
:10B1A000AA1DBB1D80933F1690934016A093411695
:10B1B000B0934216181619061A061B060CF0C6C0E4
:10B1C0004090431650904416609045167090461675
:10B1D000481459046A047B040CF0B8C080903716F8
:10B1E00090903816A0903916B0903A16881999099F
:10B1F000AA09BB0980933F1690934016A09341166D
:10B20000B093421680913B16882379F08091FF1508
:10B2100090910016F0913C168F0F911DF7FD9A95B5
:10B22000909300168093FF1563C090913D16809116
:10B23000231681119627A0910E02B0910F028091E2
:10B240001202FC91E90102C0CC0FDD1F8A95E2F7E2
:10B25000992319F0FC2BFC9304C0CE0180958F2319
:10B260008C9380913D168823B1F0809123029091B8
:10B270002402892B11F40C948263A0912502B091D1
:10B2800026028C9190E00090270202C09595879548
:10B290000A94E2F715C080911C0290911D02892B3F
:10B2A00011F40C948263A0911E02B0911F028C9144
:10B2B00090E00090200202C0959587950A94E2F7ED
:10B2C00081709091221689130C9493630C9482637D
:10B2D000A0910702B0910802FC91C90100900B02F5
:10B2E00002C0880F991F0A94E2F780958F238C93F0
:10B2F00080910E1690910F16A0911016B091111614
:10B3000080903C16992487FC9094A92CB92C880D28
:10B31000991DAA1DBB1D80930E1690930F16A09326
:10B320001016B09311168091431690914416A09177
:10B330004516B09146160196A11DB11D8093431686
:10B3400090934416A0934516B093461680916716C5
:10B35000882309F4E8C08090701690907116A09030
:10B360007216B09073168091681690916916A0912C
:10B370006A16B0916B16880D991DAA1DBB1D80938E
:10B38000681690936916A0936A16B0936B161816F8
:10B3900019061A061B060CF0C6C040906C16509099
:10B3A0006D1660906E1670906F16481459046A04FA
:10B3B0007B040CF0B8C08090601690906116A0904D
:10B3C0006216B090631688199909AA09BB0980937F
:10B3D000681690936916A0936A16B0936B168091C5
:10B3E0006416882379F08091011690910216F091ED
:10B3F00065168F0F911DF7FD9A9590930216809315
:10B40000011663C09091661680914C1681119627A3
:10B41000A0913102B091320280913502FC91E90194
:10B4200002C0CC0FDD1F8A95E2F7992319F0FC2B9F
:10B43000FC9304C0CE0180958F238C938091661677
:10B440008823B1F08091460290914702892B11F434
:10B450000C949763A0914802B09149028C9190E0BE
:10B4600000904A0202C0959587950A94E2F715C0AC
:10B4700080913F0290914002892B11F40C949763C4
:10B48000A0914102B09142028C9190E00090430261
:10B4900002C0959587950A94E2F7817090914B16BA
:10B4A00089130C94A8630C949763A0912A02B0911D
:10B4B0002B02FC91C90100902E0202C0880F991F37
:10B4C0000A94E2F780958F238C93809112169091C5
:10B4D0001316A0911416B091151680906516992434
:10B4E00087FC9094A92CB92C880D991DAA1DBB1D11
:10B4F0008093121690931316A0931416B0931516FA
:10B5000080916C1690916D16A0916E16B0916F1689
:10B510000196A11DB11D80936C1690936D16A0939A
:10B520006E16B0936F1680919016882309F4E8C0C8
:10B530008090991690909A16A0909B16B0909C16A9
:10B540008091911690919216A0919316B0919416B5
:10B55000880D991DAA1DBB1D80939116909392167C
:10B56000A0939316B0939416181619061A061B0684
:10B570000CF0C6C0409095165090961660909716A5
:10B5800070909816481459046A047B040CF0B8C0F3
:10B590008090891690908A16A0908B16B0908C1689
:10B5A00088199909AA09BB0980939116909392165C
:10B5B000A0939316B093941680918D16882379F0FA
:10B5C0008091031690910416F0918E168F0F911DA5
:10B5D000F7FD9A95909304168093031663C090919B
:10B5E0008F168091751681119627A0915402B09103
:10B5F000550280915802FC91E90102C0CC0FDD1F79
:10B600008A95E2F7992319F0FC2BFC9304C0CE0134
:10B6100080958F238C9380918F168823B1F0809131
:10B62000690290916A02892B11F40C94AC63A09189
:10B630006B02B0916C028C9190E000906D0202C0A0
:10B64000959587950A94E2F715C0809162029091D2
:10B650006302892B11F40C94AC63A0916402B09145
:10B6600065028C9190E00090660202C095958795E6
:10B670000A94E2F781709091741689130C94BD635B
:10B680000C94AC63A0914D02B0914E02FC91C901A3
:10B690000090510202C0880F991F0A94E2F780952A
:10B6A0008F238C938091161690911716A0911816DF
:10B6B000B091191680908E16992487FC9094A92C2D
:10B6C000B92C880D991DAA1DBB1D80931616909349
:10B6D0001716A0931816B09319168091951690918D
:10B6E0009616A0919716B09198160196A11DB11DBE
:10B6F0008093951690939616A0939716B0939816EC
:10B700008091B916882309F4E8C08090C216909001
:10B71000C316A090C416B090C5168091BA16909129
:10B72000BB16A091BC16B091BD16880D991DAA1D1F
:10B73000BB1D8093BA169093BB16A093BC16B09312
:10B74000BD16181619061A061B060CF0C6C0409046
:10B75000BE165090BF166090C0167090C116481467
:10B7600059046A047B040CF0B8C08090B216909023
:10B77000B316A090B416B090B51688199909AA0905
:10B78000BB098093BA169093BB16A093BC16B093D6
:10B79000BD168091B616882379F080910516909198
:10B7A0000616F091B7168F0F911DF7FD9A9590939D
:10B7B00006168093051663C09091B81680919E1668
:10B7C00081119627A0917702B091780280917B0237
:10B7D000FC91E90102C0CC0FDD1F8A95E2F79923A5
:10B7E00019F0FC2BFC9304C0CE0180958F238C9321
:10B7F0008091B8168823B1F080918C0290918D02CF
:10B80000892B11F40C94C163A0918E02B0918F0228
:10B810008C9190E00090900202C0959587950A94D3
:10B82000E2F715C08091850290918602892B11F470
:10B830000C94C163A0918702B09188028C9190E032
:10B840000090890202C0959587950A94E2F781706D
:10B8500090919D1689130C94D2630C94C163A091AE
:10B860007002B0917102FC91C9010090740202C093
:10B87000880F991F0A94E2F780958F238C9380910B
:10B880001A1690911B16A0911C16B0911D1680904F
:10B89000B716992487FC9094A92CB92C880D991D72
:10B8A000AA1DBB1D80931A1690931B16A0931C16FD
:10B8B000B0931D168091BE169091BF16A091C01630
:10B8C000B091C1160196A11DB11D8093BE16909333
:10B8D000BF16A093C016B093C1168091E2168823BC
:10B8E00009F4E4C08090EB169090EC16A090ED1651
:10B8F000B090EE168091E3169091E416A091E516B3
:10B90000B091E616880D991DAA1DBB1D8093E31604
:10B910009093E416A093E516B093E6161816190650
:10B920001A061B060CF0C2C04090E7165090E816AD
:10B930006090E9167090EA16481459046A047B0472
:10B940000CF0B4C08090DB169090DC16A090DD1651
:10B95000B090DE1688199909AA09BB098093E316ED
:10B960009093E416A093E516B093E6168091DF1647
:10B97000882379F08091071690910816F091E016CF
:10B980008F0F911DF7FD9A959093081680930716D7
:10B990005FC09091E1168091C71681119627A09102
:10B9A0009A02B0919B0280919E02FC91E90102C033
:10B9B000CC0FDD1F8A95E2F7992319F0FC2BFC933D
:10B9C00004C0CE0180958F238C938091E11688234B
:10B9D000A9F08091AF029091B002892B09F4E9C6D9
:10B9E000A091B102B091B2028C9190E00090B302AC
:10B9F00002C0959587950A94E2F714C08091A80239
:10BA00009091A902892B09F4D4C6A091AA02B09101
:10BA1000AB028C9190E00090AC0202C095958795A6
:10BA20000A94E2F781709091C6168913BFC6C1C609
:10BA3000A0919302B0919402FC91C90100909702E9
:10BA400002C0880F991F0A94E2F780958F238C9388
:10BA500080911E1690911F16A0912016B09121166C
:10BA60008090E016992487FC9094A92CB92C880D1D
:10BA7000991DAA1DBB1D80931E1690931F16A0939F
:10BA80002016B09321168091E7169091E816A091A8
:10BA9000E916B091EA160196A11DB11D8093E71633
:10BAA0009093E816A093E916B093EA1680916E0D74
:10BAB00090916F0DA091700DB091710D0196A11D27
:10BAC000B11D80936E0D90936F0DA093700DB09388
:10BAD000710D80906E0D90906F0DA090700DB090D4
:10BAE000710DA091800DB091810D54968D919D9115
:10BAF0000D90BC91A02D88169906AA06BB06B0F041
:10BB000040916E0D50916F0D6091700D7091710D9F
:10BB1000E091800DF091810D84A595A5A6A5B7A50E
:10BB200084179507A607B70730F4BDC07F5F7E175F
:10BB30000CF49FCAE5CF0091900D1091910D2091CA
:10BB4000920D3091930D44A955A966A977A9AA270A
:10BB5000059FB12D169FC001269F900D259F800D3A
:10BB6000911D069FB00D811D9A1F159FB00D811D5F
:10BB70009A1F249FB00D811D9A1F149FB10D8A1F1B
:10BB80009A1FB6958A1F9A1F1124DF01AA59BF4F29
:10BB90004D915C91480F591F50938F0D40938E0D1E
:10BBA000E25AFF4F80819181A281B38160E070E011
:10BBB00084179507A607B70720F490938F0D8093FD
:10BBC0008E0D80918E0D90918F0D9F3460F09D3978
:10BBD00030F4D3E096958795DA95E1F702C088E8CE
:10BBE00093E148E014C0983230F096958795969589
:10BBF000879544E00CC0943120F09695879542E0FB
:10BC000006C08032910510F480E290E041E040935C
:10BC10008A0D80978115D8E09D07C8F0E92FFF278E
:10BC2000EE0FFF1FEE0FFF1FE35FF74FC590D5909C
:10BC3000E590F490A601B701AA27879FF001869F9F
:10BC4000E10DFA1F0694EA1FFA1F112419C0FC0126
:10BC5000F695E795EC7FE35FF34FC590D590E590BF
:10BC6000F490A601877099278E9DF0018F9DF00DAD
:10BC70009E9DF00D112463E0F695E7956A95E1F736
:10BC80004E1B5F0B5093290140932801040F151F91
:10BC9000211D311D0093900D1093910D2093920D55
:10BCA0003093930D2AC140916E0D50916F0D6091AC
:10BCB000700D7091710D80A991A9A2A9B3A92091CD
:10BCC000950D3091960D84179507A607B70708F0D4
:10BCD00000C1232B31F481E090E09093960D809386
:10BCE000950D8091950D9091960D019771F482E0DC
:10BCF00090E09093960D8093950D1092970D109271
:10BD0000980D1092990D10929A0DEF01C05CDF4FC3
:10BD10008091970D9091980DA091990DB0919A0DE9
:10BD2000488159816A817B81840F951FA61FB71FA7
:10BD30008093970D9093980DA093990DB0939A0DC1
:10BD40000091860D1091870D2091880D3091890DFD
:10BD500044A955A966A977A9AA27059FB12D169FC1
:10BD6000C001269F900D259F800D911D069FB00D4F
:10BD7000811D9A1F159FB00D811D9A1F249FB00D24
:10BD8000811D9A1F149FB10D8A1F9A1FB6958A1F95
:10BD90009A1F112490939C0D80939B0D40918E0DC2
:10BDA00050918F0D6091800D7091810D481759074A
:10BDB00030F4FB01E659FF4F8081918114C0481B8C
:10BDC000590B50939C0D40939B0DFB01E659FF4F7F
:10BDD00080819181A281B38160E070E048175907AA
:10BDE0006A077B0720F490939C0D80939B0D8091B4
:10BDF0009B0D90919C0D9F3460F09D3930F4D3E001
:10BE000096958795DA95E1F702C088E893E148E0D6
:10BE100014C0983230F0969587959695879544E0B2
:10BE20000CC0943120F09695879542E006C0803290
:10BE3000910510F480E290E041E040938A0D8097F4
:10BE4000811548E09407C8F0E92FFF27EE0FFF1F88
:10BE5000EE0FFF1FE35FF74FC590D590E590F4908C
:10BE6000A601B701AA27879FF001869FE10DFA1F5F
:10BE70000694EA1FFA1F112419C0FC01F695E795F4
:10BE8000EC7FE35FF34FC590D590E590F490A60169
:10BE9000877099278E9DF0018F9DF00D9E9DF00D6E
:10BEA000112463E0F695E7956A95E1F74E1B5F0B69
:10BEB0005093290140932801040F151F211D311DA6
:10BEC0000093860D1093870D2093880D3093890D74
:10BED00014C0232B31F481E090E09093960D809371
:10BEE000950D80918B0D90918C0D909329018093ED
:10BEF000280180918D0D80938A0D40916E0D509197
:10BF00006F0D6091700D7091710DE091800DF09149
:10BF1000810D84899589A689B789481759076A07C9
:10BF20007B0708F482C81092810D1092800D9091C9
:10BF3000AA0D8091A90D981731F08091A90D8F5FFE
:10BF40008F708093A90D9091AA0D8091A90D9817DB
:10BF500071F0C091A90D87E7C89FE0011124C55574
:10BF6000D24FFE01EC58FF4F81E0808302C0C0E059
:10BF7000D0E0D093810DC093800D209709F4AEC31B
:10BF8000888D998DAA8DBB8D80930E1690930F1678
:10BF9000A0931016B09311168C8D9D8DAE8DBF8D14
:10BFA0008093121690931316A0931416B09315163F
:10BFB00088A199A1AAA1BBA18093161690931716E8
:10BFC000A0931816B09319168CA19DA1AEA1BFA184
:10BFD00080931A1690931B16A0931C16B0931D16EF
:10BFE00088A599A5AAA5BBA580931E1690931F1698
:10BFF000A0932016B09321168AAD8093820D809174
:10C00000830D811111C01092860D1092870D109230
:10C01000880D1092890DFE01E25AFF4F2081318177
:10C020003F3408F041C04CC0BE0144E85DE0ECE79D
:10C03000FDE020E030E0DB011C96CD90DD90ED903E
:10C04000FC901F97CD28CE28CF2819F1DA018C91CA
:10C050008823F9F0D901A658B24F8C91D901AA0FC3
:10C06000BB1FAB5FB94E882341F08D919C91119716
:10C0700000811181801B910B07C08D919C911197BC
:10C0800000811181800F911F11969C938E93DA018C
:10C090001C922F5F3F4F6C5F7F4F4F5F5F4F329619
:10C0A0002230310541F6AFCF3D3930F403E036950B
:10C0B00027950A95E1F702C028E833E188E014C02B
:10C0C000383230F0369527953695279584E00CC0A8
:10C0D000343120F03695279582E006C020323105B4
:10C0E00010F420E230E081E080938A0D2052310983
:10C0F0002115B8E03B07D8F0E32FFF27EE0FFF1F15
:10C10000EE0FFF1FE35FF74F85919591A591B491D5
:10C11000AC01BD01AA27279FC001269F810D9A1F50
:10C1200006948A1F9A1F1124481B590B1BC0F90142
:10C13000F695E795EC7FE35FF34F45915591659157
:10C140007491DB01277033272A9FB0012B9F700D5C
:10C150003A9F700D1124E3E076956795EA95E1F733
:10C16000461B570B50938C0D40938B0D80918A0D7D
:10C1700080938D0DFE01EE58FF4F8081882309F4D6
:10C1800074C0CA59DF4F8881998190938F0D809335
:10C190008E0D9F3460F09D3930F443E0969587957D
:10C1A0004A95E1F702C088E893E128E014C098328C
:10C1B00030F0969587959695879524E00CC094313C
:10C1C00020F09695879522E006C08032910510F404
:10C1D00080E290E021E020938A0D9C0120523109F9
:10C1E0002115C8E03C07D8F0E32FFF27EE0FFF1F13
:10C1F000EE0FFF1FE35FF74F85919591A591B491E5
:10C20000AC01BD01AA27279FC001269F810D9A1F5F
:10C2100006948A1F9A1F1124481B590B1BC0F90151
:10C22000F695E795EC7FE35FF34F45915591659166
:10C230007491DB01277033272A9FB0012B9F700D6B
:10C240003A9F700D112403E0769567950A95E1F702
:10C25000461B570BCA01A0E0B0E08093900D90936D
:10C26000910DA093920DB093930D5093290140939B
:10C270002801E091800DF091810D20AD2093940D67
:10C28000EA58FF4F30818091051690910616892B50
:10C2900009F033608091071690910816892B09F0F8
:10C2A00034608091031638131CC0E091800DF0912A
:10C2B000810D4081518162817381F48805891689DD
:10C2C000D789DF01AB58BF4F3C9181E04115510543
:10C2D0006105710509F480E080933E16811144C028
:10C2E00087C0A5E1B2E0E9E1F2E080E090E041E062
:10C2F00050E0BA01082E01C0660F0A94EAF7D62F63
:10C30000C0910316C327C62341F1D32370910316AE
:10C31000DD2391F0762B70930316CD91DC9111976C
:10C320001881BA01008002C0660F771F0A94E2F7F5
:10C3300060956123688311C060956723609303163D
:10C34000CD91DC9111971881BA01008002C0660F6F
:10C35000771F0A94E2F7162B188301969396B396EB
:10C360008530910531F6A1CFC22FC1708F2D902F4E
:10C37000A12FBD2F6C017D01F594E794D794C7944C
:10C38000F094E094D094C094C11CD11CE11CF11C29
:10C39000C0923F16D0924016E0924116F09242169B
:10C3A000D1E03111D0E0D0933616809337169093B8
:10C3B0003816A0933916B0933A1640934716509307
:10C3C00048166093491670934A16CC2311F08FEFEC
:10C3D00001C081E080933C1681E08C2780933D165C
:10C3E000109243161092441610924516109246165B
:10C3F0004481558166817781F48805891689D789BA
:10C4000081E0411551056105710509F480E08093D3
:10C410006716882309F446C021FBCC27C0F98F2D6D
:10C42000902FA12FBD2F6C017D01F594E794D79437
:10C43000C794F094E094D094C094C11CD11CE11C2A
:10C44000F11CC0926816D0926916E0926A16F092BA
:10C450006B16D1E0313009F0D0E0D0935F168093B5
:10C46000601690936116A0936216B0936316409382
:10C470007016509371166093721670937316CC23D6
:10C4800011F08FEF01C081E08093651681E08C2769
:10C490008093661610926C1610926D1610926E169E
:10C4A00010926F164085518562857385F4880589E1
:10C4B0001689D78981E0411551056105710509F497
:10C4C00080E080939016882309F446C022FBCC2795
:10C4D000C0F98F2D902FA12FBD2F6C017D01F594F8
:10C4E000E794D794C794F094E094D094C094C11C7E
:10C4F000D11CE11CF11CC0929116D0929216E092D0
:10C500009316F0929416D1E0323009F0D0E0D09337
:10C5100088168093891690938A16A0938B16B093F1
:10C520008C164093991650939A1660939B167093AD
:10C530009C16CC2311F08FEF01C081E080938E1602
:10C5400081E08C2780938F16109295161092961684
:10C5500010929716109298164485558566857785B2
:10C56000F48805891689D78981E04115510561054F
:10C57000710509F480E08093B916882309F446C058
:10C5800023FBCC27C0F98F2D902FA12FBD2F6C013D
:10C590007D01F594E794D794C794F094E094D094F7
:10C5A000C094C11CD11CE11CF11CC092BA16D092DF
:10C5B000BB16E092BC16F092BD16D1E0333009F004
:10C5C000D0E0D093B1168093B2169093B316A09397
:10C5D000B416B093B5164093C2165093C316609329
:10C5E000C4167093C516CC2311F08FEF01C081E003
:10C5F0008093B71681E08C278093B8161092BE16F0
:10C600001092BF161092C0161092C116408951891F
:10C61000628973891489D589C6893789EB58FF4F98
:10C62000F08181E0411551056105710509F480E053
:10C630008093E216882309F445C024FBEE27E0F935
:10C64000812F9D2FAC2FB32F8C019D013595279500
:10C650001795079530952095109501951F4F2F4FF1
:10C660003F4F0093E3161093E4162093E5163093A2
:10C67000E61621E0F43009F020E02093DA168093EA
:10C68000DB169093DC16A093DD16B093DE16409374
:10C69000EB165093EC166093ED167093EE16EE23A6
:10C6A00011F08FEF01C081E08093E01681E08E27CA
:10C6B0008093E1161092E7161092E8161092E91690
:10C6C0001092EA161092960D1092950D10926E0D22
:10C6D00010926F0D1092700D1092710D81E079C063
:10C6E0007091041680910316781711F40C94C257B8
:10C6F000A5E1B2E0E9E1F2E080E090E021E030E0A5
:10C700000C948857A0910702B0910802FC91C901CE
:10C7100000900B0202C0880F991F0A94E2F7F82BD1
:10C72000FC930C946859109209160C946859A091C6
:10C730002A02B0912B02FC91C90100902E0202C086
:10C74000880F991F0A94E2F7F82BFC930C94555A22
:10C7500010920A160C94555AA0914D02B0914E02B7
:10C76000FC91C9010090510202C0880F991F0A94E0
:10C77000E2F7F82BFC930C94425B10920B160C948E
:10C78000425BA0917002B0917102FC91C9010090CE
:10C79000740202C0880F991F0A94E2F7F82BFC93E9
:10C7A0000C942F5C10920C160C942F5C10920D16AA
:10C7B0003FC9A0919302B0919402FC91C9010090ED
:10C7C000970202C0880F991F0A94E2F7F82BFC9396
:10C7D0002FC9DF91CF911F910F91FF90EF90DF90C4
:10C7E000CF90BF90AF909F908F907F906F905F9011
:10C7F0004F90089570919D0D7F5F70939D0D809176
:10C800009E0D8F5F80939E0D50919F0D6091A10DA5
:10C8100040E081E090E03FC030919E16E0917702C9
:10C82000F091780220917B02311199C0A2C0209131
:10C830000516309106162F5F3F4F18C02091051640
:10C84000309106161216130624F530919E16E091CB
:10C850007702F091780220917B023111A0C095C03F
:10C860002091051630910616215031093093061695
:10C8700020930516E0917002F091710270819C0185
:10C880000090740202C0220F331F0A94E2F7722B49
:10C8900070834F5F70E02091051630910616232BB0
:10C8A00061F470939D0D5091A00D6091A20D709157
:10C8B0009E0D40E081E090E045C0751708F4F1CF8F
:10C8C000461379C0EECF3091C716E0919A02F091ED
:10C8D0009B0220919E02311191C084C020910716C5
:10C8E000309108162F5F3F4F18C0209107163091E6
:10C8F00008161216130624F53091C716E0919A0215
:10C90000F0919B0220919E02311182C08DC0209136
:10C9100007163091081621503109309308162093DC
:10C920000716E0919302F091940270819C010090AF
:10C93000970202C0220F331F0A94E2F7722B708312
:10C940004F5F70E02091071630910816232B09F4F1
:10C9500075C0751708F472C0461373C06FC070813C
:10C96000DC0102C0AA0FBB1F2A95E2F77A2B708365
:10C970005ECF7081DC0102C0AA0FBB1F2A95E2F7CF
:10C980009D0120952723208352CF7081DC0102C0B6
:10C99000AA0FBB1F2A95E2F77A2B708361CF7081B3
:10C9A000DC0102C0AA0FBB1F2A95E2F79D0120956A
:10C9B0002723208355CFE0917002F091710270819E
:10C9C0009C010090740202C0220F331F0A94E2F708
:10C9D000209527232083209105163091061637FFD6
:10C9E0002DCF1ACF7081DC0102C0AA0FBB1F2A9580
:10C9F000E2F79D0120952723208370CF7081DC0111
:10CA000002C0AA0FBB1F2A95E2F77A2B708366CF6C
:10CA10007081DC0102C0AA0FBB1F2A95E2F79D01BD
:10CA200020952723208373CF7081DC0102C0AA0FD9
:10CA3000BB1F2A95E2F77A2B708369CF70939E0D06
:10CA40000895E0919302F091940270819C0100900E
:10CA5000970202C0220F331F0A94E2F72095272382
:10CA60002083209107163091081637FF3ECF2BCF39
:10CA70004F925F926F927F928F929F92AF92BF92EE
:10CA8000CF92DF92EF92FF920F931F93CF93DF939A
:10CA90001092820D92E7C92E9DE0D92E2DE9E22E4B
:10CAA0002DE0F22EC1EADDE03FE9A32E3DE0B32EFA
:10CAB00000E010E055245394F6016190719081904C
:10CAC00091906F01802F8D5F0E942F7B9B01AC01A5
:10CAD000C401B3010E94E6D99B01AC0160E070E49F
:10CAE0008CE196E40E940DD83B014C0120E030E03F
:10CAF00040E85FE3772D992D0E94E2D918164CF497
:10CB0000662D772D882D992D0E94F6D73B014C017B
:10CB100010C020E030E040E85FE3662D772D882DDF
:10CB2000992D0E9409D887FF04C0612C712C812C9B
:10CB3000912C662D772D882D992D0E94B4D8462EE4
:10CB4000F50161935F01662311F018820FC0262D55
:10CB5000372D482D592D60E070E080E89FE30E945A
:10CB60000DD80E94F6D70E94B4D8688388818111BD
:10CB700001C05882F801EE0FFF1FEB5FF94E1182E2
:10CB80001082F70141927F010F5F1F4F2196023003
:10CB9000110509F091CFDF91CF911F910F91FF9077
:10CBA000EF90DF90CF90BF90AF909F908F907F904D
:10CBB0006F905F904F9008952091AA0D9091A90DCC
:10CBC00081E0291380E008950F931F93CF93DF93A3
:10CBD000FB017FB7F894EC0188819981AA81BB8120
:10CBE00080930E1690930F16A0931016B093111603
:10CBF00080819181A281B381809312169093131644
:10CC0000A0931416B0931516FA0180819181A28128
:10CC1000B3818093161690931716A0931816B093AD
:10CC20001916E90188819981AA81BB8180931A161E
:10CC300090931B16A0931C16B0931D16F8018081CB
:10CC40009181A281B38180931E1690931F16A093A9
:10CC50002016B09321167FBFDF91CF911F910F91C6
:10CC600008958F929F92AF92BF92EF92FF920F938F
:10CC70001F93CF93DF93EFB7F89480900E169090A8
:10CC80000F16A0901016B0901116DC018D929D9297
:10CC9000AD92BC9213978091121690911316A091A9
:10CCA0001416B0911516EB0188839983AA83BB8370
:10CCB0008091161690911716A0911816B09119161A
:10CCC000EA0188839983AA83BB8380911A16909185
:10CCD0001B16A0911C16B0911D16E901888399833B
:10CCE000AA83BB8380911E1690911F16A0912016D7
:10CCF000B0912116E80188839983AA83BB83809130
:10CD0000820DD7018C93EFBFDF91CF911F910F91CF
:10CD1000FF90EF90BF90AF909F908F90089580917B
:10CD200073008D7F8093730006C08091A90D8F5F83
:10CD30008F708093A90D9091AA0D8091A90D9813E1
:10CD40005DC01092810D1092800D2FB7F8948091E4
:10CD50000E1690910F16A0911016B0911116809397
:10CD6000301590933115A0933215B09333158091FF
:10CD7000121690911316A0911416B0911516809367
:10CD8000341590933515A0933615B09337158091CF
:10CD9000161690911716A0911816B0911916809337
:10CDA000381590933915A0933A15B0933B1580919F
:10CDB0001A1690911B16A0911C16B0911D16809307
:10CDC0003C1590933D15A0933E15B0933F1580916F
:10CDD0001E1690911F16A0912016B09121168093D7
:10CDE000401590934115A0934215B09343152FBF62
:10CDF0008091730082608093730008959091AA0DD2
:10CE00008091A90D981709F496CF8FCF8093830D49
:10CE100081E08093840D8093850D089540E065E85E
:10CE20007AE183EA9DE00C941DD330EC20E48894F1
:10CE300010F0921710F0921B232B3695880F991F34
:10CE400023273E7FA9F710F0880F2907231FC90168
:10CE500008952F923F924F925F926F927F928F929E
:10CE60009F92AF92BF92CF92DF92EF92FF920F9379
:10CE70001F93CF93DF93CDB7DEB768970FB6F894C3
:10CE8000DEBF0FBECDBF1C0148015901F101EE58B4
:10CE9000FF4F80818823A1F0242F352FAB01213053
:10CEA000310561E04607510524F020E030E041E023
:10CEB00050E071E087169104A706B1042CF408C075
:10CEC00020E030E041E050E0812C912C5401A3940B
:10CED00071018EE5E80EF11CD7014D905D906D90CB
:10CEE0007C90C201772766270E947AD670588F4FB0
:10CEF0009F4F9C01552737FD5095452F2D833E832D
:10CF00004F835887F70180819181A281B381772770
:10CF10006627A50194010E947AD670588F4F9F4FC3
:10CF20009C01552737FD5095452F29873A874B8718
:10CF30005C874D815E816F81788548375105610539
:10CF4000710540F468E770E080E090E06D837E83D7
:10CF50008F83988789859A85AB85BC8588379105AD
:10CF6000A105B10540F428E730E040E050E0298712
:10CF70003A874B875C872D813E814F815885CA0156
:10CF8000B9010E9449DA2B013C0129853A854B857C
:10CF90005C85CA01B9010E9449DA6D8B7E8B8F8B4B
:10CFA000988F910122593F4FD9014D915D916D911B
:10CFB0007C91498B5A8B6B8B7C8B6A017B01CC0CEF
:10CFC000DD1CEE1CFF1CF101EE58FF4F8081882311
:10CFD00009F447C091012E593F4FD9014D915D9100
:10CFE0006D917C9149835A836B837C83C114D104F6
:10CFF000E104F10469F0CB01BA01641975098609ED
:10D000009709A70196010E94AFDA49015A0103C0AE
:10D01000812C912C540122273327A9012C193D0979
:10D020004E095F092D873E874F87588B232B242B72
:10D03000252BF9F06D897E898F89988D29813A8118
:10D040004B815C81621B730B840B950B2D853E8598
:10D050004F8558890E94AFDA29833A834B835C83DA
:10D060000CC019821A821B821C82812C912C5401C3
:10D0700004C019821A821B821C82D10154964D91E0
:10D080005D916D917C9157974D875E876F87788B07
:10D09000DB01CA0188199909AA09BB0929813A81CA
:10D0A0004B815C81821B930BA40BB50BB7FF3CC07B
:10D0B0008D849E84AF84B888C114D104E104F10446
:10D0C000D9F0A7019601C501B4010E9449DA64199B
:10D0D0007509860997092D893E894F89588D620FF8
:10D0E000731F841F951FA7019601220F331F441F32
:10D0F000551F0E94AFDA03C020E030E0A901DA0139
:10D10000C90157FF03C080E090E0DC014D855E85DA
:10D110006F85788984179507A607B70714F44C0123
:10D120005D0180E090E0DC01A5019401280F391F2A
:10D130004A1F5B1F2D873E874F87588BF10123AD18
:10D14000222309F412C1892B8A2B8B2B09F073C07F
:10D15000A50194012F5F3F4F4F4F5F4F57FF20C0F6
:10D1600050954095309521953F4F4F4F5F4F6989BE
:10D170007A898B899C890E9449DA660F771F881FFC
:10D18000991F641575058605970508F04BC0A30126
:10D190009201261B370B480B590BDA01C90110C04D
:10D1A00069897A898B899C890E9449DADC01CB01E3
:10D1B000880F991FAA1FBB1F840D951DA61DB71DA3
:10D1C000811530E89307A105B10558F40E94156751
:10D1D0002C01662457FC6094762C3201552444249B
:10D1E00024C0F12C22E0B695A795979587952A95AE
:10D1F000D1F7F394811540E89407A105B10590F7A4
:10D200000E9415672C01662457FC6094762C32012D
:10D210005524442404C0440C551C661C771CFA9405
:10D22000D2F703C0412C512C32012301772457FC43
:10D230007094672C07C0F101E25AFF4F4080518083
:10D2400062807380181419041A041B04F4F4D301C7
:10D25000C2012D813E814F815885821B930BA40B07
:10D26000B50BAC0133272227609197157091981563
:10D270008091991590919A150E947AD6BB2797FDB7
:10D28000B095AB2F6C0197FF02C0C12CD12C4D85FE
:10D290005E856F8578894F5F5F4F6F4F7F4FF101DC
:10D2A00084899589A689B789481759076A077B0732
:10D2B0000CF063C029853A854B855C85421A530A78
:10D2C000640A750AA201332722276091971570918D
:10D2D00098158091991590919A150E947AD67C01A3
:10D2E0008091931590919415A0919515B0919615F4
:10D2F000892B8A2B8B2B99F169817A818B819C8177
:10D30000AB0133272227F101E259FF4F8081918140
:10D31000A281B38165E0B595A795979587956A95A4
:10D32000D1F7772766270E94E4D62B013C01609154
:10D33000931570919415809195159091961520E014
:10D3400030E044E650E00E947AD6A30192010E94A8
:10D350007AD6BB2797FDB095AB2FB7FF03C080E00F
:10D3600090E0DC01F7FE0EC00BC080E090E0DC0135
:10D37000E12CF12CC12CD12C05C080E090E0DC0127
:10D38000E12CF12C2FB7F894F101EC58FF4F3081CC
:10D39000311142C0F101EE58FF4F3081332369F063
:10D3A000F10184A695A6A6A6B7A64D855E856F85D4
:10D3B000788940AB51AB62AB73AB5101F6E6AF0E6F
:10D3C000B11C4D815E816F817885F5014083518369
:10D3D000628373835101FAE6AF0EB11C49855A8509
:10D3E0006B857C85F5014083518362837383F101F2
:10D3F000D5AEC4AEF7AEE6AEEC5BFF4F1182108245
:10D40000F101EA5BFF4F11821082F101E05CFF4FF6
:10D4100080839183A283B3832FBF68960FB6F8945D
:10D42000DEBF0FBECDBFDF91CF911F910F91FF9057
:10D43000EF90DF90CF90BF90AF909F908F907F90B4
:10D440006F905F904F903F902F9008952F923F9252
:10D450004F925F926F927F928F929F92AF92BF9204
:10D46000CF92DF92EF92FF920F931F93CF93DF93B0
:10D4700000D000D0CDB7DEB71C018B01009709F4B6
:10D4800097C16115710509F493C19C01205B3F4F61
:10D49000D9018D919D910D90BC91A02D89839A8386
:10D4A000AB83BC83F101E45BFF4F80819181A2815A
:10D4B000B38129813A814B815C8182179307A4074C
:10D4C000B50709F475C1F101E35AFF4F808181115D
:10D4D00047C1FB01ED58FF4F8081882309F440C10B
:10D4E000FB01E45BFF4F80819181A281B3818217B0
:10D4F0009307A407B5070CF033C1BC01CD015CE074
:10D5000095958795779567955A95D1F7F101E85AE2
:10D51000FF4F80809180A280B380B094A0949094BB
:10D520008094811C911CA11CB11CE6E0B594A794C9
:10D5300097948794EA95D1F7F101EC5AFF4FC08098
:10D54000D180E280F380F5E0F594E794D794C79416
:10D55000FA95D1F79B01AC010E947AD62B013C01D0
:10D56000A5019401C701B6010E947AD6461A570A4E
:10D57000680A790AF12C411451046104710409F418
:10D5800042C0D301C20188279927AA27B07E892BE0
:10D590008A2B8B2B09F4FAC01414150416041704F3
:10D5A00094F5C301BB2797FDB095AB2F36E03F152F
:10D5B000A8F40E941567AA2797FDA095BA2FDC0151
:10D5C000992788272F2D30E02650310904C0B595C2
:10D5D000A795979587952A95D2F718C00E94156749
:10D5E000AA2797FDA095BA2FDC019927882726E066
:10D5F00030E02F19310904C0880F991FAA1FBB1FE3
:10D600002A95D2F703C080E090E0DC0129813A81BD
:10D610004B815C81281739074A075B0744F4F10105
:10D62000E05BFF4F80819181A281B38191C0F801BD
:10D63000E45BFF4F6081718182819381FCE095956D
:10D64000879577956795FA95D1F7F101E85AFF4FDD
:10D6500080809180A280B380B094A09490948094B4
:10D66000811C911CA11CB11CA6E0B594A7949794B1
:10D670008794AA95D1F7F101EC5AFF4FC080D18071
:10D68000E280F380B5E0F594E794D794C794BA9517
:10D69000D1F79B01AC010E947AD62B013C01A50178
:10D6A0009401C701B6010E947AD693018201061B3C
:10D6B000170B280B390BB901A80110E041155105D2
:10D6C0006105710509F441C0DB01CA01882799276A
:10D6D000AA27B07E892B8A2B8B2B09F460C01416E5
:10D6E0001506160617068CF5CB01BB2797FDB095DE
:10D6F000AB2F1730A8F00E941567AA2797FDA095B9
:10D70000BA2FDC0199278827212F30E026503109D4
:10D7100004C0B595A795979587952A95D2F718C017
:10D720000E941567AA2797FDA095BA2FDC019927BB
:10D73000882726E030E0211B310904C0880F991F9B
:10D74000AA1FBB1F2A95D2F703C080E090E0DC013E
:10D75000F101E45BFF4F80839183A283B38310C008
:10D76000F101E45BFF4F29813A814B815C81208389
:10D77000318342835383F101ED58FF4F81E0808371
:10D78000F101E45AFF4F81E0808312C022E0440C93
:10D79000551C661C771C2A95D1F7F394ECCE92E0C9
:10D7A000440F551F661F771F9A95D1F71F5F86CFCD
:10D7B0000F900F900F900F90DF91CF911F910F91CD
:10D7C000FF90EF90DF90CF90BF90AF909F908F90A1
:10D7D0007F906F905F904F903F902F900895FF92B1
:10D7E0000F931F93CF93DF931091AA0D8FB7F894E7
:10D7F0000091A90D8FBF60E070E0A7E7FA2E0DC081
:10D80000111101C010E11150F19EE0011124C55524
:10D81000D24FCE010E94266ABE011013F1CFDF91D4
:10D82000CF911F910F91FF9008952F923F924F92A9
:10D830005F926F927F928F929F92AF92BF92CF92A0
:10D84000DF92EF92FF920F931F93CF93DF9300D05D
:10D8500000D0CDB7DEB71C018B01009709F472C16F
:10D86000FB01EE58FF4F8081882309F46BC1F10161
:10D87000E35AFF4F8081811165C1F101ED58FF4FDF
:10D880008081882309F45EC1F101E45BFF4F808150
:10D890009181A281B381FB01E45BFF4F4080518005
:10D8A0006280738084159505A605B7050CF04AC102
:10D8B000BC01CD01ECE09595879577956795EA9544
:10D8C000D1F7F101E85AFF4F80809180A280B380A8
:10D8D000F6E0B594A79497948794FA95D1F7F1015F
:10D8E000EC5AFF4FC080D180E280F380A5E0F59430
:10D8F000E794D794C794AA95D1F79B01AC010E94F5
:10D900007AD669837A838B839C83A5019401C701AE
:10D91000B6010E947AD629813A814B815C81620FDF
:10D92000731F841F951FF12C6115710581059105E9
:10D9300009F444C0812C912CA12C50EEB52E8622E6
:10D940009722A822B92289288A288B2809F4E8C0BE
:10D9500016161706180619068CF5BB2797FDB09505
:10D96000AB2F36E03F15A8F40E941567AA2797FD54
:10D97000A095BA2FDC01992788272F2D30E026505B
:10D98000310904C0B595A795979587952A95D2F743
:10D9900018C00E941567AA2797FDA095BA2FDC0131
:10D9A0009927882726E030E02F19310904C0880F15
:10D9B000991FAA1FBB1F2A95D2F703C080E090E0F1
:10D9C000DC01481659066A067B0644F4F801E45B5C
:10D9D000FF4F80819181A281B38188C0F101E45B16
:10D9E000FF4F6081718182819381FCE095958795DD
:10D9F00077956795FA95D1F7F101E85AFF4F408086
:10DA0000518062807380A6E0759467945794479420
:10DA1000AA95D1F7F101EC5AFF4FC080D180E28086
:10DA2000F380B5E0F594E794D794C794BA95D1F70D
:10DA30009B01AC010E947AD64B015C01A3019201CB
:10DA4000C701B6010E947AD6680D791D8A1D9B1DFB
:10DA5000B12C611571058105910509F444C0C12CF3
:10DA6000D12CE12CE0EEFE2EC622D722E822F922AC
:10DA7000CD28CE28CF2809F45CC016161706180644
:10DA800019068CF5BB2797FDB095AB2F46E04B15DB
:10DA9000A8F40E941567AA2797FDA095BA2FDC016C
:10DAA000992788274B2D50E04650510904C0B59561
:10DAB000A795979587954A95D2F718C00E94156744
:10DAC000AA2797FDA095BA2FDC019927882726E081
:10DAD00030E02B19310904C0880F991FAA1FBB1F02
:10DAE0002A95D2F703C080E090E0DC01F801E45B06
:10DAF000FF4F4081518162817381481759076A073E
:10DB00007B0701F180839183A283B383F801E45AF8
:10DB1000FF4F81E08083F801ED58FF4F808312C0F2
:10DB200022E0660F771F881F991F2A95D1F7F3947B
:10DB3000FBCEB2E0660F771F881F991FBA95D1F709
:10DB4000B39487CF0F900F900F900F90DF91CF91EC
:10DB50001F910F91FF90EF90DF90CF90BF90AF900B
:10DB60009F908F907F906F905F904F903F902F90FD
:10DB700008950F931F93CF93DF931091A90D80E029
:10DB800090E007E70DC0019FE0011124C555D24F79
:10DB9000BE010E94156C1F5F103109F410E0CE0128
:10DBA0002091AA0D1213EFCFDF91CF911F910F910A
:10DBB00008958F929F92AF92BF92CF92DF92EF9291
:10DBC000FF920F931F93CF93DF939090A90DC0E026
:10DBD000D0E0B7E78B2E53C0899C500111248BEA0B
:10DBE0009DE0A80EB91E209709F443C0FE01EE582F
:10DBF000FF4F80818823E9F1F501EE58FF4F8081C6
:10DC00008823B9F1FE01E45AFF4F8081811106C0DB
:10DC1000F501E45AFF4F8081882359F18E01085B9A
:10DC20001F4FF8012081318142815381F501E45B6E
:10DC3000FF4F60817181828193810E94E4D66B01E4
:10DC40007C01F8012081318142815381FE01E45B36
:10DC5000FF4F60817181828193810E94E4D6AB0184
:10DC6000BC0197018601CE010E942967C45ADF4F8B
:10DC700018829394F0E19F1201C0912CE5018091EC
:10DC8000AA0D9812A9CF2097D1F0FE01E85BFF4FB3
:10DC90002081318142815381FE01E45BFF4F60812D
:10DCA0007181828193810E94E4D6AB01BC018A011B
:10DCB0009B01CE010E942967C45ADF4F1882DF9171
:10DCC000CF911F910F91FF90EF90DF90CF90BF9079
:10DCD000AF909F908F9008950E94EF6B0E94B96D56
:10DCE0000C94D96D0F931092AA0D1092A90D109259
:10DCF0003015109231151092321510923315109282
:10DD00003415109235151092361510923715109261
:10DD100038151092391510923A1510923B15109241
:10DD20003C1510923D1510923E1510923F15109221
:10DD300040151092411510924215109243156093B0
:10DD40009715709398158093991590939A15209331
:10DD50009315309394154093951550939615009311
:10DD60001B1581E0809306020F9108952F923F9238
:10DD70004F925F926F927F928F929F92AF92BF92DB
:10DD8000CF92DF92EF92FF920F931F93CF93DF9387
:10DD9000CDB7DEB7C154D1090FB6F894DEBF0FBEC0
:10DDA000CDBF4B015C015CA34BA33DA72CA7809189
:10DDB000AF159091B015892B41F09091AA0D8091EB
:10DDC000A90D981711F40C94A8774090AA0D142D62
:10DDD0001F5F1EA7103109F41EA68091AA0D27E728
:10DDE000829F100111244BEA5DE0240E351EF101E3
:10DDF000EC58FF4F1082F101EE58FF4F0083D10124
:10DE0000DA96EC92DA978FB7F894C0903015D090EC
:10DE10003115E0903215F0903315F101C08ED18E9E
:10DE2000E28EF38E00913415109135152091361540
:10DE3000309137155C960D931D932D933C935F970E
:10DE4000409038155090391560903A1570903B15F8
:10DE50004FA658AA69AA7AAA90964D925D926D92A1
:10DE60007C92939740903C1550903D1560903E15E4
:10DE700070903F154BAA5CAA6DAA7EAA94964D920B
:10DE80005D926D927C92979740904015509041150D
:10DE900060904215709043154FAA58AE69AE7AAEA5
:10DEA00098964D925D926D927C929B978FBF409019
:10DEB00062155090631560906415709065154F8AD7
:10DEC000588E698E7A8E4D925D926D927C921397E8
:10DED00040906615509067156090681570906915B0
:10DEE0004F8E58A269A27AA214964D925D926D92BD
:10DEF0007C92179740906A1550906B1560906C1546
:10DF000070906D154FA258A669A67AA618964D92E4
:10DF10005D926D927C921B9740916E1550916F159A
:10DF20006091701570917115448755876687778762
:10DF30008091721590917315A0917415B09175151B
:10DF4000808B918BA28BB38B409077155090781576
:10DF50006090791570907A15448A558A668A778A16
:10DF6000EB58FF4F7090761570824F88588C698CF3
:10DF70007A8C452846284728D9F44F8C58A069A0A8
:10DF80007AA045284628472899F44FA058A469A4A8
:10DF90007AA445284628472859F4411551056105BA
:10DFA000710541F4E1E0EBA70097A105B10521F46B
:10DFB0001BA602C0F1E0FBA7F10110AE40901C15BA
:10DFC00050901D1560901E1570901F154C145D0427
:10DFD0006E047F041CF4FF24F394F0AEC09020156F
:10DFE000D0902115E0902215F0902315C016D1068F
:10DFF000E206F30624F4F10120AD226020AF009187
:10E0000024151091251520912615309127154FA420
:10E0100058A869A87AA8041515052605370524F41B
:10E02000F10120AD246020AF009128151091291531
:10E0300020912A1530912B154BA85CA86DA87EA8BD
:10E04000041515052605370524F4F10120AD2860D7
:10E0500020AF00912C1510912D1520912E15309187
:10E060002F154FA858AC69AC7AAC041515052605D8
:10E07000370524F4F10120AD206120AF4115510591
:10E080006105710541F00097A105B10509F009C0CE
:10E09000F10111AE0BC00097A105B10511F021E00F
:10E0A00003C0ECA5FDA52081F10121AF4F88588C5C
:10E0B000698C7A8C45284628472829F02091041637
:10E0C000216020930416CF8CD8A0E9A0FAA0CD2817
:10E0D000CE28CF2829F02091041622602093041620
:10E0E000EFA0F8A409A51AA5EF28E02AE12A29F053
:10E0F00020910416246020930416452B462B472BB1
:10E1000029F020910416286020930416892B8A2B6D
:10E110008B2B29F0809104168061809304168091E6
:10E120000416F101EA58FF4F808390911B15992343
:10E1300011F0846080836091AA0D8091A90D681B05
:10E140006F70462E512C58A24F8E452841F51092E3
:10E15000E9151092EA151092EB151092EC15109239
:10E16000ED151092EE151092EF151092F015109219
:10E17000F1151092F2151092F3151092F4151092F9
:10E18000F5151092F6151092F7151092F8151092D9
:10E19000F9151092FA151092FB151092FC15EBA1CF
:10E1A000FCA180819181A281B3818101025A1F4F1C
:10E1B000F80180839183A283B3832091AF153091BE
:10E1C000B0152115310509F443C08091060288235A
:10E1D00041F04F8C58A042165306D4F1109206021B
:10E1E00037C06F8C78A06216730694F5A301423095
:10E1F000510574F1C901AA2797FDA095BA2FAC016A
:10E2000033272227862F90E0A0E0B0E0772766270B
:10E210000E94E4D66B017C019B01AC01C501B401F5
:10E220000E947AD64B015C01F80180819181A28124
:10E23000B38177276627A70196010E947AD6BB276C
:10E2400097FDB095AB2FF80180839183A283B383B0
:10E2500081149104A104B10409F45FC0F101EC5AE6
:10E26000FF4F4BA44420C1F0D101D9969C9104E00A
:10E27000909FD0011124A557BA4E8D919D910D907C
:10E28000BC91A02DB7FF10C0B095A0959095819539
:10E290009F4FAF4FBF4F08C080917B1590917C1569
:10E2A000A0917D15B0917E1580839183A283B38365
:10E2B000F101EC5AFF4F208131814281538160E0AE
:10E2C00070E081E090E00E94E4D66B017C019B014C
:10E2D000AC01C501B4010E947AD62B013C010FE7C5
:10E2E00015E19E012F5F3F4F388F2F8BD8016D9125
:10E2F0007D918D919D918D01A30192010E947AD60D
:10E30000EF89F88D6193719381939193F88FEF8BDF
:10E31000F5E103391F0751F703C0C12CD12C760159
:10E32000F101EE58FF4F8081811120C1EBA1FCA1CA
:10E3300080819181A281B381F101E25AFF4F8083F4
:10E340009183A283B38389288A288B2809F491C0FA
:10E350008E010F5F1F4F65EBA62E65E1B62E4E01B5
:10E36000F5E18F0E911C412C512C32016394D801A0
:10E370003C9111962C91119712969C91129713969D
:10E380008C910C5F1F4FC32ED22EE92EF82EF7FE74
:10E3900008C0F094E094D094C094C11CD11CE11C3E
:10E3A000F11CF50160817181828193816C157D057D
:10E3B0008E059F05A4F4A70196010E94E4D6461697
:10E3C0005706680679065CF0D5016D917D918D91B7
:10E3D0009C91A70196010E94E4D62B013C01B4E078
:10E3E000AB0EB11C0815190511F6EBA1FCA180813B
:10E3F0009181A281B3818101025A1F4F81159048FA
:10E40000A105B10510F1F80180819181A281B3814C
:10E4100024E0B695A795979587952A95D1F780839F
:10E420009183A283B38377276627A30192010E9479
:10E430007AD6BB2797FDB095AB2F54E0880F991F74
:10E44000AA1FBB1F5A95D1F70FC0F8018081918197
:10E45000A281B38177276627A30192010E947AD611
:10E46000BB2797FDB095AB2FF80180839183A283E2
:10E47000B383D1019C961D921D921D921C929F9771
:10E4800054968D919D910D90BC91A02D0196A11D4A
:10E49000B11DF10180AB91ABA2ABB3ABE25AFF4F20
:10E4A0006081718182819381F101EE59FF4F9B015F
:10E4B000AC010E9449DA60837183828393834EA406
:10E4C0004092AA0D2FB7F89480911C1590911D15BC
:10E4D000A0911E15B0911F158093301590933115A2
:10E4E000A0933215B093331580912015909121158A
:10E4F000A0912215B0912315809334159093351572
:10E50000A0933615B0933715809124159091251559
:10E51000A0912615B0912715809338159093391541
:10E52000A0933A15B0933B15809128159091291529
:10E53000A0912A15B0912B1580933C1590933D1511
:10E54000A0933E15B0933F1580912C1590912D15F9
:10E55000A0912E15B0912F158093401590934115E1
:10E56000A0934215B09343152FBF66C55BA451100D
:10E5700035C06F8C78A0672889F5809144159091FB
:10E580004515A0914615B0914715181619061A069B
:10E590001B0624F581010C5A1F4FD8016D917D9106
:10E5A0008D919C911616170618061906BCF41814BE
:10E5B00019041A041B0494F4A50194010E94E4D6E2
:10E5C00020914415309145154091461550914715BD
:10E5D00062177307840795070CF4BFC4F101E25A70
:10E5E000FF4F6081718182819381F101EE59FF4F6C
:10E5F0009B01AC010E9449DA60837183828393831B
:10E60000F101E85BFF4F80829182A282B382F10127
:10E6100084899589A689B7898115F0E89F07A105A6
:10E62000B10568F0A7019601220F331F441F551F43
:10E63000B595A795979587957727662704C077277F
:10E640006627A70196010E947AD62B013C01F101B1
:10E65000E259FF4F9301552737FD5095452FCBA425
:10E66000CC2079F06091CD157091CE158091CF15A9
:10E670009091D0150E9449DA6083718382839383DD
:10E68000F0C06091D1157091D2158091D315909101
:10E69000D4150E9449DA60837183828393833CAEF0
:10E6A0002BAE0BE915E118A70FA32AE435E13CAB2B
:10E6B0002BABFDA7ECA7ABADBCAD6D917D918D9162
:10E6C0009D91BCAFABAF6F8B788F898F9A8F672B83
:10E6D000682B692B09F4B6C0D1015496CD90DD901A
:10E6E000ED90FC905797CFA6D8AAE9AAFAAAEBA971
:10E6F000FCA94081518162817381AFA1B8A54C15FD
:10E700005D056E057F0510F1CD90DD90ED90FC90DC
:10E71000ECA5FDA560817181828193812F89388D5F
:10E72000498D5A8D0E9449DA4B015C01A70196017F
:10E730006FA578A989A99AA90E9449DA681579056F
:10E740008A059B0508F07EC0DF0177C0CD90DD9083
:10E75000ED90FC90CFAAD8AEE9AEFAAECF88D88CB7
:10E76000E98CFA8CFF0CCC08DC2C7601CBA2DCA265
:10E77000EDA2FEA2ACA5BDA50D911D912D913C91E0
:10E7800058016901E12CF12C00E010E02F89388D4F
:10E79000498D5A8D6BA1762F862F962F0E942EDBE6
:10E7A000922E832E4BA35DAF6EAF7FAF21968FAFBE
:10E7B000219722969FAF2297EFA8F8AC09AD1AAD2A
:10E7C0006701780100E010E09801CF8AD88EE98EC9
:10E7D000FA8E0B8F1C8F2D8F3E8F8FA598A9A9A91C
:10E7E000BAA98C019D015C016901E12CF12C00E0CA
:10E7F00010E02F89388D498D5A8D60E070E080E0FF
:10E8000090E00E942EDB59016A017B018C01292DC9
:10E81000382D4BA15DAD6EAD7FAD21968FAD2197AB
:10E8200022969FAD22970E9430DC61F058F0CFA86D
:10E83000D8ACE9ACFAACACA5BDA5CD92DD92ED9219
:10E84000FC921397EFA1F8A53496F8A7EFA30BA9B4
:10E850001CA90C5F1F4F1CAB0BABEF5AF54109F025
:10E860002ACFF101E259FF4F80819181A281B381CA
:10E87000811520E89207A105B10528F477276627BE
:10E88000A301920117C0009732E0A307B105C0F4BD
:10E89000A3019201E2E05595479537952795EA95B2
:10E8A000D1F7F2E0B595A79597958795FA95D1F7A9
:10E8B000772766270E94E4D6F101E85AFF4F38C057
:10E8C0008101085A1F4F009748E0A407B105D8F40A
:10E8D000A3019201F4E05595479537952795FA9550
:10E8E000D1F764E0B595A795979587956A95D1F787
:10E8F000772766270E94E4D6D8016D937D938D9388
:10E900009C93139719C0A301920165E05595479513
:10E91000379527956A95D1F775E0B595A7959795A1
:10E9200087957A95D1F7772766270E94E4D6F80174
:10E930006083718382839383F101E259FF4F808169
:10E940009181A281B3816C017D0100E010E098010A
:10E950008F8BD88EE98EFA8E0B8F1C8F2D8F3E8F6A
:10E96000AFEDAA2EB8E1BB2E12E0C12ED12CE12CC6
:10E97000F12C00E010E02F89388D498D5A8D60E030
:10E9800070E080E090E00E942EDB0EE00E9421DC2F
:10E99000D101D4962C93D497D5963C93D597D696FF
:10E9A0004C93D697D7965C93F101E85BFF4F4F8C61
:10E9B00058A04528B9F46091B1157091B2158091B5
:10E9C000B3159091B41560935E1570935F158093A5
:10E9D00060159093611520813181428153810E949D
:10E9E000E4D6E2C280819181A281B3814091C915B0
:10E9F0005091CA156091CB157091CC1548175907E5
:10EA00006A077B076CF080935E1590935F15A09367
:10EA10006015B093611560E070E081E090E0C4C2E1
:10EA20008E010F5F1F4F29EE35E138A72FA345EB6D
:10EA300055E158A34F8FBE016B5E7F4F7E8B6D8B70
:10EA40003CA32BA3188F0F8B412C512C32016394C4
:10EA5000AF89B88D2D913D914D915D91B88FAF8B60
:10EA6000EBA1FCA181919191A191B191FCA3EBA3A8
:10EA70002115310541055105D9F1EF8DF8A1C0806F
:10EA8000D180E280F38049015A01881A990AAA0AC2
:10EA9000BB0AB7FE08C0B094A09490948094811CE7
:10EAA000911CA11CB11CC814D904EA04FB0404F590
:10EAB00082179307A407B5073CF4BC01CD016C0D88
:10EAC0007D1D8E1D9F1D06C0BC01CD016C197D09E9
:10EAD0008E099F090E94E4D6161617061806190615
:10EAE000F4F4641575058605970514F42B013C01B3
:10EAF0002F8D38A12C5F3F4F38A32F8FCF88D88C14
:10EB0000ED88FE88CE14DF0409F0A2CFC301B20164
:10EB10004114510421E06206710479F103C0412CD3
:10EB2000512C3201F101E85BFF4F608171818281DC
:10EB30009381A30192010E947AD660935E1570932F
:10EB40005F158093601590936115D8016D917D914B
:10EB50008D919D918D01A30192010E947AD6EFA122
:10EB6000F8A56193719381939193F8A7EFA3CD8852
:10EB7000DE880C151D0549F710C0F101E85BFF4F59
:10EB8000008111812281338100935E1510935F15FE
:10EB9000209360153093611507C26091B115709193
:10EBA000B2158091B3159091B4154CE09595879569
:10EBB000779567954A95D1F7F101E85AFF4F808024
:10EBC0009180A280B38056E0B594A79497948794DF
:10EBD0005A95D1F7F101EC5AFF4FC080D180E28005
:10EBE000F380E5E0F594E794D794C794EA95D1F7DC
:10EBF0009B01AC010E947AD66F8B788F898F9A8F98
:10EC0000A5019401C701B6010E947AD6EF88F88C5D
:10EC1000098D1A8D6E0D7F1D801F911F10E06115EB
:10EC200071058105910509F443C0C12CD12CE12C5B
:10EC300030EEF32EC622D722E822F922CD28CE28A4
:10EC4000CF2809F4F0C1161617061806190684F520
:10EC5000BB2797FDB095AB2F1730A8F00E94156722
:10EC6000AA2797FDA095BA2FDC0199278827212F85
:10EC700030E02650310904C0B595A7959795879542
:10EC80002A95D2F718C00E941567AA2797FDA0956C
:10EC9000BA2FDC019927882726E030E0211B3109B3
:10ECA00004C0880F991FAA1FBB1F2A95D2F703C063
:10ECB00080E090E0DC0140915E1550915F1560911D
:10ECC000601570916115C090B115D090B215E090AB
:10ECD000B315F090B4159101245B3F4F8101005BA7
:10ECE0001F4FF9014C155D056E057F0554F4C08278
:10ECF000D182E282F382F801C082D182E282F38281
:10ED000009C04083518362837383F8014083518338
:10ED100062837383F101E85BFF4F4081518162811F
:10ED20007381F101E35AFF4F84179507A607B707D0
:10ED30001CF081E0808301C01082F101E45AFF4F92
:10ED400081E08083F101ED58FF4F1082F101E05C1A
:10ED5000FF4F1082118212821382F1018485958502
:10ED6000A685B785892B8A2B8B2B41F480899189C5
:10ED7000A289B389892B8A2B8B2BD9F0FBA5F111A2
:10ED800018C08091971590919815A0919915B09100
:10ED90009A15892B8A2B8B2B19F5809193159091BD
:10EDA0009415A0919515B0919615892B8A2B8B2BD4
:10EDB000B9F4D101DB961C92DB97DD961C921E9272
:10EDC000DC97DF961C921E92DE97F101EC5BFF4F01
:10EDD00011821082F101EA5BFF4F1182108203C0A1
:10EDE00081E0F10183AF93018201B301A201C1016E
:10EDF0000E9429674EA44092AA0D2FB7F8948091E3
:10EE00001C1590911D15A0911E15B0911F15809392
:10EE1000301590933115A0933215B093331580912E
:10EE2000201590912115A0912215B0912315809362
:10EE3000341590933515A0933615B09337158091FE
:10EE4000241590912515A0912615B0912715809332
:10EE5000381590933915A0933A15B0933B158091CE
:10EE6000281590912915A0912A15B0912B15809302
:10EE70003C1590933D15A0933E15B0933F1580919E
:10EE80002C1590912D15A0912E15B0912F158093D2
:10EE9000401590934115A0934215B09343152FBF91
:10EEA0000E946C6EF10180859185A285B385892BC6
:10EEB0008A2B8B2B09F4C0C080914915882309F453
:10EEC000BBC02091481580E991E0289FA001299FAF
:10EED000500D1124662757FD6095762F80912415DB
:10EEE00090912515A0912615B091271584179507A7
:10EEF000A607B7070CF4A0C01092491587E090E070
:10EF00000E94C0A683ED9AE00E9443A789E090E0AA
:10EF10000E94C0A661E070E081E0CF5BDF4F0FB6DA
:10EF2000F894DEBF0FBECDBFDF91CF911F910F913F
:10EF3000FF90EF90DF90CF90BF90AF909F908F9019
:10EF40007F906F905F904F903F902F900C944C3C2F
:10EF500081E0809306020C94E56ED8016D917D915D
:10EF60008D919C910E94E4D62B013C01A501940156
:10EF70000E94E4D69B01AC018101025A1F4FF801A7
:10EF800080819181A281B381772766270E947AD6FA
:10EF9000BB2797FDB095AB2FF80180839183A283A7
:10EFA000B383420153011ACB09811A812B813C8121
:10EFB0000093E9151093EA152093EB153093EC15A7
:10EFC0000D811E812F8138850093ED151093EE156C
:10EFD0002093EF153093F01509851A852B853C8514
:10EFE0000093F1151093F2152093F3153093F41557
:10EFF0000D851E852F8538890093F5151093F6151C
:10F000002093F7153093F81509891A892B893C89C3
:10F010000093F9151093FA152093FB153093FC1506
:10F020002B013C01BACD02E0660F771F881F991FA4
:10F030000A95D1F71F5FF3CDCF5BDF4F0FB6F89482
:10F04000DEBF0FBECDBFDF91CF911F910F91FF901B
:10F05000EF90DF90CF90BF90AF909F908F907F9078
:10F060006F905F904F903F902F9008958093491537
:10F0700060E080E592E00E9466A0809348150895C4
:10F080008091491508958093491508950F931F9312
:10F09000CF93CFB7F894FC0180819181A281B38195
:10F0A0008093301590933115A0933215B09333159A
:10F0B000FB0180819181A281B3818093341590936B
:10F0C0003515A0933615B0933715FA0180819181DB
:10F0D000A281B3818093381590933915A0933A1586
:10F0E000B0933B15F90180819181A281B381809316
:10F0F0003C1590933D15A0933E15B0933F15F80134
:10F1000080819181A281B3818093401590934115B4
:10F11000A0934215B09343158091AA0D9091A90D2B
:10F12000891B8F7061F400E415E12CE335E148E3BD
:10F1300055E164E375E180E395E10E94E465CFBFAA
:10F14000CF911F910F91089540E065E87AE18DEF2E
:10F1500095E10C941DD32F923F924F925F926F9244
:10F160007F928F929F92AF92BF92CF92DF92EF9257
:10F17000FF920F931F93CF93DF93CDB7DEB76797BF
:10F180000FB6F894DEBF0FBECDBF898B8823B1F0D8
:10F1900060E082E090E00E9466A0F82E60E084E0EB
:10F1A00090E00E9466A08E8360E08EE092E00E9474
:10F1B00066A0813729F00E94843702C01E82F12C9C
:10F1C00082E296E19F8B8E8B07E012E090E2892E1F
:10F1D00092E0992EA2E1B2E0B887AF83EBE0F2E0D3
:10F1E000FA87E98789E192E09D838C8327E2222ECA
:10F1F00022E0322EA1E7B3E0BC87AB87E6E4F2E081
:10F20000FE87ED87A12CB12C1B821A82C12CD12C38
:10F210008F2D90E09B8B8A8BEE24E394F12CBE81A2
:10F22000AB2FB0E0BD8BAC8BC982E989EE2309F42A
:10F2300091C1FE81F7FF0AC08C899D890C2C02C008
:10F24000959587950A94E2F7817001C081E0AE89B7
:10F25000BF898C93EA81FB81EE5DF94EF88BEF87D5
:10F260008A899B890C2C02C0959587950A94E2F7B0
:10F2700081708183F501E35AFC4F408151816281A5
:10F280007381C5018C559E4F0E94A6A00E94E0D8B4
:10F2900020E034E244E759E40E940DD8AE89BF89EA
:10F2A00012966D937D938D939C931597EB85FC85BA
:10F2B000608171818D859E850E9483A0BC0180E064
:10F2C00090E00E94E0D8AE89BF8916966D937D9339
:10F2D0008D939C931997F501E558FC4F408151811E
:10F2E00062817381C501805F9D4F0E94A6A00E942C
:10F2F000E2D8EE89FF8922813381448155810E94C1
:10F30000E6D920E030E04AE754E40E94E6D90E94C2
:10F31000AFD828EE33E040E050E00E94AFDA290198
:10F320003A01F981F23011F118F0F53008F443C0D8
:10F33000C301B20122E030E040E050E00E94AFDAC9
:10F34000AE89BF8950962D933D934D935C9353970F
:10F3500088279927DC01821B930BA40BB50BEE8940
:10F36000FF8984879587A687B78737C040E050E03C
:10F37000BA01C5018C5D9D4F0E94A6A00E94E0D8F5
:10F38000AE89BF8912962D913D914D915C91159753
:10F390000E94E6D90E94AFD8461A570A680A790A2D
:10F3A000EE89FF89408A518A628A738A148615869B
:10F3B0001686178612C0EE89FF89208B318B428B0F
:10F3C000538B7094609450944094411C511C611C68
:10F3D000711C4486558666867786D8011C96ED9109
:10F3E000FC911D972081C701AF81B8850C9002C0A8
:10F3F000880F991F0A94E2F7282B2083D8011596CD
:10F40000ED91FC9116972081C701A985BA850C90D2
:10F4100002C0880F991F0A94E2F7282B2083D80195
:10F420001E96ED91FC911F972081C701AC81BD8193
:10F430000C9002C0880F991F0A94E2F7282B2083B2
:10F44000D8015396ED91FC9154972081C701AC816E
:10F45000BD810C9002C0880F991F0A94E2F7282BF7
:10F460002083F801848D958D892B81F101A0F2A173
:10F47000E02D2081C701D1010C9002C0880F991F97
:10F480000A94E2F7809582238083EE89FF89808148
:10F49000D8015C96ED91FC915D972081882359F00D
:10F4A000C701D1010C9002C0880F991F0A94E2F79E
:10F4B000282B20830BC0C701D1010C9002C0880FFC
:10F4C000991F0A94E2F7809582238083F801858949
:10F4D0009689892B81F1028CF38DE02D2081C70163
:10F4E000D4010C9002C0880F991F0A94E2F780950E
:10F4F00082238083EE89FF898081D8015596ED9122
:10F50000FC9156972081882359F0C701D4010C90B3
:10F5100002C0880F991F0A94E2F7282B20830BC0A2
:10F52000C701D4010C9002C0880F991F0A94E2F71A
:10F53000809582238083F601EE0FFF1FEE0FFF1FE1
:10F54000E25FF94E1082118212821382EF85F889F0
:10F5500012861386F601E75FF94E1082EA81FB817D
:10F56000EE5DF94E81E09981933008F480E0818F5F
:10F57000AE89BF895D961D921D921D921C92909737
:10F58000B1E0B28F138E148AEE89FF89158A168A2C
:10F59000178A108EDF0111A212A213A214A215A2C3
:10F5A00016A217A210A6FFEFCF1ADF0A8A819B814D
:10F5B00089969B838A839996BF8BAE8B0D5D1F4F77
:10F5C000B3E28B0E911CEF81F885B396F887EF8339
:10F5D00089859A8583969A878987AC81BD81939620
:10F5E000BD83AC83B3E22B0E311CE4E0AE0EB11C44
:10F5F0008B859C8502969C878B87AD85BE851296F0
:10F60000BE87AD87B5E0CB16D10409F00DCEE989F0
:10F61000EE2321F010920416109203161092061693
:10F6200010920516109208161092071667960FB6DC
:10F63000F894DEBF0FBECDBFDF91CF911F910F9128
:10F64000FF90EF90DF90CF90BF90AF909F908F9002
:10F650007F906F905F904F903F902F90089599E228
:10F66000899FF0011124EE5DF94EDF01129652815F
:10F6700011964C91119712963C91129713962C91DA
:10F68000652F742F832F922F0895CF93DF931F92AE
:10F69000CDB7DEB749830E94E2D8498129E2429F73
:10F6A000F0011124EE5DF94E2281338144815581B0
:10F6B0000E940DD80F90DF91CF9108954F925F92E5
:10F6C0006F927F928F929F92AF92BF92CF92DF9272
:10F6D000EF92FF920F931F93CF93DF93142F20E0AD
:10F6E00030E04AE754E40E94E6D90E9475D8290127
:10F6F0003A014B01D82FC92F89E2189FF00111243C
:10F70000EE5DF94E62817381848195810E9475D886
:10F7100059016A017B018C019201A301B4018D2F73
:10F720009C2F0E942EDBE8EEAE2EF3E0BF2EC12C04
:10F73000D12CE12CF12C00E010E00E94F1DA952FA1
:10F74000B901842FDF91CF911F910F91FF90EF901E
:10F75000DF90CF90BF90AF909F908F907F906F90F1
:10F760005F904F90089540E065E87AE18FEE96E172
:10F770000C941DD31F93CF93DF93C0E0D0E01BE028
:10F780001C9FC0011D9F900D11246C2F865C984E0C
:10F790000E94E79F2196C530D10591F7DF91CF9167
:10F7A0001F91089580913917811103C080913817F6
:10F7B000089581E008956F927F929F92AF92BF92D9
:10F7C000CF92DF92EF92FF920F931F93CF93DF932D
:10F7D00000D000D0CDB7DEB79FB6F89408E312E0B2
:10F7E000612C712C40E050E0BA01C8010E94A6A033
:10F7F0006B017C01862D0E942F7B9B01AC01B30124
:10F8000088EF96E129833A834B835C830E94074FFC
:10F810005C01C701B6010E94E2D829813A814B817F
:10F820005C810E94E6D920E030E04AE754E40E947F
:10F830000DD80E94AFD8F5016083718382839383D2
:10F84000FFEF6F1A7F0A0C5F1F4F83E06816710489
:10F8500049F602E010E0B80188EF96E10E94074FF8
:10F86000FC0110821182128213820F5F1F4F05303C
:10F87000110589F700E010E0B8018CE097E10E94E3
:10F88000074FFC0110821182128213820F5F1F4FFB
:10F890000530110589F79FBE0F900F900F900F90C4
:10F8A000DF91CF911F910F91FF90EF90DF90CF905C
:10F8B000BF90AF909F907F906F90089510923917EE
:10F8C0001092381781E00E94AB780E94BA7B4FEF0C
:10F8D0005FEFBA0188E392E00E94A6A06F3F7F4FDE
:10F8E0008F4F9F4F11F40C94E93608957F928F92B9
:10F8F0009F92AF92BF92CF92DF92EF92FF920F93BF
:10F900001F93CF93DF93CDB7DEB764970FB6F8940C
:10F91000DEBF0FBECDBF44E1FC019E012F5F3F4F14
:10F92000D90101900D924A95E1F78DE2E82E86E12A
:10F93000F82E00E010E077247394D22EC32EF70146
:10F940007082B8018091F6169091F7160E94074FC9
:10F95000FC0180809180A280B380B8018D2D9C2D08
:10F960000E94074FFC014081518162817381480DE3
:10F97000591D6A1D7B1D40835183628373830F5F12
:10F980001F4FF9E2EF0EF11C05301105C1F664E0DE
:10F9900070E08D2D9C2D0E94074F8C0163E070E07C
:10F9A0008D2D9C2D0E94074F4C0162E070E08D2D43
:10F9B0009C2D0E94074F5C0161E070E08D2D9C2D15
:10F9C0000E94074F7C0160E070E08D2D9C2D0E940D
:10F9D000074F9401A501B7010E94467864960FB6BF
:10F9E000F894DEBF0FBECDBFDF91CF911F910F9175
:10F9F000FF90EF90DF90CF90BF90AF909F908F904F
:10FA00007F900895AF92BF92CF92DF92EF92FF92D4
:10FA10000F931F93CF93DF93CDB7DEB764970FB6E5
:10FA2000F894DEBF0FBECDBF24E1FC01DE011196CC
:10FA300001900D922A95E1F781E080932D16809335
:10FA4000561680937F168093A8168093D11664E093
:10FA500070E0CE0101960E94074F8C0163E070E0D8
:10FA6000CE0101960E94074F5C0162E070E0CE017A
:10FA700001960E94074F6C0161E070E0CE01019693
:10FA80000E94074F7C0160E070E0CE0101960E9469
:10FA9000074F9501A601B7010E94467864960FB6FC
:10FAA000F894DEBF0FBECDBFDF91CF911F910F91B4
:10FAB000FF90EF90DF90CF90BF90AF9008955F924E
:10FAC0006F927F928F929F92AF92BF92CF92DF926E
:10FAD000EF92FF920F931F93CF93DF93CDB7DEB7D3
:10FAE00064970FB6F894DEBF0FBECDBF3C010E94F5
:10FAF000CA4E5FB6F89480903C1590903D15A0904A
:10FB00003E15B0903F15C0903815D0903915E09053
:10FB10003A15F0903B150091341510913515209150
:10FB2000361530913715409130155091311560914F
:10FB3000321570913315809143158F938091421542
:10FB40008F93809141158F93809140158F93CE01B3
:10FB500001960E94CB4E84E1FE013196D3010190C3
:10FB60000D928A95E1F70F900F900F900F9000E0A3
:10FB700010E0B8018091F6169091F7160E94074F99
:10FB8000FC01C080D180E280F380B801C3010E94F3
:10FB9000074FFC0140815181628173814C195D09DD
:10FBA0006E097F0940835183628373830F5F1F4F08
:10FBB00005301105F1F65FBEC30164960FB6F894E7
:10FBC000DEBF0FBECDBFDF91CF911F910F91FF9090
:10FBD000EF90DF90CF90BF90AF909F908F907F90ED
:10FBE0006F905F9008956F927F928F929F92AF92E5
:10FBF000BF92CF92DF92EF92FF920F931F93CF931A
:10FC0000DF93CDB7DEB765970FB6F894DEBF0FBEB2
:10FC1000CDBF3C0145E1E42EF12CEC0EFD1E8E0122
:10FC20000F5E1F4F9E01235F3F4FAE01475F5F4F47
:10FC3000BE016B5F7F4FCE0101960E9431668D89B8
:10FC400081708D8B813029F438EFC32E36E1D32EAD
:10FC500004C02CE0C22E27E1D22EEE24E394F12C36
:10FC6000EC0EFD1E00E010E0B801C6010E94074F37
:10FC7000F7014081518162817381FC018081918112
:10FC8000A281B381481B590B6A0B7B0BF70141938F
:10FC90005193619371937F010F5F1F4F05301105E1
:10FCA00019F78D849E84AF84B888C984DA84EB8484
:10FCB000FC840D811E812F81388549815A816B8199
:10FCC0007C818C898F938B898F938A898F93898983
:10FCD0008F93C3010E94CB4E0F900F900F900F9007
:10FCE000C30165960FB6F894DEBF0FBECDBFDF919E
:10FCF000CF911F910F91FF90EF90DF90CF90BF9029
:10FD0000AF909F908F907F906F900895809322176F
:10FD100008954F925F926F927F928F929F92AF92CF
:10FD2000BF92CF92DF92EF92FF920F931F93CF93E8
:10FD3000DF93CDB7DEB728970FB6F894DEBF0FBEBE
:10FD4000CDBF6C019A01AB010CE115E17801A12C4A
:10FD5000B12CB501C6012D833E834F8358870E9485
:10FD6000FF4EFC014080518062807380B50180911C
:10FD7000F6169091F7160E94074FFC018081918141
:10FD8000A281B381840D951DA61DB71DF701819336
:10FD90009193A193B1937F01FFEFAF1ABF0A2D8119
:10FDA0003E814F81588585E0A816B10491F6C09038
:10FDB0002415D0902515E0902615F09027158091F8
:10FDC000841690918516A0918616B0918716C81654
:10FDD000D906EA06FB0614F4D701C6018093241560
:10FDE00090932515A0932615B093271560E3862ED2
:10FDF00065E1962E62E675E1B12CA12CC12CD12CC7
:10FE00007601F80181919191A191B1918F01F40155
:10FE100041905190619071904F0184199509A60904
:10FE2000B709B7FF07C0B095A095909581959F4FF2
:10FE3000AF4FBF4FFB0181939193A193B193BF014A
:10FE4000C816D906EA06FB061CF4AB2C6C017D0132
:10FE5000B394F5E0BF12D5CFA0927615C092771576
:10FE6000D0927815E0927915F0927A15CD28CE28A7
:10FE7000CF2839F160E472E48FE090E00E94AFDABD
:10FE800029833A834B835C83E090F51600E025EFED
:10FE900036E1AE014F5F5F4F60E070E0CB010E9442
:10FEA000B66E8091AA0D9091A90D891B8F709091CB
:10FEB0003717891720F081E08093391702C010921C
:10FEC000391728960FB6F894DEBF0FBECDBFDF916D
:10FED000CF911F910F91FF90EF90DF90CF90BF9047
:10FEE000AF909F908F907F906F905F904F9008950C
:10FEF0002F923F924F925F926F927F928F929F923A
:10FF0000AF92BF92CF92DF92EF92FF920F931F9327
:10FF1000CF93DF93CDB7DEB72A970FB6F894DEBF45
:10FF20000FBECDBF5C014F83588769877A8770E326
:10FF3000272E75E1372E8CE195E19E838D837C0120
:10FF4000610100E010E0822E912CC401002E02C05D
:10FF5000959587950A94E2F780FF0AC0F6014080E4
:10FF6000518062807380B801C5010E94FF4E10C0AD
:10FF7000B801C5010E94FF4EFC01408051806280A3
:10FF80007380B8018091F6169091F7160E94074F82
:10FF9000FC0180819181A281B381840D951DA61DF4
:10FFA000B71DF70180839183A283B3830F5F1F4F37
:10FFB000F4E0CF0ED11C84E0E80EF11C05301105F1
:10FFC00021F64091241550912515609126157091C8
:10FFD00027158091841690918516A0918616B09170
:10FFE0008716481759076A077B0714F4DB01CA0113
:10FFF0008093241590932515A0932615B09327156B
:020000021000EC
:1000000002E615E160E070E020E030E0A901ED815A
:10001000FE8181919191A191B191FE83ED83F101D6
:10002000C190D190E190F1901F018C199D09AE090A
:10003000BF09B7FF07C0B095A095909581959F4FD8
:10004000AF4FBF4FF80181939193A193B1938F016B
:10005000281739074A075B071CF4762F9C01AD016E
:100060006F5F6530A1F67093761520937715309306
:1000700078154093791550937A152115310541056E
:10008000510569F16F81788589859A850E94AFDA7B
:1000900060E472E48FE090E00E94AFDA29833A8353
:1000A0004B835C83E090F51600E025EF36E1AE016E
:1000B0004F5F5F4F60E070E0CB010E94B66E8091B1
:1000C000AA0D9091A90D891B8F70909137178917F0
:1000D00020F081E08093391702C0109239172A96D8
:1000E0000FB6F894DEBF0FBECDBFDF91CF911F9149
:1000F0000F91FF90EF90DF90CF90BF90AF909F90C7
:100100008F907F906F905F904F903F902F900895C9
:100110002F923F924F925F926F927F928F929F9217
:10012000AF92BF92CF92DF92EF92FF920F931F9305
:10013000CF93DF93CDB7DEB766970FB6F894DEBFE7
:100140000FBECDBF1C014D875E876F87788B47013F
:100150005801DA8AC98A40E355E15C874B878CE114
:1001600095E19A8789873C012A0100E010E0422F3F
:1001700050E05E834D838D819E81002E02C0959557
:1001800087950A94E2F780FF0AC0F201C080D1800F
:10019000E280F380B801C1010E94FF4E10C0B80197
:1001A000C1010E94FF4EFC01C080D180E280F3803B
:1001B000B8018091F6169091F7160E94074FFC0146
:1001C00080819181A281B3818C0D9D1DAE1DBF1DCB
:1001D000F30180839183A283B3830F5F1F4FF4E009
:1001E0004F0E511C24E0620E711C0530110519F6EA
:1001F0004091241550912515609126157091271571
:100200008091841690918516A0918616B0918716DC
:10021000481759076A077B0714F4DB01CA0180936A
:10022000241590932515A0932615B09327151092A9
:100230007615A2E62A2EA5E13A2E43E257E1588729
:100240004F830FE715E11D82412C512C3201E985C6
:10025000FA856191719181919191FA87E987EB8596
:10026000FC85C190D190E190F190FC87EB876C19EF
:100270007D098E099F09F1016083718382839383D5
:100280006B017C0197FF07C0CC24DD247601C61AE0
:10029000D70AE80AF90AC114F0E8DF06E104F1041C
:1002A00064F4EF81F8852081318142815381CB0153
:1002B000772766270E947AD624C00E94E2D86B8BEB
:1002C0007C8B8D8B9E8BEF81F88560817181828123
:1002D00093810E94E2D820E030E040E857E30E949A
:1002E000E6D99B01AC016B897C898D899E890E942E
:1002F000E6D920E030E040E857E40E94E6D90E94C9
:10030000AFD8F8016083718382839383F101C08247
:10031000D182E282F3824C145D046E047F042CF4DB
:10032000FD81F09376152601370124E0220E311C61
:100330003D813F5F3D834F8158854C5F5F4F5887BC
:100340004F830C5F1F4F353009F081CF40927715F6
:10035000509278156092791570927A154528462842
:10036000472809F459C020E030E0A901C501B401D3
:100370000E9409D8882309F44FC020E030E040E80B
:1003800057E4C501B4010E94E6D90E94AFD860933A
:100390007B1570937C1580937D1590937E1520912D
:1003A000B602222379F0E989FA89BF01882777FD0F
:1003B0008095982FEAE0660F771F881F991FEA95AE
:1003C000D1F703C060E070E0CB01E090F516222386
:1003D00019F00091B70201C000E02D853E854F85E0
:1003E000588929833A834B835C8325EF36E1AE013C
:1003F0004F5F5F4F0E94B66E8091AA0D9091A90D3C
:10040000891B8F7090913717891720F081E08093B6
:10041000391702C01092391766960FB6F894DEBFEE
:100420000FBECDBFDF91CF911F910F91FF90EF9045
:10043000DF90CF90BF90AF909F908F907F906F9004
:100440005F904F903F902F9008952F923F924F9240
:100450005F926F927F929F92AF92BF92CF92DF9204
:10046000EF92FF920F931F93CF93DF93CDB7DEB739
:1004700068970FB6F894DEBF0FBECDBF982EA62E9C
:100480001092B7028E010F5F1F4FC8012D8B3E8B5C
:100490004F8B588F0E94F37D8CE2C82E86E1D82EB8
:1004A000E12CF12CB12C302E212E11E0588D4F89EA
:1004B0003E892D89C5010E2C02C0959587950A9419
:1004C000E2F780FD05C0F701E75FF94E10822BC00F
:1004D000B701832D922D2D8B3E8B4F8B588F0E9411
:1004E000074F2D893E894F89588D992039F0442432
:1004F0004A94542C642C0FE3702E05C0412C512CCF
:10050000612CB0EC7B2EFC014082518262827382AE
:10051000F701E75FF94E1083F2E0EF1202C010938B
:100520002117F6011083FFEFEF1AFF0A89E2C80EC8
:10053000D11CE5E0EE16F10409F0BCCFBA01A90127
:10054000CE0101960E94897E81E0809338176896DB
:100550000FB6F894DEBF0FBECDBFDF91CF911F91D4
:100560000F91FF90EF90DF90CF90BF90AF909F9052
:100570007F906F905F904F903F902F9008958530BF
:1005800098F49091041621E030E0082E01C0220F6B
:100590000A94EAF7662321F0922B909304160895AB
:1005A0002095292320930416089580910416089518
:1005B000853040F42BE0829FC0011124865C984E68
:1005C0000C94EC9F08958093B702089581708093F6
:1005D000F516813019F488EF96E102C08CE097E1BE
:1005E0009093F7168093F616089580916902909182
:1005F0006A02892B99F0E0916B02F0916C02808184
:1006000090E000906D0202C0959587950A94E2F7FC
:10061000817091E020917416821301C090E0892FBF
:1006200090E0E5E0880F991FEA95E1F720916202DA
:1006300030916302232B99F0E0916402F0916502FE
:10064000208130E00090660202C0359527950A941B
:10065000E2F7217031E040917416241301C030E0BC
:10066000232F30E074E0220F331F7A95E1F7282B17
:10067000392B8091460290914702892B99F0E091A5
:100680004802F0914902808190E000904A0202C045
:10069000959587950A94E2F7817091E040914B1609
:1006A000841301C090E0892F90E063E0880F991FC8
:1006B0006A95E1F7822B932B20913F023091400203
:1006C000232B99F0E0914102F0914202208130E029
:1006D0000090430202C0359527950A94E2F72170F5
:1006E00031E040914B16241301C030E0232F30E05D
:1006F000220F331F220F331F282B392B8091230207
:1007000090912402892B99F0E0912502F091260224
:10071000808190E00090270202C0959587950A9409
:10072000E2F7817091E040912216841301C090E0BD
:10073000892F90E0880F991F822B932B20911C0208
:1007400030911D02232B99F0E0911E02F0911F02BF
:10075000208130E00090200202C0359527950A9450
:10076000E2F7217031E040912216241301C030E0FD
:10077000832B08959091B602911101C080E00C94F2
:1007800006670E948F66109239171092381780E022
:100790000E94AB788091B6028093B70281E00C94FE
:1007A000BA832F923F924F925F927F928F929F9245
:1007B000AF92BF92CF92DF92EF92FF920F931F936F
:1007C000CF93DF9380E00E94AB780E94BA7B1092B7
:1007D0002017109221170E94DB7B80E00E94E682A6
:1007E0006FEF88E891E00E9466A0803811F00E94C7
:1007F000013560E08EE691E00E9466A081708093F2
:10080000B6028093B70281E00E94BA83C3E2D7E1C7
:1008100010E0812F0E942F7B9B01AC0160E070E013
:1008200080E89FE30E940DD820E030E040E857E4E4
:100830000E94E6D90E94AFD86993799389939993DE
:100840001F5F153031F768EE73E082E791E00E9498
:1008500083A0A0E0B0E08093D5159093D615A09327
:10086000D715B093D81568EE73E084E791E00E9445
:1008700083A0A0E0B0E08093D9159093DA15A093FF
:10088000DB15B093DC1566E970E086E791E00E9425
:1008900083A0A0E0B0E08093DD159093DE15A093D7
:1008A000DF15B093E01560EA7FE088E791E00E94F1
:1008B00083A0A0E0B0E08093E1159093E215A093AF
:1008C000E315B093E41560EA7FE08AE791E00E94C7
:1008D00083A0A0E0B0E08093E5159093E615A09387
:1008E000E715B093E815C5EDD5E1ABE9EA2EA5E132
:1008F000FA2E0AE415E1712C88248A94982C54016C
:100900006E01288039804A805B80872D0E942F7B72
:100910009B01AC0160EF7FEF8FE799E40E940DD857
:100920000E94B4D8621573058405950588F4872D57
:100930000E942F7B9B01AC0160EF7FEF8FE799E472
:100940000E940DD80E94B4D8688379838A839B83E0
:100950002496F60160817181828193810E94E0D8A2
:100960001B012C01872D0E942F7B9B01AC01C20132
:10097000B1010E94E6D90E94B4D89B01AC01F701F5
:1009800061937193819391937F01C501B4010E949A
:100990008DDAF80121933193419351938F01739430
:1009A000F5E07F12ADCF60ED77E080E791E00E9447
:1009B00083A0A0E0B0E0813127E29207A105B10554
:1009C00008F404C080E197E2A0E0B0E08093D11584
:1009D0009093D215A093D315B093D41560EA7FE01D
:1009E00086E891E00E9483A0A0E0B0E08131E7E2D8
:1009F0009E07A105B10508F404C080E197E2A0E0DC
:100A0000B0E08093CD159093CE15A093CF15B09301
:100A1000D01560E070E080EE91E00E9483A090939A
:100A20007D0D80937C0D60E070E082EE91E00E948D
:100A300083A090937F0D80937E0D6AE070E08CE739
:100A400091E00E9483A0BC0180E090E00E94E0D889
:100A500020E030E040E857E40E94E6D90E94AFD899
:100A60006093B5157093B6158093B7159093B8152C
:100A70006AE070E08EE791E00E9483A0BC0180E014
:100A800090E00E94E0D820E030E040E857E40E9487
:100A9000E6D90E94AFD86093B9157093BA158093C8
:100AA000BB159093BC156AE070E080E891E00E946D
:100AB00083A0BC0180E090E00E94E0D820E030E01C
:100AC00040E857E40E94E6D90E94AFD86093BD1574
:100AD0007093BE158093BF159093C0156EE170E0C2
:100AE00082E891E00E9483A0BC0180E090E00E9437
:100AF000E0D820E030E040E857E40E94E6D90E94C8
:100B0000AFD86093C1157093C2158093C3159093AD
:100B1000C4156EE170E084E891E00E9483A0BC01FE
:100B200080E090E00E94E0D820E030E040E857E428
:100B30000E94E6D90E94AFD86093C5157093C61580
:100B40008093C7159093C8158091BD159091BE15DF
:100B5000A091BF15B091C015E5EBF5E14191519120
:100B600061917191481759076A077B0714F4DB01FB
:100B7000CA0125E1E93CF20789F78093C9159093F2
:100B8000CA15A093CB15B093CC1542E553E060E0B5
:100B900070E088ED91E00E94A6A00E94E0D820E0DD
:100BA00030E543EC57E40E940DD820E030E040E807
:100BB00057E40E94E6D90E94AFD87B01D82FC92FF5
:100BC00044E853E060E070E08CED91E00E94A6A064
:100BD0000E94E0D820E030E543EC57E40E940DD8B5
:100BE00020E030E040E857E40E94E6D90E94AFD808
:100BF000B62EA72E6C018EE195E0A0E0B0E08093C8
:100C0000441590934515A0934615B093471580E081
:100C100090E0A2E0B0E08093B1159093B215A0935C
:100C2000B315B093B41561E084EE91E00E9466A024
:100C3000882309F184E090E09093B0158093AF157C
:100C40000E94885081110AC08091AF159091B01513
:100C5000880F991F9093B0158093AF158091AF15B1
:100C60009091B01509975CF088E090E09093B015F2
:100C70008093AF1504C01092B0151092AF1581E0AB
:100C800080937A0D80937B0D0091A3161091A4168A
:100C90002091A5163091A6160093720D1093730D36
:100CA0002093740D3093750D0091CC161091CD16D4
:100CB0002091CE163091CF160093760D1093770DBC
:100CC0002093780D3093790D8FE080933717009142
:100CD00022172B2D3A2DA601B7018D2F9C2F0E9494
:100CE000726EDF91CF911F910F91FF90EF90DF9087
:100CF000CF90BF90AF909F908F907F905F904F90DC
:100D00003F902F900C9438650E948A538111109265
:100D1000391780913817882361F110923817809124
:100D2000091690913817892B8093381780910A16ED
:100D300090913817892B8093381780910B169091DA
:100D40003817892B8093381780913817811111C07B
:100D50000E948F6680912117882339F08091201797
:100D60008F5F80932017109221178091B602809395
:100D7000B70208950C94FA63809120170895CF93D9
:100D8000DF9300D000D000D0CDB7DEB740E065E8FB
:100D90007AE181E797E10E941DD345E065E97AE1B8
:100DA000CE0101960E941DD34FE853E0BE016F5F54
:100DB0007F4F8AE397E10E94739F46E067E87AE1FC
:100DC000CE0101960E941DD34FE853E0BE016F5F34
:100DD0007F4F85E497E10E94739F43E067E87AE1E3
:100DE000CE0101960E941DD34FE853E0BE016F5F14
:100DF0007F4F80E597E10E94739F44E06BE97AE1C1
:100E0000CE0101960E941DD34FE853E0BE016F5FF3
:100E10007F4F8BE597E10E94739F47E06BE87AE193
:100E2000CE0101960E941DD34FE853E0BE016F5FD3
:100E30007F4F86E697E10E94739F8CE097E10E94C6
:100E4000CA4E88EF96E10E94CA4E26960FB6F894D5
:100E5000DEBF0FBECDBFDF91CF91089594EA90938E
:100E6000BC009091BC0097FFFCCF9091B900987F97
:100E7000983061F58093BB0084E88093BC0080913A
:100E8000BC0087FFFCCF8091B900887F883101F5D5
:100E9000CB01FB0150E064E80EC021912093BB0020
:100EA0006093BC002091BC0027FFFCCF2091B900CB
:100EB000287F283279F49F01281B390B2417350726
:100EC00064F384E98093BC0080E0089581E0089594
:100ED00082E0089583E008951092B90080E2809343
:100EE000B800089580917E17089510927E1781E0D2
:100EF00080937717089581E040917C1750917D177A
:100F000020917A1730917B17421753070CF080E03D
:100F1000089580917C1790917D1720917A173091D8
:100F20007B17821793076CF4E0917817F09179178B
:100F3000E80FF91F019690937D1780937C17849199
:100F4000089580E00895809177170895CF93C82F72
:100F500081E080937E1710927D1710927C1710927B
:100F60007717C13039F018F0C23009F516C02DE0FE
:100F700030E106C00E94C335882339F02CE630E109
:100F8000309379172093781716C082EA98E19093EE
:100F9000791780937817C2E00EC08093771788ED99
:100FA00090E29093791780937817C3E004C0109271
:100FB0007E1780E00EC0EC2FF0E0EE0FFF1FE9522D
:100FC000FE4C8591949180937A1790937B17809132
:100FD0007E17CF91089510927E1781E08093771746
:100FE000089540E065E87AE18FE797E10C941DD31E
:100FF000CF93DF9300D000D000D0CDB7DEB71092F2
:1010000086171092871740E251EA67E070E0FC0112
:1010100040A351A362A373A3E4E0F1E08081877849
:101020008083E5E0F1E080818778808342E06FE8AB
:101030007AE1CE0101960E941DD360E0CE010196B7
:101040000E944CD326960FB6F894DEBF0FBECDBFDC
:10105000DF91CF9108957F928F929F92AF92BF922E
:10106000CF92DF92EF92FF920F931F93CF93DF9374
:10107000CDB7DEB72F970FB6F894DEBF0FBECDBF4A
:101080008C01FC0181818111A9C0F090030198E7D6
:10109000892E8F2092B2F4E09F22809187178925B4
:1010A000909186179825892B51F080E291EAA7E06C
:1010B000B0E0F80180A391A3A2A3B3A30CC0F801F0
:1010C0008281882309F480C0C80102960E94F8D466
:1010D00081117AC083C06801F2E0CF0ED11CC60135
:1010E0000E9427D5F3FC10C08091851781111BC089
:1010F00040E856E968E970E0C80141960E94D4D4FE
:1011000081E0809385170FC0CE0101960E94D0D454
:101110008FE0FE013196D801519601900D928A958B
:10112000E1F710928517780181E1E80EF11CC70103
:101130000E94F8D4882389F0F801108281E081832D
:10114000CE0101960E94D0D48FE0FE013196D701E6
:1011500001900D928A95E1F741C091100CC082E098
:10116000F801808381E0818340A151A162A173A134
:10117000C6010E94D4D483E0E82EF12CA82CB12C17
:1011800077247394C5010E2C02C0959587950A9417
:10119000E2F780FD0DC0F8018181811109C0E08274
:1011A000718240A151A162A173A1C6010E94D4D451
:1011B000FFEFEF1AFF0A87E0E816F10419F79092A3
:1011C0008717809286170AC040EA56E861E070E00F
:1011D000F80140A351A362A373A37DCF2F960FB64E
:1011E000F894DEBF0FBECDBFDF91CF911F910F915D
:1011F000FF90EF90DF90CF90BF90AF909F908F9037
:101200007F900895FC01F8948181908111827894F7
:10121000882319F0FB01908311820895FC0140A3FB
:1012200051A362A373A3089540E065E87AE188E8DA
:1012300097E10C941DD32F923F924F925F926F9241
:101240007F928F929F92AF92CF92DF92EF92FF9216
:101250000F931F93CF93DF93EC01D62E1A01290130
:10126000602F47010E94ED8B85E993E09E838D837B
:10127000DF823E0188E0680E711C8AE0E80EF11CF6
:10128000AE014B5F5F4FAD2CCC24C39400E910ED51
:1012900023E030E0BE01C3010E944EA2B101CE01A5
:1012A0008E579F4F0E9434D3FE01E857FF4FD082E4
:1012B000A401465E5F4F9201B301CE0187579F4F55
:1012C0000E94569FC356DF4F99828882DF91CF914B
:1012D0001F910F91FF90EF90DF90CF90AF909F9074
:1012E0008F907F906F905F904F903F902F900895D8
:1012F0000F931F93CF93DF93EC018C010E571F4F79
:1013000060E0C8010E946CD361E0C8010E944CD328
:10131000CE0108960E945AA1CE010E94CC8BCE012C
:1013200087579F4FDF91CF911F910F910C94299F69
:10133000CF93DF93EC0108960E944CA5CE0187570E
:101340009F4FDF91CF910C94E69E87579F4F61117D
:101350000C94DA9E0C94259F882321F080919000B4
:10136000806803C0809190008F73809390000895EF
:10137000882321F080919000886003C080919000C4
:10138000837F8093900008950F931F93CF93DF93F3
:1013900000D000D000D0CDB7DEB7162F0FB7F8942D
:1013A000FC018281811112C0862F81508E3F28F06E
:1013B00080E00E94B88945E013C070E070939D0002
:1013C00060939C0080919000886021C0813009F575
:1013D000862F81508E3F98F080E00E94AC8943E0D8
:1013E00063E97AE1CE0101960E941DD361E01F3FBF
:1013F00009F060E0CE0101960E946CD30AC070E053
:101400007093990060939800809190008068809319
:1014100090000FBF26960FB6F894DEBF0FBECDBF6B
:10142000DF91CF911F910F91089540E065E87AE137
:101430008EE897E10C941DD30F931F93CF93DF9306
:1014400000D000D000D0CDB7DEB7062F142F94E027
:101450009D838E8342E0BE016B5F7F4F84EC0E94D0
:101460002E8787EC90E00197F1F700C0000083E041
:101470008B830C8342E0BE016D5F7F4F84EC0E9442
:101480002E8787EC90E00197F1F700C0000082E022
:1014900089831A8342E0BE016F5F7F4F84EC0E9414
:1014A0002E8726960FB6F894DEBF0FBECDBFDF9114
:1014B000CF911F910F9108951F93CF93DF93C82F62
:1014C000D62F142F0E94BA3421E0412F6D2F8C2F7C
:1014D000DF91CF911F910C941C8A8F929F92AF92B3
:1014E000BF92CF92DF92EF92FF92CF9361E080E4C0
:1014F00091E00E9466A0C82F4FEF5FEFBA0184E42D
:1015000091E00E94A6A06B017C01C430F1F048F488
:10151000C130B1F070F0C230E1F0C33009F041C029
:101520001CC0C630F9F048F0C73061F1C830C9F5C9
:101530001EC021E04FEF6FEF06C021E04FEF24C047
:1015400021E040E060E08FEF21C021E040E06FEF5C
:101550001CC021E040E062E308C021E046E460E016
:1015600086E414C021E048EC60E088EC0FC08D2CCC
:101570009E2CAF2CBB24B7018827992721E0482D4A
:101580008F2D04C021E040E060E080E0CF91FF902B
:10159000EF90DF90CF90BF90AF909F908F900C9482
:1015A0001C8ACF91FF90EF90DF90CF90BF90AF90CB
:1015B0009F908F9008951F93CF93DF93CDB7DEB7A1
:1015C00028970FB6F894DEBF0FBECDBF182F81E06D
:1015D0008F831123E1F184E3888742E0BE01695FD4
:1015E0007F4F84EC0E942E8787EC90E00197F1F703
:1015F00000C0000088E08D838FE38E8342E0BE014F
:101600006B5F7F4F84EC0E942E8787EC90E0019700
:10161000F1F700C0000086E08B8380E88C8342E015
:10162000BE016D5F7F4F84EC0E942E8787EC90E0B7
:101630000197F1F700C0000087E089831A8342E038
:10164000BE016F5F7F4F84EC0E942E8744C084E10F
:10165000888742E0BE01695F7F4F84EC0E942E873D
:1016600087EC90E00197F1F700C0000088E08D83DF
:101670008AE28E8342E0BE016B5F7F4F84EC0E9462
:101680002E8787EC90E00197F1F700C000001C82E4
:101690001B8286E08B8342E0BE016D5F7F4F84EC4E
:1016A0000E942E8787EC90E00197F1F700C00000C0
:1016B0001A82198287E0898342E0BE016F5F7F4F03
:1016C00084EC0E942E8787EC90E00197F1F700C030
:1016D00000000E946D8A28960FB6F894DEBF0FBEF8
:1016E000CDBFDF91CF911F9108951F93CF93DF93CB
:1016F00000D000D000D0CDB7DEB70E946C871D822D
:1017000011E01E8342E0BE016B5F7F4F84EC0E94BC
:101710002E8787EC90E00197F1F700C000001B8353
:1017200084E18C8342E0BE016D5F7F4F84EC0E94B8
:101730002E8787EC90E00197F1F700C0000088E069
:1017400089838AEA8A8342E0BE016F5F7F4F84EC1F
:101750000E942E8787EC90E00197F1F700C000000F
:101760000E946D8A26960FB6F894DEBF0FBECDBFDD
:10177000DF91CF911F91089521E040E060E08FEF6D
:101780000E941C8A8CE00C94DB8A40E065E87AE1D8
:1017900084E997E10C941DD3FC0113821282089511
:1017A0000F931F93CF93DF9300D0CDB7DEB78C019B
:1017B000AE014F5F5F4FFC01648189E099E00E94B8
:1017C000BC8C29813A81F801338322830F900F90DA
:1017D000DF91CF911F910F9108952BE933E0FC0128
:1017E000318320836483089540E065E87AE18AE9E3
:1017F00097E10C941DD3AF92BF92CF92DF92EF92FC
:10180000FF920F931F93CF93DF93EC017B016A014B
:101810005901B8010E9434D3B601CE0106960E9448
:1018200034D3B701CE010C960E9434D3B501CE015A
:101830004296DF91CF911F910F91FF90EF90DF9033
:10184000CF90BF90AF900C9434D3AF92BF92CF9211
:10185000DF92EF92FF920F931F93CF93DF93EC01F0
:101860008C010A5F1F4F60E0C8010E946CD31A8E82
:101870001B8E88E78C8FEBA0FCA0FCA6EBA6B0E14A
:10188000CB2ED12C5E018CE0A80EB11C6E2D6170A8
:10189000C5010E946CD3F694E79461E0C8010E94F0
:1018A0006CD360E0C8010E946CD381E0C81AD108F3
:1018B00069F7F0E1EF2EF12C629660E0C5010E941D
:1018C0006CD361E0C8010E946CD3CE010E945FD34B
:1018D00060E0C8010E946CD381E0E81AF10869F762
:1018E00060E0C801DF91CF911F910F91FF90EF90C1
:1018F000DF90CF90BF90AF900C946CD30F931F9359
:10190000CF93DF93EC0161E00C960E944CD38E01E3
:101910000A5F1F4F61E0C8010E944CD360E0CE0116
:1019200042960E944CD361E0CE010E944CD380E3EA
:1019300096E49CA38BA38CE396E49EA38DA380E006
:101940009EE498A78FA318A21F8E1AA219A21E8E1A
:101950001D8E60E0CE010E946CD360E0C8010E9441
:101960006CD31AA619A6198E188ECE01DF91CF91CD
:101970001F910F910C94258CFC01611103C0878D80
:1019800090A102C081A192A1DA018D939C93808DD8
:10199000918D08954F925F926F927F928F929F9256
:1019A000AF92BF92CF92DF92EF92FF920F931F936D
:1019B000CF93DF93EC017C0186E0E80EF11C60E040
:1019C000C7010E946CD35E0182E1A80EB11CC50163
:1019D0000E945FD38111B3C08A8D813039F018F035
:1019E000823051F406C0CBA0DCA008C0CDA0DEA0A0
:1019F00005C0CFA0D8A402C0C12CD12C460130E133
:101A0000632E712C00E010E02E018CE0480E511C7A
:101A1000682D6170C2010E946CD39694879461E036
:101A2000C7010E946CD3000F111FC5010E945FD334
:101A30008111016060E0C7010E946CD381E0681AE7
:101A4000710831F780E1882E912C60E0C2010E947C
:101A50006CD361E0C7010E946CD3C5010E945FD3C3
:101A600060E0C7010E946CD381E0881A910869F791
:101A700060E0C7010E946CD38B8D813039F180F01A
:101A8000823009F041C040E951E062E0C80196951A
:101A90008795969587950E94D4D39E8F8D8F34C05D
:101AA0000F3F8FE7180709F415C040E951E061E0E6
:101AB000C8010E94D4D32D8D3E8D280F391F2139A6
:101AC00081E03807ECF438A32F8F17C00F3F8FE762
:101AD000180719F483E090E015C040E951E061E097
:101AE000C8010E94D4D32D8D3E8D280F391F213976
:101AF00081E038072CF43AA329A3198E188E04C06C
:101B000084E090E0998F888F8B8D89A71AA68A8DA3
:101B10008B8FDCA6CBA6813039F018F0823089F4A7
:101B20000CC081E08A8F0EC08C8D8F5F8C8F8837C0
:101B300020F01C8E82E08A8F04C01A8E02C080E0E2
:101B400001C081E0DF91CF911F910F91FF90EF9045
:101B5000DF90CF90BF90AF909F908F907F906F90CD
:101B60005F904F90089540E065E87AE180EA97E160
:101B70000C941DD34F925F926F927F92AF92BF925F
:101B8000CF92DF92EF92FF920F931F93CF93DF9349
:101B900000D0CDB7DEB75C01009709F448C06230D1
:101BA000710508F444C0DC0116964D905D906D906F
:101BB0007C901997660F771F73016201C60ED71EBE
:101BC000E11CF11CD501ED91FC910190F081E02D1B
:101BD00022E030E0AE014F5F5F4FC701B6010995CB
:101BE000882329F109811A8101151105F1F0C80135
:101BF00040960897E0F0083FBFEF1B0710F000E0A9
:101C000010E01A821982D501ED91FC910480F581D2
